 freetype

 Timestamp is ffffffff (Sun Feb  7 06:28:15 2106)

 Preferred load address is 10000000

 Start         Length     Name                   Class
 0001:00000000 00050fc4H .text$mn                CODE
 0002:00000000 000000d0H .idata$5                DATA
 0002:000000d0 00000004H .00cfg                  DATA
 0002:000000d4 00000004H .CRT$XCA                DATA
 0002:000000d8 00000004H .CRT$XCZ                DATA
 0002:000000dc 00000004H .CRT$XIA                DATA
 0002:000000e0 00000004H .CRT$XIZ                DATA
 0002:000000e4 00000004H .CRT$XPA                DATA
 0002:000000e8 00000004H .CRT$XPZ                DATA
 0002:000000ec 00000004H .CRT$XTA                DATA
 0002:000000f0 00000010H .CRT$XTZ                DATA
 0002:000000f4 00000000H .gfids$y                DATA
 0002:00000100 000171c0H .rdata                  DATA
 0002:000172c0 00000004H .rdata$sxdata           DATA
 0002:000172c4 00000288H .rdata$zzzdbg           DATA
 0002:0001754c 00000004H .rtc$IAA                DATA
 0002:00017550 00000004H .rtc$IZZ                DATA
 0002:00017554 00000004H .rtc$TAA                DATA
 0002:00017558 00000008H .rtc$TZZ                DATA
 0002:00017560 00000090H .xdata$x                DATA
 0002:000175f0 000014e8H .edata                  DATA
 0002:00018ad8 000000b4H .idata$2                DATA
 0002:00018b8c 00000014H .idata$3                DATA
 0002:00018ba0 000000d0H .idata$4                DATA
 0002:00018c70 000003daH .idata$6                DATA
 0003:00000000 00000028H .data                   DATA
 0003:00000028 0000036cH .bss                    DATA
 0004:00000000 00000060H .rsrc$01                DATA
 0004:00000060 00000328H .rsrc$02                DATA

  Address         Publics by Value              Rva+Base       Lib:Object

 0000:00000000       ___guard_eh_cont_table     00000000     <absolute>
 0000:00000000       ___AbsoluteZero            00000000     <absolute>
 0000:00000000       ___enclave_config          00000000     <absolute>
 0000:00000000       ___arm64x_redirection_metadata_count 00000000     <absolute>
 0000:00000000       ___hybrid_auxiliary_iat    00000000     <absolute>
 0000:00000000       ___arm64x_redirection_metadata 00000000     <absolute>
 0000:00000000       ___guard_iat_table         00000000     <absolute>
 0000:00000000       ___guard_eh_cont_count     00000000     <absolute>
 0000:00000000       ___arm64x_extra_rfe_table_size 00000000     <absolute>
 0000:00000000       ___guard_fids_table        00000000     <absolute>
 0000:00000000       ___x64_code_ranges_to_entry_points_count 00000000     <absolute>
 0000:00000000       ___arm64x_native_entrypoint 00000000     <absolute>
 0000:00000000       ___arm64x_extra_rfe_table  00000000     <absolute>
 0000:00000000       ___guard_longjmp_count     00000000     <absolute>
 0000:00000000       ___x64_code_ranges_to_entry_points 00000000     <absolute>
 0000:00000000       ___guard_fids_count        00000000     <absolute>
 0000:00000000       ___dynamic_value_reloc_table 00000000     <absolute>
 0000:00000000       ___volatile_metadata       00000000     <absolute>
 0000:00000000       ___hybrid_code_map         00000000     <absolute>
 0000:00000000       ___guard_longjmp_table     00000000     <absolute>
 0000:00000000       ___hybrid_code_map_count   00000000     <absolute>
 0000:00000000       ___guard_iat_count         00000000     <absolute>
 0000:00000001       ___safe_se_handler_count   00000001     <absolute>
 0000:00000100       ___guard_flags             00000100     <absolute>
 0000:00000000       ___ImageBase               10000000     <linker-defined>
 0001:00000000       _af_cjk_metrics_init       10001000 f   afcjk.obj
 0001:00000120       _af_cjk_metrics_scale      10001120 f   afcjk.obj
 0001:00000160       _af_cjk_hints_init         10001160 f   afcjk.obj
 0001:000001e0       _af_cjk_hints_apply        100011e0 f   afcjk.obj
 0001:000003d0       _af_cjk_get_standard_widths 100013d0 f   afcjk.obj
 0001:00001370       _af_cjk_metrics_check_digits 10002370 f   afcjk.obj
 0001:00001770       _af_cjk_metrics_init_widths 10002770 f   afcjk.obj
 0001:00002170       _af_face_globals_free      10003170 f   afglobal.obj
 0001:000021e0       _af_face_globals_get_metrics 100031e0 f   afglobal.obj
 0001:00002320       _af_face_globals_is_digit  10003320 f   afglobal.obj
 0001:00002340       _af_face_globals_new       10003340 f   afglobal.obj
 0001:00002460       _af_axis_hints_new_edge    10003460 f   afhints.obj
 0001:000025f0       _af_axis_hints_new_segment 100035f0 f   afhints.obj
 0001:00002700       _af_glyph_hints_align_edge_points 10003700 f   afhints.obj
 0001:000027c0       _af_glyph_hints_align_strong_points 100037c0 f   afhints.obj
 0001:000029b0       _af_glyph_hints_align_weak_points 100039b0 f   afhints.obj
 0001:00002bd0       _af_glyph_hints_done       10003bd0 f   afhints.obj
 0001:00002cc0       _af_glyph_hints_init       10003cc0 f   afhints.obj
 0001:00002ce0       _af_glyph_hints_reload     10003ce0 f   afhints.obj
 0001:000033c0       _af_glyph_hints_rescale    100043c0 f   afhints.obj
 0001:000033e0       _af_glyph_hints_save       100043e0 f   afhints.obj
 0001:00003560       _af_sort_and_quantize_widths 10004560 f   afhints.obj
 0001:00003840       _af_sort_pos               10004840 f   afhints.obj
 0001:00003910       _af_latin_metrics_init     10004910 f   aflatin.obj
 0001:00003a50       _af_latin_metrics_scale    10004a50 f   aflatin.obj
 0001:00003a90       _af_latin_get_standard_widths 10004a90 f   aflatin.obj
 0001:000048b0       _af_latin_hints_compute_edges 100058b0 f   aflatin.obj
 0001:00004cf0       _af_latin_hints_compute_segments 10005cf0 f   aflatin.obj
 0001:00005640       _af_latin_hints_link_segments 10006640 f   aflatin.obj
 0001:00006320       _af_latin_metrics_init_widths 10007320 f   aflatin.obj
 0001:00006a90       _af_loader_compute_darkening 10007a90 f   afloader.obj
 0001:00006cf0       _af_loader_done            10007cf0 f   afloader.obj
 0001:00006d10       _af_loader_init            10007d10 f   afloader.obj
 0001:00006d80       _af_loader_load_glyph      10007d80 f   afloader.obj
 0001:00007be0       _FT_Trace_Disable          10008be0 f   ftdebug.obj
 0001:00007be0       _FT_Set_Default_Log_Handler 10008be0 f   ftdebug.obj
 0001:00007be0       @_guard_check_icall_nop@4  10008be0 f   MSVCRT:guard_support.obj
 0001:00007be0       _ps_parser_done            10008be0 f   psobjs.obj
 0001:00007be0       _FT_Trace_Set_Level        10008be0 f   ftdebug.obj
 0001:00007be0       _cid_driver_done           10008be0 f   cidobjs.obj
 0001:00007be0       _FT_Set_Log_Handler        10008be0 f   ftdebug.obj
 0001:00007be0       _cff_driver_done           10008be0 f   cffobjs.obj
 0001:00007be0       _T1_Driver_Done            10008be0 f   t1objs.obj
 0001:00007be0       _FT_Trace_Enable           10008be0 f   ftdebug.obj
 0001:00007be0       _tt_driver_done            10008be0 f   ttobjs.obj
 0001:00007be0       _af_shaper_buf_destroy     10008be0 f   afshaper.obj
 0001:00007be0       _FT_Trace_Set_Default_Level 10008be0 f   ftdebug.obj
 0001:00008100       _afm_parser_done           10009100 f   afmparse.obj
 0001:00008120       _afm_parser_init           10009120 f   afmparse.obj
 0001:00008180       _afm_parser_parse          10009180 f   afmparse.obj
 0001:00008630       _afm_parser_read_vals      10009630 f   afmparse.obj
 0001:00008940       _af_shaper_get_cluster     10009940 f   afshaper.obj
 0001:00008a60       _af_shaper_get_coverage    10009a60 f   afshaper.obj
 0001:00008a60       ___scrt_stub_for_is_c_termination_complete 10009a60 f   MSVCRT:ucrt_stubs.obj
 0001:00008a60       __is_c_termination_complete 10009a60 f   MSVCRT:ucrt_stubs.obj
 0001:00008a70       _af_shaper_get_elem        10009a70 f   afshaper.obj
 0001:00008ad0       _cf2_arrstack_clear        10009ad0 f   psarrst.obj
 0001:00008c40       _cff_decoder_init          10009c40 f   cffdecode.obj
 0001:00008cf0       _cff_decoder_prepare       10009cf0 f   cffdecode.obj
 0001:00008dd0       _cff_lookup_glyph_by_stdcharcode 10009dd0 f   cffdecode.obj
 0001:00009730       _cff_free_glyph_data       1000a730 f   cffgload.obj
 0001:00009790       _cff_get_glyph_data        1000a790 f   cffgload.obj
 0001:000097f0       _cff_slot_load             1000a7f0 f   cffgload.obj
 0001:0000a220       _cff_blend_build_vector    1000b220 f   cffload.obj
 0001:0000a490       _cff_blend_check_vector    1000b490 f   cffload.obj
 0001:0000a510       _cff_blend_doBlend         1000b510 f   cffload.obj
 0001:0000a750       _cff_charset_cid_to_gindex 1000b750 f   cffload.obj
 0001:0000ab00       _cff_done_blend            1000bb00 f   cffload.obj
 0001:0000aeb0       _cff_fd_select_get         1000beb0 f   cffload.obj
 0001:0000af50       _cff_font_done             1000bf50 f   cffload.obj
 0001:0000b260       _cff_font_load             1000c260 f   cffload.obj
 0001:0000b940       _cff_get_standard_encoding 1000c940 f   cffload.obj
 0001:0000b960       _cff_get_var_blend         1000c960 f   cffload.obj
 0001:0000b980       _cff_index_access_element  1000c980 f   cffload.obj
 0001:0000bb20       _cff_index_forget_element  1000cb20 f   cffload.obj
 0001:0000bb40       _cff_index_get_name        1000cb40 f   cffload.obj
 0001:0000bd90       _cff_index_get_sid_string  1000cd90 f   cffload.obj
 0001:0000bde0       _cff_index_get_string      1000cde0 f   cffload.obj
 0001:0000c170       _cff_load_private_dict     1000d170 f   cffload.obj
 0001:0000cd80       _T1_Driver_Init            1000dd80 f   t1objs.obj
 0001:0000cd80       _cff_driver_init           1000dd80 f   cffobjs.obj
 0001:0000cd80       _cid_driver_init           1000dd80 f   cidobjs.obj
 0001:0000ce10       _cff_face_done             1000de10 f   cffobjs.obj
 0001:0000ce70       _cff_face_init             1000de70 f   cffobjs.obj
 0001:0000d9e0       _cff_size_done             1000e9e0 f   cffobjs.obj
 0001:0000da70       _cff_size_init             1000ea70 f   cffobjs.obj
 0001:0000dc50       _cff_size_request          1000ec50 f   cffobjs.obj
 0001:0000dec0       _cff_size_select           1000eec0 f   cffobjs.obj
 0001:0000dff0       _cid_slot_done             1000eff0 f   cidobjs.obj
 0001:0000dff0       _cff_slot_done             1000eff0 f   cffobjs.obj
 0001:0000e010       _cff_slot_init             1000f010 f   cffobjs.obj
 0001:0000e990       _cff_parse_num             1000f990 f   cffparse.obj
 0001:0000ed90       _cff_parser_done           1000fd90 f   cffparse.obj
 0001:0000edb0       _cff_parser_init           1000fdb0 f   cffparse.obj
 0001:0000ee60       _cff_parser_run            1000fe60 f   cffparse.obj
 0001:0000f660       _cid_slot_load_glyph       10010660 f   cidgload.obj
 0001:0000fd50       _cid_face_open             10010d50 f   cidload.obj
 0001:0000ffc0       _cid_get_offset            10010fc0 f   cidload.obj
 0001:00010760       _cid_face_done             10011760 f   cidobjs.obj
 0001:00010900       _cid_face_init             10011900 f   cidobjs.obj
 0001:00010b80       _cid_size_done             10011b80 f   cidobjs.obj
 0001:00010be0       _cid_size_init             10011be0 f   cidobjs.obj
 0001:00010c60       _cid_size_request          10011c60 f   cidobjs.obj
 0001:00010cd0       _cid_slot_init             10011cd0 f   cidobjs.obj
 0001:00010d20       _cid_parser_done           10011d20 f   cidparse.obj
 0001:00010d50       _cid_parser_new            10011d50 f   cidparse.obj
 0001:00011170       _FT_Get_Advance            10012170 f   ftadvanc.obj
 0001:00011200       _FT_Get_Advances           10012200 f   ftadvanc.obj
 0001:000115a0       _FT_Outline_Get_BBox       100125a0 f   ftbbox.obj
 0001:00011890       _FT_Bitmap_Blend           10012890 f   ftbitmap.obj
 0001:00011ed0       _FT_Bitmap_Convert         10012ed0 f   ftbitmap.obj
 0001:00012360       _FT_Bitmap_Copy            10013360 f   ftbitmap.obj
 0001:000124c0       _FT_Bitmap_Done            100134c0 f   ftbitmap.obj
 0001:00012510       _FT_Bitmap_Embolden        10013510 f   ftbitmap.obj
 0001:000127f0       _FT_Bitmap_Init            100137f0 f   ftbitmap.obj
 0001:000127f0       _FT_Bitmap_New             100137f0 f   ftbitmap.obj
 0001:00012810       _FT_GlyphSlot_Own_Bitmap   10013810 f   ftbitmap.obj
 0001:00012ae0       _FT_CeilFix                10013ae0 f   ftcalc.obj
 0001:00012af0       _FT_DivFix                 10013af0 f   ftcalc.obj
 0001:00012b90       _FT_FloorFix               10013b90 f   ftcalc.obj
 0001:00012ba0       _FT_Hypot                  10013ba0 f   ftcalc.obj
 0001:00012bc0       _FT_Matrix_Check           10013bc0 f   ftcalc.obj
 0001:00012dc0       _FT_Matrix_Invert          10013dc0 f   ftcalc.obj
 0001:00012e90       _FT_Matrix_Multiply        10013e90 f   ftcalc.obj
 0001:000130a0       _FT_Matrix_Multiply_Scaled 100140a0 f   ftcalc.obj
 0001:00013190       _FT_MulDiv                 10014190 f   ftcalc.obj
 0001:00013270       _FT_MulDiv_No_Round        10014270 f   ftcalc.obj
 0001:00013340       _FT_MulFix                 10014340 f   ftcalc.obj
 0001:00013370       _FT_RoundFix               10014370 f   ftcalc.obj
 0001:00013390       _FT_Vector_NormLen         10014390 f   ftcalc.obj
 0001:00013510       _FT_Vector_Transform_Scaled 10014510 f   ftcalc.obj
 0001:00013580       _ft_corner_is_flat         10014580 f   ftcalc.obj
 0001:00013640       _ft_corner_orientation     10014640 f   ftcalc.obj
 0001:00013680       _FT_Get_CID_From_Glyph_Index 10014680 f   ftcid.obj
 0001:000136e0       _FT_Get_CID_Is_Internally_CID_Keyed 100146e0 f   ftcid.obj
 0001:00013740       _FT_Get_CID_Registry_Ordering_Supplement 10014740 f   ftcid.obj
 0001:000137e0       _FT_Get_X11_Font_Format    100147e0 f   ftfntfmt.obj
 0001:000137e0       _FT_Get_Font_Format        100147e0 f   ftfntfmt.obj
 0001:00013810       _FT_Get_FSType_Flags       10014810 f   ftfstype.obj
 0001:00013880       _FT_Get_Gasp               10014880 f   ftgasp.obj
 0001:000138e0       _FT_GlyphLoader_Add        100148e0 f   ftgloadr.obj
 0001:00013ac0       _FT_GlyphLoader_CheckPoints 10014ac0 f   ftgloadr.obj
 0001:00013c50       _FT_GlyphLoader_CheckSubGlyphs 10014c50 f   ftgloadr.obj
 0001:00013cc0       _FT_GlyphLoader_CreateExtra 10014cc0 f   ftgloadr.obj
 0001:00013d20       _FT_GlyphLoader_Done       10014d20 f   ftgloadr.obj
 0001:00013d40       _FT_GlyphLoader_New        10014d40 f   ftgloadr.obj
 0001:00013d70       _FT_GlyphLoader_Prepare    10014d70 f   ftgloadr.obj
 0001:00013db0       _FT_GlyphLoader_Reset      10014db0 f   ftgloadr.obj
 0001:00013e50       _FT_GlyphLoader_Rewind     10014e50 f   ftgloadr.obj
 0001:000140b0       _FT_Done_Glyph             100150b0 f   ftglyph.obj
 0001:000140e0       _FT_Get_Glyph              100150e0 f   ftglyph.obj
 0001:00014200       _FT_Glyph_Copy             10015200 f   ftglyph.obj
 0001:000142c0       _FT_Glyph_Get_CBox         100152c0 f   ftglyph.obj
 0001:00014360       _FT_Glyph_To_Bitmap        10015360 f   ftglyph.obj
 0001:000145c0       _FT_Glyph_Transform        100155c0 f   ftglyph.obj
 0001:00014610       _FT_New_Glyph              10015610 f   ftglyph.obj
 0001:00015a10       _ft_hash_num_init          10016a10 f   fthash.obj
 0001:00015a60       _ft_hash_num_insert        10016a60 f   fthash.obj
 0001:00015a70       _ft_hash_num_lookup        10016a70 f   fthash.obj
 0001:00015a90       _ft_hash_str_free          10016a90 f   fthash.obj
 0001:00015cc0       _FT_Add_Default_Modules    10016cc0 f   ftinit.obj
 0001:00015cf0       _FT_Done_FreeType          10016cf0 f   ftinit.obj
 0001:00015d20       _FT_Init_FreeType          10016d20 f   ftinit.obj
 0001:00015d80       _FT_Set_Default_Properties 10016d80 f   ftinit.obj
 0001:00015fe0       _FT_Library_SetLcdFilterWeights 10016fe0 f   ftlcdfil.obj
 0001:00015fe0       _FT_Library_SetLcdFilter   10016fe0 f   ftlcdfil.obj
 0001:00015ff0       _FT_Library_SetLcdGeometry 10016ff0 f   ftlcdfil.obj
 0001:00016030       _ft_lcd_padding            10017030 f   ftlcdfil.obj
 0001:00016100       _FT_Done_MM_Var            10017100 f   ftmm.obj
 0001:00016120       _FT_Get_Var_Blend_Coordinates 10017120 f   ftmm.obj
 0001:00016120       _FT_Get_MM_Blend_Coordinates 10017120 f   ftmm.obj
 0001:000161b0       _FT_Get_MM_Var             100171b0 f   ftmm.obj
 0001:00016240       _FT_Get_MM_WeightVector    10017240 f   ftmm.obj
 0001:000162e0       _FT_Get_Multi_Master       100172e0 f   ftmm.obj
 0001:00016370       _FT_Get_Var_Axis_Flags     10017370 f   ftmm.obj
 0001:000163a0       _FT_Get_Var_Design_Coordinates 100173a0 f   ftmm.obj
 0001:00016430       _FT_Set_MM_Blend_Coordinates 10017430 f   ftmm.obj
 0001:00016430       _FT_Set_Var_Blend_Coordinates 10017430 f   ftmm.obj
 0001:00016530       _FT_Set_MM_Design_Coordinates 10017530 f   ftmm.obj
 0001:000165f0       _FT_Set_MM_WeightVector    100175f0 f   ftmm.obj
 0001:000166b0       _FT_Set_Named_Instance     100176b0 f   ftmm.obj
 0001:000167c0       _FT_Set_Var_Design_Coordinates 100177c0 f   ftmm.obj
 0001:00016940       _FT_Activate_Size          10017940 f   ftobjs.obj
 0001:00016970       _FT_Add_Module             10017970 f   ftobjs.obj
 0001:00016be0       _FT_Attach_File            10017be0 f   ftobjs.obj
 0001:00016ce0       _FT_Attach_Stream          10017ce0 f   ftobjs.obj
 0001:00016d70       _FT_CMap_New               10017d70 f   ftobjs.obj
 0001:00016e40       _FT_Done_Face              10017e40 f   ftobjs.obj
 0001:00016ec0       _FT_Done_GlyphSlot         10017ec0 f   ftobjs.obj
 0001:00016f20       _FT_Done_Library           10017f20 f   ftobjs.obj
 0001:000170b0       _FT_Done_Size              100180b0 f   ftobjs.obj
 0001:00017150       _FT_Face_GetCharVariantIndex 10018150 f   ftobjs.obj
 0001:000171a0       _FT_Face_GetCharVariantIsDefault 100181a0 f   ftobjs.obj
 0001:000171d0       _FT_Face_GetCharsOfVariant 100181d0 f   ftobjs.obj
 0001:00017210       _FT_Face_GetVariantSelectors 10018210 f   ftobjs.obj
 0001:00017240       _FT_Face_GetVariantsOfChar 10018240 f   ftobjs.obj
 0001:00017280       _FT_Face_Properties        10018280 f   ftobjs.obj
 0001:00017330       _FT_Get_CMap_Format        10018330 f   ftobjs.obj
 0001:00017380       _FT_Get_CMap_Language_ID   10018380 f   ftobjs.obj
 0001:000173d0       _FT_Get_Char_Index         100183d0 f   ftobjs.obj
 0001:00017400       _FT_Get_Charmap_Index      10018400 f   ftobjs.obj
 0001:00017440       _FT_Get_Color_Glyph_ClipBox 10018440 f   ftobjs.obj
 0001:00017480       _FT_Get_Color_Glyph_Layer  10018480 f   ftobjs.obj
 0001:000174e0       _FT_Get_Color_Glyph_Paint  100184e0 f   ftobjs.obj
 0001:00017520       _FT_Get_Colorline_Stops    10018520 f   ftobjs.obj
 0001:00017560       _FT_Get_First_Char         10018560 f   ftobjs.obj
 0001:000175e0       _FT_Get_Glyph_Name         100185e0 f   ftobjs.obj
 0001:00017690       _FT_Get_Kerning            10018690 f   ftobjs.obj
 0001:000177d0       _FT_Get_Module             100187d0 f   ftobjs.obj
 0001:00017840       _FT_Get_Module_Interface   10018840 f   ftobjs.obj
 0001:000178c0       _FT_Get_Name_Index         100188c0 f   ftobjs.obj
 0001:00017940       _FT_Get_Next_Char          10018940 f   ftobjs.obj
 0001:000179a0       _FT_Get_Paint              100189a0 f   ftobjs.obj
 0001:000179e0       _FT_Get_Paint_Layers       100189e0 f   ftobjs.obj
 0001:00017a20       _FT_Get_Postscript_Name    10018a20 f   ftobjs.obj
 0001:00017a90       _FT_Get_Renderer           10018a90 f   ftobjs.obj
 0001:00017ac0       _FT_Get_Sfnt_Table         10018ac0 f   ftobjs.obj
 0001:00017b00       _FT_Get_SubGlyph_Info      10018b00 f   ftobjs.obj
 0001:00017b70       _FT_Get_Track_Kerning      10018b70 f   ftobjs.obj
 0001:00017bd0       _FT_Get_Transform          10018bd0 f   ftobjs.obj
 0001:00017c00       _FT_Get_TrueType_Engine_Type 10018c00 f   ftobjs.obj
 0001:00017c90       _FT_Library_Version        10018c90 f   ftobjs.obj
 0001:00017cd0       _FT_Load_Char              10018cd0 f   ftobjs.obj
 0001:00017d10       _FT_Load_Glyph             10018d10 f   ftobjs.obj
 0001:000182d0       _FT_Load_Sfnt_Table        100192d0 f   ftobjs.obj
 0001:00018330       _FT_Lookup_Renderer        10019330 f   ftobjs.obj
 0001:00018380       _FT_Match_Size             10019380 f   ftobjs.obj
 0001:00018470       _FT_New_Face               10019470 f   ftobjs.obj
 0001:000184c0       _FT_New_GlyphSlot          100194c0 f   ftobjs.obj
 0001:000185e0       _FT_New_Library            100195e0 f   ftobjs.obj
 0001:00018650       _FT_New_Memory_Face        10019650 f   ftobjs.obj
 0001:000186a0       _FT_New_Size               100196a0 f   ftobjs.obj
 0001:000187b0       _FT_Open_Face              100197b0 f   ftobjs.obj
 0001:000187d0       _FT_Property_Get           100197d0 f   ftobjs.obj
 0001:000188a0       _FT_Property_Set           100198a0 f   ftobjs.obj
 0001:00018970       _FT_Reference_Face         10019970 f   ftobjs.obj
 0001:00018990       _FT_Reference_Library      10019990 f   ftobjs.obj
 0001:000189b0       _FT_Remove_Module          100199b0 f   ftobjs.obj
 0001:00018b10       _FT_Render_Glyph           10019b10 f   ftobjs.obj
 0001:00018b40       _FT_Render_Glyph_Internal  10019b40 f   ftobjs.obj
 0001:00018d30       _FT_Request_Metrics        10019d30 f   ftobjs.obj
 0001:00018fe0       _FT_Request_Size           10019fe0 f   ftobjs.obj
 0001:00019140       _FT_Select_Charmap         1001a140 f   ftobjs.obj
 0001:000191b0       _FT_Select_Metrics         1001a1b0 f   ftobjs.obj
 0001:00019250       _FT_Select_Size            1001a250 f   ftobjs.obj
 0001:00019340       _FT_Set_Char_Size          1001a340 f   ftobjs.obj
 0001:000193e0       _FT_Set_Charmap            1001a3e0 f   ftobjs.obj
 0001:00019480       _FT_Set_Debug_Hook         1001a480 f   ftobjs.obj
 0001:000194b0       _FT_Set_Pixel_Sizes        1001a4b0 f   ftobjs.obj
 0001:00019540       _FT_Set_Renderer           1001a540 f   ftobjs.obj
 0001:000195e0       _FT_Set_Transform          1001a5e0 f   ftobjs.obj
 0001:00019680       _FT_Sfnt_Table_Info        1001a680 f   ftobjs.obj
 0001:000196e0       _FT_Stream_Free            1001a6e0 f   ftobjs.obj
 0001:00019710       _FT_Stream_New             1001a710 f   ftobjs.obj
 0001:0001a0d0       _ft_glyphslot_alloc_bitmap 1001b0d0 f   ftobjs.obj
 0001:0001a1d0       _ft_glyphslot_preset_bitmap 1001b1d0 f   ftobjs.obj
 0001:0001a500       _ft_glyphslot_set_bitmap   1001b500 f   ftobjs.obj
 0001:0001a550       _ft_module_get_service     1001b550 f   ftobjs.obj
 0001:0001ad60       _ft_property_string_set    1001bd60 f   ftobjs.obj
 0001:0001af50       _ft_service_list_lookup    1001bf50 f   ftobjs.obj
 0001:0001afc0       _ft_synthesize_vertical_metrics 1001bfc0 f   ftobjs.obj
 0001:0001b020       _ft_validator_error        1001c020 f   ftobjs.obj
 0001:0001b040       _ft_validator_init         1001c040 f   ftobjs.obj
 0001:0001b3e0       _open_face_PS_from_sfnt_stream 1001c3e0 f   ftobjs.obj
 0001:0001b650       _open_face_from_buffer     1001c650 f   ftobjs.obj
 0001:0001b750       _FT_Outline_Check          1001c750 f   ftoutln.obj
 0001:0001b7b0       _FT_Outline_Copy           1001c7b0 f   ftoutln.obj
 0001:0001b850       _FT_Outline_Decompose      1001c850 f   ftoutln.obj
 0001:0001bc30       _FT_Outline_Done           1001cc30 f   ftoutln.obj
 0001:0001bcb0       _FT_Outline_Embolden       1001ccb0 f   ftoutln.obj
 0001:0001bcd0       _FT_Outline_EmboldenXY     1001ccd0 f   ftoutln.obj
 0001:0001c100       _FT_Outline_Get_Bitmap     1001d100 f   ftoutln.obj
 0001:0001c180       _FT_Outline_Get_CBox       1001d180 f   ftoutln.obj
 0001:0001c230       _FT_Outline_Get_Orientation 1001d230 f   ftoutln.obj
 0001:0001c480       _FT_Outline_New            1001d480 f   ftoutln.obj
 0001:0001c580       _FT_Outline_Render         1001d580 f   ftoutln.obj
 0001:0001c6a0       _FT_Outline_Reverse        1001d6a0 f   ftoutln.obj
 0001:0001c750       _FT_Outline_Transform      1001d750 f   ftoutln.obj
 0001:0001c790       _FT_Outline_Translate      1001d790 f   ftoutln.obj
 0001:0001c7d0       _FT_Vector_Transform       1001d7d0 f   ftoutln.obj
 0001:0001c8e0       _FT_Face_SetUnpatentedHinting 1001d8e0 f   ftpatent.obj
 0001:0001c8e0       _FT_Face_CheckTrueTypePatents 1001d8e0 f   ftpatent.obj
 0001:0001c8f0       _ps_property_get           1001d8f0 f   ftpsprop.obj
 0001:0001c9f0       _ps_property_set           1001d9f0 f   ftpsprop.obj
 0001:0001f2b0       _FT_Raccess_Get_DataOffsets 100202b0 f   ftrfork.obj
 0001:0001f530       _FT_Raccess_Get_HeaderInfo 10020530 f   ftrfork.obj
 0001:0001f7c0       _FT_Raccess_Guess          100207c0 f   ftrfork.obj
 0001:0001f860       _ft_raccess_rule_by_darwin_vfs 10020860 f   ftrfork.obj
 0001:00020200       _FT_Get_Sfnt_LangTag       10021200 f   ftsnames.obj
 0001:00020310       _FT_Get_Sfnt_Name          10021310 f   ftsnames.obj
 0001:00020420       _FT_Get_Sfnt_Name_Count    10021420 f   ftsnames.obj
 0001:00020440       _FT_Stream_Close           10021440 f   ftstream.obj
 0001:00020460       _FT_Stream_EnterFrame      10021460 f   ftstream.obj
 0001:00020550       _FT_Stream_ExitFrame       10021550 f   ftstream.obj
 0001:00020580       _FT_Stream_ExtractFrame    10021580 f   ftstream.obj
 0001:000205b0       _FT_Stream_GetByte         100215b0 f   ftstream.obj
 0001:000205d0       _FT_Stream_GetULong        100215d0 f   ftstream.obj
 0001:00020610       _FT_Stream_GetUShort       10021610 f   ftstream.obj
 0001:00020650       _FT_Stream_OpenMemory      10021650 f   ftstream.obj
 0001:00020680       _FT_Stream_Pos             10021680 f   ftstream.obj
 0001:00020690       _FT_Stream_Read            10021690 f   ftstream.obj
 0001:00020710       _FT_Stream_ReadAt          10021710 f   ftstream.obj
 0001:00020790       _FT_Stream_ReadByte        10021790 f   ftstream.obj
 0001:00020800       _FT_Stream_ReadFields      10021800 f   ftstream.obj
 0001:00020a30       _FT_Stream_ReadULong       10021a30 f   ftstream.obj
 0001:00020ab0       _FT_Stream_ReadULongLE     10021ab0 f   ftstream.obj
 0001:00020b30       _FT_Stream_ReadUShort      10021b30 f   ftstream.obj
 0001:00020bb0       _FT_Stream_ReleaseFrame    10021bb0 f   ftstream.obj
 0001:00020bf0       _FT_Stream_Seek            10021bf0 f   ftstream.obj
 0001:00020c30       _FT_Stream_Skip            10021c30 f   ftstream.obj
 0001:00020c80       _FT_Glyph_Stroke           10021c80 f   ftstroke.obj
 0001:00020dc0       _FT_Glyph_StrokeBorder     10021dc0 f   ftstroke.obj
 0001:00020f00       _FT_Outline_GetInsideBorder 10021f00 f   ftstroke.obj
 0001:00020f20       _FT_Outline_GetOutsideBorder 10021f20 f   ftstroke.obj
 0001:00020f40       _FT_Stroker_BeginSubPath   10021f40 f   ftstroke.obj
 0001:00020fa0       _FT_Stroker_ConicTo        10021fa0 f   ftstroke.obj
 0001:000215a0       _FT_Stroker_CubicTo        100225a0 f   ftstroke.obj
 0001:00021c10       _FT_Stroker_Done           10022c10 f   ftstroke.obj
 0001:00021cc0       _FT_Stroker_EndSubPath     10022cc0 f   ftstroke.obj
 0001:00021e40       _FT_Stroker_Export         10022e40 f   ftstroke.obj
 0001:00021e70       _FT_Stroker_ExportBorder   10022e70 f   ftstroke.obj
 0001:00021f60       _FT_Stroker_GetBorderCounts 10022f60 f   ftstroke.obj
 0001:00021fc0       _FT_Stroker_GetCounts      10022fc0 f   ftstroke.obj
 0001:00022040       _FT_Stroker_LineTo         10023040 f   ftstroke.obj
 0001:00022170       _FT_Stroker_New            10023170 f   ftstroke.obj
 0001:000221f0       _FT_Stroker_ParseOutline   100231f0 f   ftstroke.obj
 0001:00022560       _FT_Stroker_Rewind         10023560 f   ftstroke.obj
 0001:00022590       _FT_Stroker_Set            10023590 f   ftstroke.obj
 0001:00023370       _FT_GlyphSlot_Embolden     10024370 f   ftsynth.obj
 0001:00023470       _FT_GlyphSlot_Oblique      10024470 f   ftsynth.obj
 0001:000234d0       _FT_Done_Memory            100244d0 f   ftsystem.obj
 0001:000234e0       _FT_New_Memory             100244e0 f   ftsystem.obj
 0001:00023510       _FT_Stream_Open            10024510 f   ftsystem.obj
 0001:00023680       _FT_Angle_Diff             10024680 f   fttrigon.obj
 0001:000236f0       _FT_Atan2                  100246f0 f   fttrigon.obj
 0001:00023760       _FT_Cos                    10024760 f   fttrigon.obj
 0001:00023790       _FT_Sin                    10024790 f   fttrigon.obj
 0001:000237c0       _FT_Tan                    100247c0 f   fttrigon.obj
 0001:00023800       _FT_Vector_From_Polar      10024800 f   fttrigon.obj
 0001:00023830       _FT_Vector_Length          10024830 f   fttrigon.obj
 0001:000238b0       _FT_Vector_Polarize        100248b0 f   fttrigon.obj
 0001:00023940       _FT_Vector_Rotate          10024940 f   fttrigon.obj
 0001:00023a50       _FT_Vector_Unit            10024a50 f   fttrigon.obj
 0001:00023cd0       _FT_Get_PS_Font_Info       10024cd0 f   fttype1.obj
 0001:00023d20       _FT_Get_PS_Font_Private    10024d20 f   fttype1.obj
 0001:00023d70       _FT_Get_PS_Font_Value      10024d70 f   fttype1.obj
 0001:00023dc0       _FT_Has_PS_Glyph_Names     10024dc0 f   fttype1.obj
 0001:00023e00       _FT_List_Add               10024e00 f   ftutil.obj
 0001:00023e30       _FT_List_Finalize          10024e30 f   ftutil.obj
 0001:00023e90       _FT_List_Find              10024e90 f   ftutil.obj
 0001:00023ec0       _FT_List_Insert            10024ec0 f   ftutil.obj
 0001:00023ef0       _FT_List_Iterate           10024ef0 f   ftutil.obj
 0001:00023f40       _FT_List_Remove            10024f40 f   ftutil.obj
 0001:00023f70       _FT_List_Up                10024f70 f   ftutil.obj
 0001:00023fc0       _ft_mem_alloc              10024fc0 f   ftutil.obj
 0001:00024030       _ft_mem_free               10025030 f   ftutil.obj
 0001:00024050       _ft_mem_qalloc             10025050 f   ftutil.obj
 0001:000240a0       _ft_mem_qrealloc           100250a0 f   ftutil.obj
 0001:00024190       _ft_mem_realloc            10025190 f   ftutil.obj
 0001:000242b0       _ft_mem_strcpyn            100252b0 f   ftutil.obj
 0001:000242e0       _ft_mem_strdup             100252e0 f   ftutil.obj
 0001:00024370       _cf2_arrstack_finalize     10025370 f   psarrst.obj
 0001:000243a0       _cf2_arrstack_getBuffer    100253a0 f   psarrst.obj
 0001:000243b0       _cf2_arrstack_getPointer   100253b0 f   psarrst.obj
 0001:000243e0       _cf2_arrstack_init         100253e0 f   psarrst.obj
 0001:00024420       _cf2_arrstack_push         10025420 f   psarrst.obj
 0001:00024470       _cf2_arrstack_setCount     10025470 f   psarrst.obj
 0001:00024530       _cf2_arrstack_size         10025530 f   psarrst.obj
 0001:00024540       _cf2_blues_capture         10025540 f   psblues.obj
 0001:000246d0       _cf2_blues_init            100256d0 f   psblues.obj
 0001:00024c30       _PS_Conv_ASCIIHexDecode    10025c30 f   psconv.obj
 0001:00024ce0       _PS_Conv_EexecDecode       10025ce0 f   psconv.obj
 0001:00024d70       _PS_Conv_Strtol            10025d70 f   psconv.obj
 0001:00024e70       _PS_Conv_ToFixed           10025e70 f   psconv.obj
 0001:000250e0       _PS_Conv_ToInt             100260e0 f   psconv.obj
 0001:00025140       _cf2_setError              10026140 f   pserror.obj
 0001:000256b0       _cf2_getGlyphOutline       100266b0 f   psfont.obj
 0001:00025890       _cf2_decoder_parse_charstrings 10026890 f   psft.obj
 0001:00025bf0       _cf2_freeSeacComponent     10026bf0 f   psft.obj
 0001:00025c20       _cf2_freeT1SeacComponent   10026c20 f   psft.obj
 0001:00025ca0       _cf2_getBlueMetrics        10026ca0 f   psft.obj
 0001:00025cf0       _cf2_getBlueValues         10026cf0 f   psft.obj
 0001:00025d20       _cf2_getDefaultWidthX      10026d20 f   psft.obj
 0001:00025d40       _cf2_getFamilyBlues        10026d40 f   psft.obj
 0001:00025d70       _cf2_getFamilyOtherBlues   10026d70 f   psft.obj
 0001:00025da0       _cf2_getLanguageGroup      10026da0 f   psft.obj
 0001:00025dc0       _cf2_getMaxstack           10026dc0 f   psft.obj
 0001:00025de0       _cf2_getNominalWidthX      10026de0 f   psft.obj
 0001:00025e00       _cf2_getNormalizedVector   10026e00 f   psft.obj
 0001:00025e30       _cf2_getOtherBlues         10026e30 f   psft.obj
 0001:00025e60       _cf2_getPpemY              10026e60 f   psft.obj
 0001:00025e80       _cf2_getSeacComponent      10026e80 f   psft.obj
 0001:00025f10       _cf2_getStdHW              10026f10 f   psft.obj
 0001:00025f30       _cf2_getStdVW              10026f30 f   psft.obj
 0001:00025f50       _cf2_getSubfont            10026f50 f   psft.obj
 0001:00025f60       _cf2_getT1SeacComponent    10026f60 f   psft.obj
 0001:00025fe0       _cf2_getVStore             10026fe0 f   psft.obj
 0001:00025ff0       _cf2_initGlobalRegionBuffer 10026ff0 f   psft.obj
 0001:00026040       _cf2_initLocalRegionBuffer 10027040 f   psft.obj
 0001:000260e0       _cf2_outline_close         100270e0 f   psft.obj
 0001:00026100       _cf2_outline_reset         10027100 f   psft.obj
 0001:00026120       _ps_hints_apply            10027120 f   pshalgo.obj
 0001:000284a0       _psh_blues_snap_stem       100294a0 f   pshglob.obj
 0001:000285e0       _psh_globals_funcs_init    100295e0 f   pshglob.obj
 0001:00028950       _psh_globals_set_scale     10029950 f   pshglob.obj
 0001:000289d0       _cf2_glyphpath_closeOpenPath 100299d0 f   pshints.obj
 0001:00029170       _cf2_glyphpath_curveTo     1002a170 f   pshints.obj
 0001:00029360       _cf2_glyphpath_finalize    1002a360 f   pshints.obj
 0001:000294f0       _cf2_glyphpath_init        1002a4f0 f   pshints.obj
 0001:00029690       _cf2_glyphpath_lineTo      1002a690 f   pshints.obj
 0001:00029820       _cf2_glyphpath_moveTo      1002a820 f   pshints.obj
 0001:00029ec0       _cf2_hint_isBottom         1002aec0 f   pshints.obj
 0001:00029ed0       _cf2_hint_isTop            1002aed0 f   pshints.obj
 0001:00029ee0       _cf2_hint_isValid          1002aee0 f   pshints.obj
 0001:00029ef0       _cf2_hint_lock             1002aef0 f   pshints.obj
 0001:0002a140       _cf2_hintmap_build         1002b140 f   pshints.obj
 0001:0002a4f0       _cf2_hintmap_init          1002b4f0 f   pshints.obj
 0001:0002ae60       _ps_hints_done             1002be60 f   pshrec.obj
 0001:0002aee0       _ps_hints_init             1002bee0 f   pshrec.obj
 0001:0002b630       _t1_hints_funcs_init       1002c630 f   pshrec.obj
 0001:0002b700       _t2_hints_funcs_init       1002c700 f   pshrec.obj
 0001:0002bbb0       _cf2_hintmask_getMaskPtr   1002cbb0 f   psintrp.obj
 0001:0002bbc0       _cf2_hintmask_init         1002cbc0 f   psintrp.obj
 0001:0002bc00       _cf2_hintmask_isNew        1002cc00 f   psintrp.obj
 0001:0002bc10       _cf2_hintmask_isValid      1002cc10 f   psintrp.obj
 0001:0002bc80       _cf2_hintmask_setAll       1002cc80 f   psintrp.obj
 0001:0002bcf0       _cf2_hintmask_setNew       1002ccf0 f   psintrp.obj
 0001:0002bd00       _cf2_interpT2CharString    1002cd00 f   psintrp.obj
 0001:0002e900       _cff_builder_add_contour   1002f900 f   psobjs.obj
 0001:0002e970       _cff_builder_add_point     1002f970 f   psobjs.obj
 0001:0002e9c0       _cff_builder_add_point1    1002f9c0 f   psobjs.obj
 0001:0002ea30       _cff_builder_close_contour 1002fa30 f   psobjs.obj
 0001:0002ea30       _ps_builder_close_contour  1002fa30 f   psobjs.obj
 0001:0002ea30       _t1_builder_close_contour  1002fa30 f   psobjs.obj
 0001:0002eb10       _t1_builder_done           1002fb10 f   psobjs.obj
 0001:0002eb10       _ps_builder_done           1002fb10 f   psobjs.obj
 0001:0002eb10       _cff_builder_done          1002fb10 f   psobjs.obj
 0001:0002eb30       _cff_builder_init          1002fb30 f   psobjs.obj
 0001:0002ebf0       _cff_builder_start_point   1002fbf0 f   psobjs.obj
 0001:0002ecd0       _cff_check_points          1002fcd0 f   psobjs.obj
 0001:0002ecd0       _t1_builder_check_points   1002fcd0 f   psobjs.obj
 0001:0002ecd0       _ps_builder_check_points   1002fcd0 f   psobjs.obj
 0001:0002ed10       _cff_random                1002fd10 f   psobjs.obj
 0001:0002ed30       _ps_builder_add_point      1002fd30 f   psobjs.obj
 0001:0002ed80       _ps_builder_add_point1     1002fd80 f   psobjs.obj
 0001:0002edf0       _ps_builder_init           1002fdf0 f   psobjs.obj
 0001:0002eeb0       _ps_builder_start_point    1002feb0 f   psobjs.obj
 0001:0002efa0       _ps_decoder_init           1002ffa0 f   psobjs.obj
 0001:0002f130       _ps_parser_init            10030130 f   psobjs.obj
 0001:0002f180       _ps_parser_load_field      10030180 f   psobjs.obj
 0001:0002f610       _ps_parser_load_field_table 10030610 f   psobjs.obj
 0001:0002f740       _ps_parser_skip_PS_token   10030740 f   psobjs.obj
 0001:0002f880       _ps_parser_skip_spaces     10030880 f   psobjs.obj
 0001:0002f8a0       _ps_parser_to_bytes        100308a0 f   psobjs.obj
 0001:0002f930       _ps_parser_to_coord_array  10030930 f   psobjs.obj
 0001:0002fa30       _ps_parser_to_fixed        10030a30 f   psobjs.obj
 0001:0002fa50       _ps_parser_to_fixed_array  10030a50 f   psobjs.obj
 0001:0002fa80       _ps_parser_to_int          10030a80 f   psobjs.obj
 0001:0002faa0       _ps_parser_to_token        10030aa0 f   psobjs.obj
 0001:0002fbd0       _ps_parser_to_token_array  10030bd0 f   psobjs.obj
 0001:0002fdb0       _ps_table_add              10030db0 f   psobjs.obj
 0001:0002fe60       _ps_table_done             10030e60 f   psobjs.obj
 0001:0002fe80       _ps_table_new              10030e80 f   psobjs.obj
 0001:0002ff80       _ps_table_release          10030f80 f   psobjs.obj
 0001:00030450       _t1_builder_add_contour    10031450 f   psobjs.obj
 0001:000304d0       _t1_builder_add_point      100314d0 f   psobjs.obj
 0001:00030530       _t1_builder_add_point1     10031530 f   psobjs.obj
 0001:000305b0       _t1_builder_init           100315b0 f   psobjs.obj
 0001:00030670       _t1_builder_start_point    10031670 f   psobjs.obj
 0001:00030770       _t1_decrypt                10031770 f   psobjs.obj
 0001:000307a0       _t1_make_subfont           100317a0 f   psobjs.obj
 0001:000309c0       _cf2_buf_isEnd             100319c0 f   psread.obj
 0001:000309d0       _cf2_buf_readByte          100319d0 f   psread.obj
 0001:00030a00       _cf2_stack_clear           10031a00 f   psstack.obj
 0001:00030a10       _cf2_stack_count           10031a10 f   psstack.obj
 0001:00030a20       _cf2_stack_free            10031a20 f   psstack.obj
 0001:00030a50       _cf2_stack_getReal         10031a50 f   psstack.obj
 0001:00030ab0       _cf2_stack_init            10031ab0 f   psstack.obj
 0001:00030b30       _cf2_stack_pop             10031b30 f   psstack.obj
 0001:00030b70       _cf2_stack_popFixed        10031b70 f   psstack.obj
 0001:00030bc0       _cf2_stack_popInt          10031bc0 f   psstack.obj
 0001:00030c10       _cf2_stack_pushFixed       10031c10 f   psstack.obj
 0001:00030c50       _cf2_stack_pushInt         10031c50 f   psstack.obj
 0001:00030c90       _cf2_stack_roll            10031c90 f   psstack.obj
 0001:00030db0       _cf2_stack_setReal         10031db0 f   psstack.obj
 0001:00031d40       _sfnt_done_face            10032d40 f   sfobjs.obj
 0001:00031f60       _sfnt_init_face            10032f60 f   sfobjs.obj
 0001:00032600       _sfnt_load_face            10033600 f   sfobjs.obj
 0001:00032fd0       _tt_face_get_name          10033fd0 f   sfobjs.obj
 0001:00033300       _T1_Done_Metrics           10034300 f   t1afm.obj
 0001:00033350       _T1_Get_Kerning            10034350 f   t1afm.obj
 0001:000333d0       _T1_Get_Track_Kerning      100343d0 f   t1afm.obj
 0001:00033460       _T1_Read_Metrics           10034460 f   t1afm.obj
 0001:00033cb0       _t1_decoder_done           10034cb0 f   t1decode.obj
 0001:00033cf0       _t1_decoder_init           10034cf0 f   t1decode.obj
 0001:00033d90       _t1_decoder_parse_metrics  10034d90 f   t1decode.obj
 0001:00034250       _t1_lookup_glyph_by_stdcharcode_ps 10035250 f   t1decode.obj
 0001:00034fb0       _T1_Compute_Max_Advance    10035fb0 f   t1gload.obj
 0001:00035110       _T1_Get_Advances           10036110 f   t1gload.obj
 0001:000352b0       _T1_Load_Glyph             100362b0 f   t1gload.obj
 0001:00037050       _T1_Done_Blend             10038050 f   t1load.obj
 0001:000371b0       _T1_Get_MM_Blend           100381b0 f   t1load.obj
 0001:00037250       _T1_Get_MM_Var             10038250 f   t1load.obj
 0001:00037500       _T1_Get_MM_WeightVector    10038500 f   t1load.obj
 0001:00037580       _T1_Get_Multi_Master       10038580 f   t1load.obj
 0001:000375f0       _T1_Get_Var_Design         100385f0 f   t1load.obj
 0001:000376b0       _T1_Open_Face              100386b0 f   t1load.obj
 0001:00037c50       _T1_Reset_MM_Blend         10038c50 f   t1load.obj
 0001:00037c70       _T1_Set_MM_Blend           10038c70 f   t1load.obj
 0001:00037cb0       _T1_Set_MM_Design          10038cb0 f   t1load.obj
 0001:00037e10       _T1_Set_MM_WeightVector    10038e10 f   t1load.obj
 0001:00037ee0       _T1_Set_Var_Design         10038ee0 f   t1load.obj
 0001:00038a20       _T1_Face_Done              10039a20 f   t1objs.obj
 0001:00038c20       _T1_Face_Init              10039c20 f   t1objs.obj
 0001:00039000       _T1_GlyphSlot_Done         1003a000 f   t1objs.obj
 0001:00039020       _T1_GlyphSlot_Init         1003a020 f   t1objs.obj
 0001:00039070       _T1_Size_Done              1003a070 f   t1objs.obj
 0001:000390d0       _T1_Size_Init              1003a0d0 f   t1objs.obj
 0001:00039140       _T1_Size_Request           1003a140 f   t1objs.obj
 0001:000391b0       _T1_Finalize_Parser        1003a1b0 f   t1parse.obj
 0001:00039200       _T1_Get_Private_Dict       1003a200 f   t1parse.obj
 0001:00039620       _T1_New_Parser             1003a620 f   t1parse.obj
 0001:0003cd40       _tt_face_build_cmaps       1003dd40 f   ttcmap.obj
 0001:0003cf90       _tt_get_cmap_info          1003df90 f   ttcmap.obj
 0001:0003d780       _tt_face_colr_blend_layer  1003e780 f   ttcolr.obj
 0001:0003db90       _tt_face_free_colr         1003eb90 f   ttcolr.obj
 0001:0003dbc0       _tt_face_get_color_glyph_clipbox 1003ebc0 f   ttcolr.obj
 0001:0003ded0       _tt_face_get_colorline_stops 1003eed0 f   ttcolr.obj
 0001:0003df60       _tt_face_get_colr_glyph_paint 1003ef60 f   ttcolr.obj
 0001:0003e030       _tt_face_get_colr_layer    1003f030 f   ttcolr.obj
 0001:0003e170       _tt_face_get_paint         1003f170 f   ttcolr.obj
 0001:0003e2c0       _tt_face_get_paint_layers  1003f2c0 f   ttcolr.obj
 0001:0003e370       _tt_face_load_colr         1003f370 f   ttcolr.obj
 0001:0003e6e0       _tt_face_free_cpal         1003f6e0 f   ttcpal.obj
 0001:0003e710       _tt_face_load_cpal         1003f710 f   ttcpal.obj
 0001:0003ebe0       _tt_face_palette_set       1003fbe0 f   ttcpal.obj
 0001:0003f0f0       _TT_Get_HMetrics           100400f0 f   ttgload.obj
 0001:0003f120       _TT_Get_VMetrics           10040120 f   ttgload.obj
 0001:0003f480       _TT_Init_Glyph_Loading     10040480 f   ttgload.obj
 0001:0003f730       _TT_Load_Glyph             10040730 f   ttgload.obj
 0001:00042120       _TT_Get_MM_Blend           10043120 f   ttgxvar.obj
 0001:000421c0       _TT_Get_MM_Var             100431c0 f   ttgxvar.obj
 0001:00042810       _TT_Get_Var_Design         10043810 f   ttgxvar.obj
 0001:000428b0       _TT_Set_MM_Blend           100438b0 f   ttgxvar.obj
 0001:000428f0       _TT_Set_Named_Instance     100438f0 f   ttgxvar.obj
 0001:000429d0       _TT_Set_Var_Design         100439d0 f   ttgxvar.obj
 0001:00042ba0       _TT_Vary_Apply_Glyph_Deltas 10043ba0 f   ttgxvar.obj
 0001:000451a0       _tt_apply_mvar             100461a0 f   ttgxvar.obj
 0001:00045420       _tt_done_blend             10046420 f   ttgxvar.obj
 0001:000455e0       _tt_face_vary_cvt          100465e0 f   ttgxvar.obj
 0001:00045ba0       _tt_get_var_blend          10046ba0 f   ttgxvar.obj
 0001:00045c30       _tt_hadvance_adjust        10046c30 f   ttgxvar.obj
 0001:00046190       _tt_vadvance_adjust        10047190 f   ttgxvar.obj
 0001:00047d90       _TT_Clear_CodeRange        10048d90 f   ttinterp.obj
 0001:00047db0       _TT_Done_Context           10048db0 f   ttinterp.obj
 0001:00047f20       _TT_Goto_CodeRange         10048f20 f   ttinterp.obj
 0001:00047f60       _TT_Load_Context           10048f60 f   ttinterp.obj
 0001:000482b0       _TT_New_Context            100492b0 f   ttinterp.obj
 0001:00048320       _TT_RunIns                 10049320 f   ttinterp.obj
 0001:0004b0d0       _TT_Run_Context            1004c0d0 f   ttinterp.obj
 0001:0004b1c0       _TT_Save_Context           1004c1c0 f   ttinterp.obj
 0001:0004b250       _TT_Set_CodeRange          1004c250 f   ttinterp.obj
 0001:0004b270       _Update_Max                1004c270 f   ttinterp.obj
 0001:0004b4c0       _tt_face_done_kern         1004c4c0 f   ttkern.obj
 0001:0004b510       _tt_face_get_kerning       1004c510 f   ttkern.obj
 0001:0004b730       _tt_face_load_kern         1004c730 f   ttkern.obj
 0001:0004bb10       _tt_face_free_name         1004cb10 f   ttload.obj
 0001:0004bbf0       _tt_face_goto_table        1004cbf0 f   ttload.obj
 0001:0004bc50       _tt_face_load_any          1004cc50 f   ttload.obj
 0001:0004bcb0       _tt_face_load_bhed         1004ccb0 f   ttload.obj
 0001:0004bcf0       _tt_face_load_cmap         1004ccf0 f   ttload.obj
 0001:0004bd40       _tt_face_load_font_dir     1004cd40 f   ttload.obj
 0001:0004bf70       _tt_face_load_gasp         1004cf70 f   ttload.obj
 0001:0004c0b0       _tt_face_load_head         1004d0b0 f   ttload.obj
 0001:0004c0f0       _tt_face_load_maxp         1004d0f0 f   ttload.obj
 0001:0004c180       _tt_face_load_name         1004d180 f   ttload.obj
 0001:0004c480       _tt_face_load_os2          1004d480 f   ttload.obj
 0001:0004c520       _tt_face_load_pclt         1004d520 f   ttload.obj
 0001:0004c560       _tt_face_load_post         1004d560 f   ttload.obj
 0001:0004c5d0       _tt_face_lookup_table      1004d5d0 f   ttload.obj
 0001:0004c610       _tt_face_get_metrics       1004d610 f   ttmtx.obj
 0001:0004c7e0       _tt_face_load_hhea         1004d7e0 f   ttmtx.obj
 0001:0004c850       _tt_face_load_hmtx         1004d850 f   ttmtx.obj
 0001:0004caf0       _tt_driver_init            1004daf0 f   ttobjs.obj
 0001:0004cb00       _tt_face_done              1004db00 f   ttobjs.obj
 0001:0004cbb0       _tt_face_init              1004dbb0 f   ttobjs.obj
 0001:0004cee0       _tt_glyphzone_done         1004dee0 f   ttobjs.obj
 0001:0004cf50       _tt_size_done              1004df50 f   ttobjs.obj
 0001:0004d070       _tt_size_init              1004e070 f   ttobjs.obj
 0001:0004d530       _tt_size_ready_bytecode    1004e530 f   ttobjs.obj
 0001:0004d7b0       _tt_size_reset             1004e7b0 f   ttobjs.obj
 0001:0004d9e0       _tt_size_run_prep          1004e9e0 f   ttobjs.obj
 0001:0004db70       _tt_slot_init              1004eb70 f   ttobjs.obj
 0001:0004dbb0       _tt_face_done_loca         1004ebb0 f   ttpload.obj
 0001:0004dbe0       _tt_face_free_hdmx         1004ebe0 f   ttpload.obj
 0001:0004dc20       _tt_face_get_device_metrics 1004ec20 f   ttpload.obj
 0001:0004dc80       _tt_face_get_location      1004ec80 f   ttpload.obj
 0001:0004dd90       _tt_face_load_cvt          1004ed90 f   ttpload.obj
 0001:0004de80       _tt_face_load_fpgm         1004ee80 f   ttpload.obj
 0001:0004dee0       _tt_face_load_hdmx         1004eee0 f   ttpload.obj
 0001:0004e070       _tt_face_load_loca         1004f070 f   ttpload.obj
 0001:0004e1e0       _tt_face_load_prep         1004f1e0 f   ttpload.obj
 0001:0004e640       _tt_face_free_ps_names     1004f640 f   ttpost.obj
 0001:0004e720       _tt_face_get_ps_name       1004f720 f   ttpost.obj
 0001:0004e850       _tt_face_free_sbit         1004f850 f   ttsbit.obj
 0001:0004e890       _tt_face_load_sbit         1004f890 f   ttsbit.obj
 0001:0004ec40       _tt_face_load_sbit_image   1004fc40 f   ttsbit.obj
 0001:0004f0c0       _tt_face_load_strike_metrics 100500c0 f   ttsbit.obj
 0001:0004f360       _tt_face_set_sbit_strike   10050360 f   ttsbit.obj
 0001:0004fff2       @__security_check_cookie@4 10050ff2 f   MSVCRT:secchk.obj
 0001:00050010       __chkstk                   10051010 f   MSVCRT:chkstk.obj
 0001:00050010       __alloca_probe             10051010 f   MSVCRT:chkstk.obj
 0001:00050040       __allmul                   10051040 f   MSVCRT:llmul.obj
 0001:00050080       __aulldiv                  10051080 f   MSVCRT:ulldiv.obj
 0001:000500f0       __alldiv                   100510f0 f   MSVCRT:lldiv.obj
 0001:000501a0       __allshl                   100511a0 f   MSVCRT:llshl.obj
 0001:000501bf       ___raise_securityfailure   100511bf f   MSVCRT:gs_report.obj
 0001:000501e7       ___report_gsfailure        100511e7 f   MSVCRT:gs_report.obj
 0001:000502e0       ___report_rangecheckfailure 100512e0 f   MSVCRT:gs_report.obj
 0001:000502ec       ___report_securityfailure  100512ec f   MSVCRT:gs_report.obj
 0001:000506fa       __DllMainCRTStartup@12     100516fa f   MSVCRT:dll_dllmain.obj
 0001:0005076a       ___security_init_cookie    1005176a f   MSVCRT:gs_support.obj
 0001:000507b5       _DllMain@12                100517b5 f   MSVCRT:dll_dllmain_stub.obj
 0001:000507d7       ?__scrt_initialize_type_info@@YAXXZ 100517d7 f   MSVCRT:tncleanup.obj
 0001:000507e3       ?__scrt_uninitialize_type_info@@YAXXZ 100517e3 f   MSVCRT:tncleanup.obj
 0001:000507ef       ___local_stdio_printf_options 100517ef f i MSVCRT:default_local_stdio_options.obj
 0001:000507f5       ___local_stdio_scanf_options 100517f5 f i MSVCRT:default_local_stdio_options.obj
 0001:000507fb       ___scrt_initialize_default_local_stdio_options 100517fb f   MSVCRT:default_local_stdio_options.obj
 0001:0005085c       ___scrt_acquire_startup_lock 1005185c f   MSVCRT:utility.obj
 0001:0005088e       ___scrt_dllmain_after_initialize_c 1005188e f   MSVCRT:utility.obj
 0001:000508b9       ___scrt_dllmain_before_initialize_c 100518b9 f   MSVCRT:utility.obj
 0001:000508c7       ___scrt_dllmain_crt_thread_attach 100518c7 f   MSVCRT:utility.obj
 0001:000508e6       ___scrt_dllmain_crt_thread_detach 100518e6 f   MSVCRT:utility.obj
 0001:000508f3       ___scrt_dllmain_exception_filter 100518f3 f   MSVCRT:utility.obj
 0001:00050927       ___scrt_dllmain_uninitialize_c 10051927 f   MSVCRT:utility.obj
 0001:0005094a       ___scrt_dllmain_uninitialize_critical 1005194a f   MSVCRT:utility.obj
 0001:00050957       ___scrt_initialize_crt     10051957 f   MSVCRT:utility.obj
 0001:00050990       ___scrt_initialize_onexit_tables 10051990 f   MSVCRT:utility.obj
 0001:00050a17       ___scrt_is_nonwritable_in_current_image 10051a17 f   MSVCRT:utility.obj
 0001:00050aab       ___scrt_release_startup_lock 10051aab f   MSVCRT:utility.obj
 0001:00050ac8       ___scrt_uninitialize_crt   10051ac8 f   MSVCRT:utility.obj
 0001:00050af0       ___scrt_get_dyn_tls_init_callback 10051af0 f   MSVCRT:dyn_tls_init.obj
 0001:00050af6       ___scrt_fastfail           10051af6 f   MSVCRT:utility_desktop.obj
 0001:00050c10       __crt_debugger_hook        10051c10 f   MSVCRT:utility_desktop.obj
 0001:00050c18       __RTC_Initialize           10051c18 f   MSVCRT:initsect.obj
 0001:00050c44       __RTC_Terminate            10051c44 f   MSVCRT:initsect.obj
 0001:00050c70       __SEH_prolog4              10051c70 f   MSVCRT:sehprolg4.obj
 0001:00050cb4       __SEH_epilog4              10051cb4 f   MSVCRT:sehprolg4.obj
 0001:00050cc8       __except_handler4          10051cc8 f   MSVCRT:chandler4gs.obj
 0001:00050cf7       ___isa_available_init      10051cf7 f   MSVCRT:cpu_disp.obj
 0001:00050ec7       __get_startup_argv_mode    10051ec7 f   MSVCRT:argv_mode.obj
 0001:00050ecb       ___scrt_is_ucrt_dll_in_use 10051ecb f   MSVCRT:ucrt_detection.obj
 0001:00050ed7       _IsProcessorFeaturePresent@4 10051ed7 f   kernel32:KERNEL32.dll
 0001:00050edd       _memset                    10051edd f   vcruntime:VCRUNTIME140.dll
 0001:00050ee3       _memcpy                    10051ee3 f   vcruntime:VCRUNTIME140.dll
 0001:00050ee9       _strstr                    10051ee9 f   vcruntime:VCRUNTIME140.dll
 0001:00050eef       _memmove                   10051eef f   vcruntime:VCRUNTIME140.dll
 0001:00050ef5       _longjmp                   10051ef5 f   vcruntime:VCRUNTIME140.dll
 0001:00050efb       __setjmp3                  10051efb f   vcruntime:VCRUNTIME140.dll
 0001:00050f01       _strrchr                   10051f01 f   vcruntime:VCRUNTIME140.dll
 0001:00050f07       _memchr                    10051f07 f   vcruntime:VCRUNTIME140.dll
 0001:00050f0d       ___std_type_info_destroy_list 10051f0d f   vcruntime:VCRUNTIME140.dll
 0001:00050f13       __except_handler4_common   10051f13 f   vcruntime:VCRUNTIME140.dll
 0001:00050f19       __initterm                 10051f19 f   ucrt:api-ms-win-crt-runtime-l1-1-0.dll
 0001:00050f1f       __initterm_e               10051f1f f   ucrt:api-ms-win-crt-runtime-l1-1-0.dll
 0001:00050f25       __seh_filter_dll           10051f25 f   ucrt:api-ms-win-crt-runtime-l1-1-0.dll
 0001:00050f2b       __configure_narrow_argv    10051f2b f   ucrt:api-ms-win-crt-runtime-l1-1-0.dll
 0001:00050f31       __initialize_narrow_environment 10051f31 f   ucrt:api-ms-win-crt-runtime-l1-1-0.dll
 0001:00050f37       __initialize_onexit_table  10051f37 f   ucrt:api-ms-win-crt-runtime-l1-1-0.dll
 0001:00050f3d       __execute_onexit_table     10051f3d f   ucrt:api-ms-win-crt-runtime-l1-1-0.dll
 0001:00050f43       __cexit                    10051f43 f   ucrt:api-ms-win-crt-runtime-l1-1-0.dll
 0001:00050f49       ___vcrt_initialize         10051f49 f   MSVCRT:ucrt_stubs.obj
 0001:00050f49       ___acrt_thread_attach      10051f49 f   MSVCRT:ucrt_stubs.obj
 0001:00050f49       ___scrt_stub_for_acrt_thread_detach 10051f49 f   MSVCRT:ucrt_stubs.obj
 0001:00050f49       ___scrt_stub_for_acrt_thread_attach 10051f49 f   MSVCRT:ucrt_stubs.obj
 0001:00050f49       ___vcrt_thread_attach      10051f49 f   MSVCRT:ucrt_stubs.obj
 0001:00050f49       ___vcrt_uninitialize       10051f49 f   MSVCRT:ucrt_stubs.obj
 0001:00050f49       ___vcrt_uninitialize_critical 10051f49 f   MSVCRT:ucrt_stubs.obj
 0001:00050f49       ___scrt_stub_for_acrt_uninitialize 10051f49 f   MSVCRT:ucrt_stubs.obj
 0001:00050f49       ___scrt_stub_for_acrt_initialize 10051f49 f   MSVCRT:ucrt_stubs.obj
 0001:00050f49       ___acrt_thread_detach      10051f49 f   MSVCRT:ucrt_stubs.obj
 0001:00050f49       ___acrt_initialize         10051f49 f   MSVCRT:ucrt_stubs.obj
 0001:00050f49       ___acrt_uninitialize       10051f49 f   MSVCRT:ucrt_stubs.obj
 0001:00050f49       ___vcrt_thread_detach      10051f49 f   MSVCRT:ucrt_stubs.obj
 0001:00050f49       ___scrt_stub_for_acrt_uninitialize_critical 10051f49 f   MSVCRT:ucrt_stubs.obj
 0001:00050f49       ___acrt_uninitialize_critical 10051f49 f   MSVCRT:ucrt_stubs.obj
 0001:00050f4c       __filter_x86_sse2_floating_point_exception 10051f4c f   MSVCRT:x86_exception_filter.obj
 0001:00050f4c       __filter_x86_sse2_floating_point_exception_default 10051f4c f   MSVCRT:x86_exception_filter.obj
 0002:00000000       __imp__UnhandledExceptionFilter@4 10052000     kernel32:KERNEL32.dll
 0002:00000004       __imp__SetUnhandledExceptionFilter@4 10052004     kernel32:KERNEL32.dll
 0002:00000008       __imp__GetCurrentProcess@0 10052008     kernel32:KERNEL32.dll
 0002:0000000c       __imp__TerminateProcess@8  1005200c     kernel32:KERNEL32.dll
 0002:00000010       __imp__IsProcessorFeaturePresent@4 10052010     kernel32:KERNEL32.dll
 0002:00000014       __imp__QueryPerformanceCounter@4 10052014     kernel32:KERNEL32.dll
 0002:00000018       __imp__GetCurrentProcessId@0 10052018     kernel32:KERNEL32.dll
 0002:0000001c       __imp__GetCurrentThreadId@0 1005201c     kernel32:KERNEL32.dll
 0002:00000020       __imp__GetSystemTimeAsFileTime@4 10052020     kernel32:KERNEL32.dll
 0002:00000024       __imp__DisableThreadLibraryCalls@4 10052024     kernel32:KERNEL32.dll
 0002:00000028       __imp__InitializeSListHead@4 10052028     kernel32:KERNEL32.dll
 0002:0000002c       __imp__IsDebuggerPresent@0 1005202c     kernel32:KERNEL32.dll
 0002:00000030       \177KERNEL32_NULL_THUNK_DATA 10052030     kernel32:KERNEL32.dll
 0002:00000034       __imp__memset              10052034     vcruntime:VCRUNTIME140.dll
 0002:00000038       __imp__memcpy              10052038     vcruntime:VCRUNTIME140.dll
 0002:0000003c       __imp__strstr              1005203c     vcruntime:VCRUNTIME140.dll
 0002:00000040       __imp__memmove             10052040     vcruntime:VCRUNTIME140.dll
 0002:00000044       __imp__longjmp             10052044     vcruntime:VCRUNTIME140.dll
 0002:00000048       __imp___setjmp3            10052048     vcruntime:VCRUNTIME140.dll
 0002:0000004c       __imp__strrchr             1005204c     vcruntime:VCRUNTIME140.dll
 0002:00000050       __imp__memchr              10052050     vcruntime:VCRUNTIME140.dll
 0002:00000054       __imp____std_type_info_destroy_list 10052054     vcruntime:VCRUNTIME140.dll
 0002:00000058       __imp___except_handler4_common 10052058     vcruntime:VCRUNTIME140.dll
 0002:0000005c       \177VCRUNTIME140_NULL_THUNK_DATA 1005205c     vcruntime:VCRUNTIME140.dll
 0002:00000060       __imp__strtol              10052060     ucrt:api-ms-win-crt-convert-l1-1-0.dll
 0002:00000064       \177api-ms-win-crt-convert-l1-1-0_NULL_THUNK_DATA 10052064     ucrt:api-ms-win-crt-convert-l1-1-0.dll
 0002:00000068       __imp__getenv              10052068     ucrt:api-ms-win-crt-environment-l1-1-0.dll
 0002:0000006c       \177api-ms-win-crt-environment-l1-1-0_NULL_THUNK_DATA 1005206c     ucrt:api-ms-win-crt-environment-l1-1-0.dll
 0002:00000070       __imp__malloc              10052070     ucrt:api-ms-win-crt-heap-l1-1-0.dll
 0002:00000074       __imp__realloc             10052074     ucrt:api-ms-win-crt-heap-l1-1-0.dll
 0002:00000078       __imp__free                10052078     ucrt:api-ms-win-crt-heap-l1-1-0.dll
 0002:0000007c       \177api-ms-win-crt-heap-l1-1-0_NULL_THUNK_DATA 1005207c     ucrt:api-ms-win-crt-heap-l1-1-0.dll
 0002:00000080       __imp___cexit              10052080     ucrt:api-ms-win-crt-runtime-l1-1-0.dll
 0002:00000084       __imp___initterm           10052084     ucrt:api-ms-win-crt-runtime-l1-1-0.dll
 0002:00000088       __imp___initterm_e         10052088     ucrt:api-ms-win-crt-runtime-l1-1-0.dll
 0002:0000008c       __imp___seh_filter_dll     1005208c     ucrt:api-ms-win-crt-runtime-l1-1-0.dll
 0002:00000090       __imp___configure_narrow_argv 10052090     ucrt:api-ms-win-crt-runtime-l1-1-0.dll
 0002:00000094       __imp___initialize_narrow_environment 10052094     ucrt:api-ms-win-crt-runtime-l1-1-0.dll
 0002:00000098       __imp___initialize_onexit_table 10052098     ucrt:api-ms-win-crt-runtime-l1-1-0.dll
 0002:0000009c       __imp___execute_onexit_table 1005209c     ucrt:api-ms-win-crt-runtime-l1-1-0.dll
 0002:000000a0       \177api-ms-win-crt-runtime-l1-1-0_NULL_THUNK_DATA 100520a0     ucrt:api-ms-win-crt-runtime-l1-1-0.dll
 0002:000000a4       __imp__ftell               100520a4     ucrt:api-ms-win-crt-stdio-l1-1-0.dll
 0002:000000a8       __imp__fseek               100520a8     ucrt:api-ms-win-crt-stdio-l1-1-0.dll
 0002:000000ac       __imp__fread               100520ac     ucrt:api-ms-win-crt-stdio-l1-1-0.dll
 0002:000000b0       __imp__fopen               100520b0     ucrt:api-ms-win-crt-stdio-l1-1-0.dll
 0002:000000b4       __imp__fclose              100520b4     ucrt:api-ms-win-crt-stdio-l1-1-0.dll
 0002:000000b8       \177api-ms-win-crt-stdio-l1-1-0_NULL_THUNK_DATA 100520b8     ucrt:api-ms-win-crt-stdio-l1-1-0.dll
 0002:000000bc       __imp__strncpy             100520bc     ucrt:api-ms-win-crt-string-l1-1-0.dll
 0002:000000c0       __imp__strncmp             100520c0     ucrt:api-ms-win-crt-string-l1-1-0.dll
 0002:000000c4       \177api-ms-win-crt-string-l1-1-0_NULL_THUNK_DATA 100520c4     ucrt:api-ms-win-crt-string-l1-1-0.dll
 0002:000000c8       __imp__qsort               100520c8     ucrt:api-ms-win-crt-utility-l1-1-0.dll
 0002:000000cc       \177api-ms-win-crt-utility-l1-1-0_NULL_THUNK_DATA 100520cc     ucrt:api-ms-win-crt-utility-l1-1-0.dll
 0002:000000d0       ___guard_check_icall_fptr  100520d0     MSVCRT:guard_support.obj
 0002:000000d4       ___xc_a                    100520d4     MSVCRT:initializers.obj
 0002:000000d8       ___xc_z                    100520d8     MSVCRT:initializers.obj
 0002:000000dc       ___xi_a                    100520dc     MSVCRT:initializers.obj
 0002:000000e0       ___xi_z                    100520e0     MSVCRT:initializers.obj
 0002:000000e4       ___xp_a                    100520e4     MSVCRT:initializers.obj
 0002:000000e8       ___xp_z                    100520e8     MSVCRT:initializers.obj
 0002:000000ec       ___xt_a                    100520ec     MSVCRT:initializers.obj
 0002:000000f0       ___xt_z                    100520f0     MSVCRT:initializers.obj
 0002:00000100       _af_blue_strings           10052100     afblue.obj
 0002:000016a0       _af_blue_stringsets        100536a0     afblue.obj
 0002:00001ee8       _af_cjk_writing_system_class 10053ee8     afcjk.obj
 0002:00001f08       ??_C@_0BE@MOFLNEOP@0?51?52?53?54?55?56?57?58?59@ 10053f08     afcjk.obj
 0002:00001f20       __xmm@00000000000000000001000000010000 10053f20     afcjk.obj
 0002:00001f30       _af_dummy_writing_system_class 10053f30     afdummy.obj
 0002:00001f50       _af_writing_system_classes 10053f50     afglobal.obj
 0002:00001f64       _af_adlm_script_class      10053f64     afglobal.obj
 0002:00001f78       _af_arab_script_class      10053f78     afglobal.obj
 0002:00001f8c       _af_armn_script_class      10053f8c     afglobal.obj
 0002:00001fa0       _af_avst_script_class      10053fa0     afglobal.obj
 0002:00001fb4       _af_bamu_script_class      10053fb4     afglobal.obj
 0002:00001fc8       _af_beng_script_class      10053fc8     afglobal.obj
 0002:00001fdc       _af_buhd_script_class      10053fdc     afglobal.obj
 0002:00001ff0       _af_cakm_script_class      10053ff0     afglobal.obj
 0002:00002004       _af_cans_script_class      10054004     afglobal.obj
 0002:00002018       _af_cari_script_class      10054018     afglobal.obj
 0002:0000202c       _af_cher_script_class      1005402c     afglobal.obj
 0002:00002040       _af_copt_script_class      10054040     afglobal.obj
 0002:00002054       _af_cprt_script_class      10054054     afglobal.obj
 0002:00002068       _af_cyrl_script_class      10054068     afglobal.obj
 0002:0000207c       _af_deva_script_class      1005407c     afglobal.obj
 0002:00002090       _af_dsrt_script_class      10054090     afglobal.obj
 0002:000020a4       _af_ethi_script_class      100540a4     afglobal.obj
 0002:000020b8       _af_geor_script_class      100540b8     afglobal.obj
 0002:000020cc       _af_geok_script_class      100540cc     afglobal.obj
 0002:000020e0       _af_glag_script_class      100540e0     afglobal.obj
 0002:000020f4       _af_goth_script_class      100540f4     afglobal.obj
 0002:00002108       _af_grek_script_class      10054108     afglobal.obj
 0002:0000211c       _af_gujr_script_class      1005411c     afglobal.obj
 0002:00002130       _af_guru_script_class      10054130     afglobal.obj
 0002:00002144       _af_hebr_script_class      10054144     afglobal.obj
 0002:00002158       _af_kali_script_class      10054158     afglobal.obj
 0002:0000216c       _af_khmr_script_class      1005416c     afglobal.obj
 0002:00002180       _af_khms_script_class      10054180     afglobal.obj
 0002:00002194       _af_knda_script_class      10054194     afglobal.obj
 0002:000021a8       _af_lao_script_class       100541a8     afglobal.obj
 0002:000021bc       _af_latn_script_class      100541bc     afglobal.obj
 0002:000021d0       _af_latb_script_class      100541d0     afglobal.obj
 0002:000021e4       _af_latp_script_class      100541e4     afglobal.obj
 0002:000021f8       _af_lisu_script_class      100541f8     afglobal.obj
 0002:0000220c       _af_mlym_script_class      1005420c     afglobal.obj
 0002:00002220       _af_medf_script_class      10054220     afglobal.obj
 0002:00002234       _af_mong_script_class      10054234     afglobal.obj
 0002:00002248       _af_mymr_script_class      10054248     afglobal.obj
 0002:0000225c       _af_nkoo_script_class      1005425c     afglobal.obj
 0002:00002270       _af_none_script_class      10054270     afglobal.obj
 0002:00002284       _af_olck_script_class      10054284     afglobal.obj
 0002:00002298       _af_orkh_script_class      10054298     afglobal.obj
 0002:000022ac       _af_osge_script_class      100542ac     afglobal.obj
 0002:000022c0       _af_osma_script_class      100542c0     afglobal.obj
 0002:000022d4       _af_rohg_script_class      100542d4     afglobal.obj
 0002:000022e8       _af_saur_script_class      100542e8     afglobal.obj
 0002:000022fc       _af_shaw_script_class      100542fc     afglobal.obj
 0002:00002310       _af_sinh_script_class      10054310     afglobal.obj
 0002:00002324       _af_sund_script_class      10054324     afglobal.obj
 0002:00002338       _af_taml_script_class      10054338     afglobal.obj
 0002:0000234c       _af_tavt_script_class      1005434c     afglobal.obj
 0002:00002360       _af_telu_script_class      10054360     afglobal.obj
 0002:00002374       _af_tfng_script_class      10054374     afglobal.obj
 0002:00002388       _af_thai_script_class      10054388     afglobal.obj
 0002:0000239c       _af_vaii_script_class      1005439c     afglobal.obj
 0002:000023b0       _af_limb_script_class      100543b0     afglobal.obj
 0002:000023c4       _af_orya_script_class      100543c4     afglobal.obj
 0002:000023d8       _af_sylo_script_class      100543d8     afglobal.obj
 0002:000023ec       _af_tibt_script_class      100543ec     afglobal.obj
 0002:00002400       _af_hani_script_class      10054400     afglobal.obj
 0002:00002414       _af_adlm_dflt_style_class  10054414     afglobal.obj
 0002:00002428       _af_script_classes         10054428     afglobal.obj
 0002:0000251c       _af_arab_dflt_style_class  1005451c     afglobal.obj
 0002:00002530       _af_armn_dflt_style_class  10054530     afglobal.obj
 0002:00002544       _af_avst_dflt_style_class  10054544     afglobal.obj
 0002:00002558       _af_bamu_dflt_style_class  10054558     afglobal.obj
 0002:0000256c       _af_beng_dflt_style_class  1005456c     afglobal.obj
 0002:00002580       _af_buhd_dflt_style_class  10054580     afglobal.obj
 0002:00002594       _af_cakm_dflt_style_class  10054594     afglobal.obj
 0002:000025a8       _af_cans_dflt_style_class  100545a8     afglobal.obj
 0002:000025bc       _af_cari_dflt_style_class  100545bc     afglobal.obj
 0002:000025d0       _af_cher_dflt_style_class  100545d0     afglobal.obj
 0002:000025e4       _af_copt_dflt_style_class  100545e4     afglobal.obj
 0002:000025f8       _af_cprt_dflt_style_class  100545f8     afglobal.obj
 0002:0000260c       _af_cyrl_c2cp_style_class  1005460c     afglobal.obj
 0002:00002620       _af_cyrl_c2sc_style_class  10054620     afglobal.obj
 0002:00002634       _af_cyrl_ordn_style_class  10054634     afglobal.obj
 0002:00002648       _af_cyrl_pcap_style_class  10054648     afglobal.obj
 0002:0000265c       _af_cyrl_sinf_style_class  1005465c     afglobal.obj
 0002:00002670       _af_cyrl_smcp_style_class  10054670     afglobal.obj
 0002:00002684       _af_cyrl_subs_style_class  10054684     afglobal.obj
 0002:00002698       _af_cyrl_sups_style_class  10054698     afglobal.obj
 0002:000026ac       _af_cyrl_titl_style_class  100546ac     afglobal.obj
 0002:000026c0       _af_cyrl_dflt_style_class  100546c0     afglobal.obj
 0002:000026d4       _af_deva_dflt_style_class  100546d4     afglobal.obj
 0002:000026e8       _af_dsrt_dflt_style_class  100546e8     afglobal.obj
 0002:000026fc       _af_ethi_dflt_style_class  100546fc     afglobal.obj
 0002:00002710       _af_geor_dflt_style_class  10054710     afglobal.obj
 0002:00002724       _af_geok_dflt_style_class  10054724     afglobal.obj
 0002:00002738       _af_glag_dflt_style_class  10054738     afglobal.obj
 0002:0000274c       _af_goth_dflt_style_class  1005474c     afglobal.obj
 0002:00002760       _af_grek_c2cp_style_class  10054760     afglobal.obj
 0002:00002774       _af_grek_c2sc_style_class  10054774     afglobal.obj
 0002:00002788       _af_grek_ordn_style_class  10054788     afglobal.obj
 0002:0000279c       _af_grek_pcap_style_class  1005479c     afglobal.obj
 0002:000027b0       _af_grek_sinf_style_class  100547b0     afglobal.obj
 0002:000027c4       _af_grek_smcp_style_class  100547c4     afglobal.obj
 0002:000027d8       _af_grek_subs_style_class  100547d8     afglobal.obj
 0002:000027ec       _af_grek_sups_style_class  100547ec     afglobal.obj
 0002:00002800       _af_grek_titl_style_class  10054800     afglobal.obj
 0002:00002814       _af_grek_dflt_style_class  10054814     afglobal.obj
 0002:00002828       _af_gujr_dflt_style_class  10054828     afglobal.obj
 0002:0000283c       _af_guru_dflt_style_class  1005483c     afglobal.obj
 0002:00002850       _af_hebr_dflt_style_class  10054850     afglobal.obj
 0002:00002864       _af_kali_dflt_style_class  10054864     afglobal.obj
 0002:00002878       _af_khmr_dflt_style_class  10054878     afglobal.obj
 0002:0000288c       _af_khms_dflt_style_class  1005488c     afglobal.obj
 0002:000028a0       _af_knda_dflt_style_class  100548a0     afglobal.obj
 0002:000028b4       _af_lao_dflt_style_class   100548b4     afglobal.obj
 0002:000028c8       _af_latn_c2cp_style_class  100548c8     afglobal.obj
 0002:000028dc       _af_latn_c2sc_style_class  100548dc     afglobal.obj
 0002:000028f0       _af_latn_ordn_style_class  100548f0     afglobal.obj
 0002:00002904       _af_latn_pcap_style_class  10054904     afglobal.obj
 0002:00002918       _af_latn_sinf_style_class  10054918     afglobal.obj
 0002:0000292c       _af_latn_smcp_style_class  1005492c     afglobal.obj
 0002:00002940       _af_latn_subs_style_class  10054940     afglobal.obj
 0002:00002954       _af_latn_sups_style_class  10054954     afglobal.obj
 0002:00002968       _af_latn_titl_style_class  10054968     afglobal.obj
 0002:0000297c       _af_latn_dflt_style_class  1005497c     afglobal.obj
 0002:00002990       _af_latb_dflt_style_class  10054990     afglobal.obj
 0002:000029a4       _af_latp_dflt_style_class  100549a4     afglobal.obj
 0002:000029b8       _af_lisu_dflt_style_class  100549b8     afglobal.obj
 0002:000029cc       _af_mlym_dflt_style_class  100549cc     afglobal.obj
 0002:000029e0       _af_medf_dflt_style_class  100549e0     afglobal.obj
 0002:000029f4       _af_mong_dflt_style_class  100549f4     afglobal.obj
 0002:00002a08       _af_mymr_dflt_style_class  10054a08     afglobal.obj
 0002:00002a1c       _af_nkoo_dflt_style_class  10054a1c     afglobal.obj
 0002:00002a30       _af_none_dflt_style_class  10054a30     afglobal.obj
 0002:00002a44       _af_olck_dflt_style_class  10054a44     afglobal.obj
 0002:00002a58       _af_orkh_dflt_style_class  10054a58     afglobal.obj
 0002:00002a6c       _af_osge_dflt_style_class  10054a6c     afglobal.obj
 0002:00002a80       _af_osma_dflt_style_class  10054a80     afglobal.obj
 0002:00002a94       _af_rohg_dflt_style_class  10054a94     afglobal.obj
 0002:00002aa8       _af_saur_dflt_style_class  10054aa8     afglobal.obj
 0002:00002abc       _af_shaw_dflt_style_class  10054abc     afglobal.obj
 0002:00002ad0       _af_sinh_dflt_style_class  10054ad0     afglobal.obj
 0002:00002ae4       _af_sund_dflt_style_class  10054ae4     afglobal.obj
 0002:00002af8       _af_taml_dflt_style_class  10054af8     afglobal.obj
 0002:00002b0c       _af_tavt_dflt_style_class  10054b0c     afglobal.obj
 0002:00002b20       _af_telu_dflt_style_class  10054b20     afglobal.obj
 0002:00002b34       _af_tfng_dflt_style_class  10054b34     afglobal.obj
 0002:00002b48       _af_thai_dflt_style_class  10054b48     afglobal.obj
 0002:00002b5c       _af_vaii_dflt_style_class  10054b5c     afglobal.obj
 0002:00002b70       _af_limb_dflt_style_class  10054b70     afglobal.obj
 0002:00002b84       _af_orya_dflt_style_class  10054b84     afglobal.obj
 0002:00002b98       _af_sylo_dflt_style_class  10054b98     afglobal.obj
 0002:00002bac       _af_tibt_dflt_style_class  10054bac     afglobal.obj
 0002:00002bc0       _af_hani_dflt_style_class  10054bc0     afglobal.obj
 0002:00002bd8       _af_style_classes          10054bd8     afglobal.obj
 0002:00002d38       ??_C@_09JDCNEMGL@?p?$JO?$KE?$IM?5?p?$JO?$KE?$KO@ 10054d38     afglobal.obj
 0002:00002d44       ??_C@_08NGKNFCCA@?Y?$IE?5?X?$KN?5?Y?$IA@ 10054d44     afglobal.obj
 0002:00002d50       ??_C@_05EBMEKBIG@?U?$LN?5?U?$IN@ 10054d50     afglobal.obj
 0002:00002d58       ??_C@_04JHGFHPIP@?p?$JA?$KM?$JK@ 10054d58     afglobal.obj
 0002:00002d60       ??_C@_07BADEIFOL@?j?$JL?$IB?5?j?$JL?$KP@ 10054d60     afglobal.obj
 0002:00002d68       ??_C@_07MLCFGLFO@?$OA?$KH?$KG?5?$OA?$KH?$KK@ 10054d68     afglobal.obj
 0002:00002d70       ??_C@_07MJBNFAPA@?a?$JN?$IL?5?a?$JN?$IP@ 10054d70     afglobal.obj
 0002:00002d78       ??_C@_0P@LMDGGGAE@?p?$JB?$IE?$KE?5?p?$JB?$IE?$IJ?5?p?$JB?$IE?$JL@ 10054d78     afglobal.obj
 0002:00002d88       ??_C@_07COJDMBCC@?a?$JB?$IM?5?a?$JD?$JK@ 10054d88     afglobal.obj
 0002:00002d90       ??_C@_09LEACCEAE@?p?$JA?$IK?$KL?5?p?$JA?$IL?$IJ@ 10054d90     afglobal.obj
 0002:00002d9c       ??_C@_0M@IIEFPKGE@?a?$IO?$KE?5?a?$IP?$IF?5?j?$KO?$JF@ 10054d9c     afglobal.obj
 0002:00002da8       ??_C@_07EGBKDBCM@?b?$LC?$JO?5?b?$LC?$JP@ 10054da8     afglobal.obj
 0002:00002db0       ??_C@_09BIEFHNHC@?p?$JA?$KA?$IF?5?p?$JA?$KA?$KD@ 10054db0     afglobal.obj
 0002:00002dbc       ??_C@_05DBINMJJM@?P?$LO?5?P?$JO@ 10054dbc     afglobal.obj
 0002:00002dc4       ??_C@_0M@ODJHCGEP@?$OA?$KE?$KA?5?$OA?$KE?$LF?5?$OA?$KE?$JP@ 10054dc4     afglobal.obj
 0002:00002dd0       ??_C@_09JIAMNMOE@?p?$JA?$JA?$IE?5?p?$JA?$JA?$KM@ 10054dd0     afglobal.obj
 0002:00002ddc       ??_C@_03CMFJHIMF@?a?$IL?$JA@ 10054ddc     afglobal.obj
 0002:00002de0       ??_C@_0BA@HEGJLNGN@?a?$ID?$JI?5?a?$ID?$JE?5?a?$ID?$JA?5?a?$LC?$LP@ 10054de0     afglobal.obj
 0002:00002df0       ??_C@_0M@CHIIFMEI@?a?$IC?$LG?5?a?$IC?$LB?5?b?$LE?$JJ@ 10054df0     afglobal.obj
 0002:00002dfc       ??_C@_07JCJJEEE@?b?$LA?$JF?5?b?$LB?$IF@ 10054dfc     afglobal.obj
 0002:00002e04       ??_C@_0P@OLAOOJHK@?p?$JA?$IM?$LE?5?p?$JA?$IM?$LO?5?p?$JA?$IN?$ID@ 10054e04     afglobal.obj
 0002:00002e14       ??_C@_05DKJCDMPM@?N?$LP?5?N?$JP@ 10054e14     afglobal.obj
 0002:00002e1c       ??_C@_07CMCIOKJD@?$OA?$KK?$JP?5?$OA?$KL?$KG@ 10054e1c     afglobal.obj
 0002:00002e24       ??_C@_0M@HILMFBKG@?$OA?$KI?$KA?5?$OA?$KI?$LA?5?$OA?$KJ?$KG@ 10054e24     afglobal.obj
 0002:00002e30       ??_C@_02EMJHPBAP@?W?$JN@   10054e30     afglobal.obj
 0002:00002e34       ??_C@_07EPGAKOL@?j?$KE?$IN?5?j?$KE?$IA@ 10054e34     afglobal.obj
 0002:00002e3c       ??_C@_03OIDAEFJK@?a?$JP?$KA@ 10054e3c     afglobal.obj
 0002:00002e40       ??_C@_07KCDGDMBN@?a?$KH?$KB?5?a?$KH?$KK@ 10054e40     afglobal.obj
 0002:00002e48       ??_C@_07BEADBFJO@?$OA?$LD?$KG?5?$OA?$LC?$KM@ 10054e48     afglobal.obj
 0002:00002e50       ??_C@_03LAIOPKDA@?$OA?$LL?$JA@ 10054e50     afglobal.obj
 0002:00002e54       ??_C@_05FCCCPEKP@o?5O?50@  10054e54     afglobal.obj
 0002:00002e5c       ??_C@_07HAIKLPAL@?b?$IC?$JC?5?b?$IC?$IA@ 10054e5c     afglobal.obj
 0002:00002e64       ??_C@_0M@HBKEJKFL@?a?$LF?$JC?5?a?$LE?$LM?5?b?$IB?$LA@ 10054e64     afglobal.obj
 0002:00002e70       ??_C@_03FHMEHKGN@?j?$JD?$LD@ 10054e70     afglobal.obj
 0002:00002e74       ??_C@_07PMBMNIKD@?$OA?$LE?$KA?5?$OA?$LE?$LB@ 10054e74     afglobal.obj
 0002:00002e7c       ??_C@_0P@IBKLCNIK@?p?$JG?$LJ?$KB?5?p?$JG?$LJ?$JL?5?p?$JG?$LJ?$KP@ 10054e7c     afglobal.obj
 0002:00002e8c       ??_C@_07EFJBGIDK@?a?$KB?$IC?5?a?$KA?$KK@ 10054e8c     afglobal.obj
 0002:00002e94       ??_C@_0M@JDJALDKB@?a?$IA?$JN?5?a?$IA?$IE?5?a?$IA?$IC@ 10054e94     afglobal.obj
 0002:00002ea0       ??_C@_05HGAHDEFN@?$NP?$IL?5?$NP?$IA@ 10054ea0     afglobal.obj
 0002:00002ea6       ??_C@_00CNPNBAHC@@         10054ea6     afglobal.obj
 0002:00002ea8       ??_C@_03OGFBMBEI@?a?$LB?$JL@ 10054ea8     afglobal.obj
 0002:00002eac       ??_C@_04DHPHFLNG@?p?$JA?$LA?$JH@ 10054eac     afglobal.obj
 0002:00002eb4       ??_C@_09CBEPPHOC@?p?$JA?$JD?$IC?5?p?$JA?$JD?$KK@ 10054eb4     afglobal.obj
 0002:00002ec0       ??_C@_09OCIHFBNC@?p?$JA?$JC?$IG?5?p?$JA?$JC?$KA@ 10054ec0     afglobal.obj
 0002:00002ecc       ??_C@_04OKDLEBGP@?p?$JA?$LE?$LA@ 10054ecc     afglobal.obj
 0002:00002ed4       ??_C@_07CLHNDJJO@?j?$KC?$JN?5?j?$KD?$JA@ 10054ed4     afglobal.obj
 0002:00002edc       ??_C@_04LANBAAGA@?p?$JA?$JB?$LE@ 10054edc     afglobal.obj
 0002:00002ee4       ??_C@_03CIFBMJFH@?$OA?$LG?$KH@ 10054ee4     afglobal.obj
 0002:00002ee8       ??_C@_03IHFLNIGM@?a?$KO?$LA@ 10054ee8     afglobal.obj
 0002:00002eec       ??_C@_03CCLNGAOJ@?$OA?$KP?$KG@ 10054eec     afglobal.obj
 0002:00002ef0       ??_C@_07NKKHBBJL@?j?$KK?$JC?5?j?$KK?$KL@ 10054ef0     afglobal.obj
 0002:00002ef8       ??_C@_07GCCOGDCF@?$OA?$LB?$KG?5?$OA?$LB?$KH@ 10054ef8     afglobal.obj
 0002:00002f00       ??_C@_03HEHFNKLF@?b?$LF?$JE@ 10054f00     afglobal.obj
 0002:00002f04       ??_C@_0M@PFDFPHNJ@?$OA?$LI?$LC?5?$OA?$LJ?$IF?5?$OA?$LJ?$JA@ 10054f04     afglobal.obj
 0002:00002f10       ??_C@_0M@BIKJPOHA@?j?$JI?$JD?5?j?$JG?$JM?5?j?$JG?$LE@ 10054f10     afglobal.obj
 0002:00002f1c       ??_C@_01FMEDJKGI@o@        10054f1c     afglobal.obj
 0002:00002f20       ??_C@_07PNKDJIHG@?g?$JE?$LA?5?e?$JL?$JH@ 10054f20     afglobal.obj
 0002:00002f28       _af_indic_writing_system_class 10054f28     afindic.obj
 0002:00002f48       _af_latin_writing_system_class 10054f48     aflatin.obj
 0002:00002f68       _af_autofitter_interface   10054f68     afmodule.obj
 0002:00002f78       _autofit_module_class      10054f78     afmodule.obj
 0002:00002fb4       ??_C@_0L@CIHKIEFA@properties@ 10054fb4     afmodule.obj
 0002:00002fc0       ??_C@_0L@MNEBCNMP@autofitter@ 10054fc0     afmodule.obj
 0002:00002fcc       ??_C@_0BA@OKOILHEH@fallback?9script@ 10054fcc     afmodule.obj
 0002:00002fdc       ??_C@_0P@PHBNIPOP@default?9script@ 10054fdc     afmodule.obj
 0002:00002fec       ??_C@_0BC@OOHNGIJD@increase?9x?9height@ 10054fec     afmodule.obj
 0002:00003000       ??_C@_0BF@GIDENNON@darkening?9parameters@ 10055000     afmodule.obj
 0002:00003018       ??_C@_0BC@GFOLLGHN@no?9stem?9darkening@ 10055018     afmodule.obj
 0002:0000302c       ??_C@_0BE@CELKBFDM@glyph?9to?9script?9map@ 1005502c     afmodule.obj
 0002:00003168       ??_C@_08NBPEBJDA@Ascender@ 10055168     afmparse.obj
 0002:00003174       ??_C@_09POOBGNPO@AxisLabel@ 10055174     afmparse.obj
 0002:00003180       ??_C@_08KLONHBMG@AxisType@ 10055180     afmparse.obj
 0002:0000318c       ??_C@_01HMGJMAIH@B@        1005518c     afmparse.obj
 0002:00003190       ??_C@_0P@LEAACMFJ@BlendAxisTypes@ 10055190     afmparse.obj
 0002:000031a0       ??_C@_0P@FPDIEJKK@BlendDesignMap@ 100551a0     afmparse.obj
 0002:000031b0       ??_C@_0BF@BEKHBPMN@BlendDesignPositions@ 100551b0     afmparse.obj
 0002:000031c8       ??_C@_01GFHCPBMG@C@        100551c8     afmparse.obj
 0002:000031cc       ??_C@_02KJDGAJLC@CC@       100551cc     afmparse.obj
 0002:000031d0       ??_C@_02EKMCNAHJ@CH@       100551d0     afmparse.obj
 0002:000031d4       ??_C@_09JOCJHGEG@CapHeight@ 100551d4     afmparse.obj
 0002:000031e0       ??_C@_09CGMEAFLF@CharWidth@ 100551e0     afmparse.obj
 0002:000031ec       ??_C@_0N@LHPDLMAH@CharacterSet@ 100551ec     afmparse.obj
 0002:000031fc       ??_C@_0L@EMODJLOD@Characters@ 100551fc     afmparse.obj
 0002:00003208       ??_C@_09JMDLBBJN@Descender@ 10055208     afmparse.obj
 0002:00003214       ??_C@_0P@JNPLONMI@EncodingScheme@ 10055214     afmparse.obj
 0002:00003224       ??_C@_07DLEALFPL@EndAxis@  10055224     afmparse.obj
 0002:0000322c       ??_C@_0P@GFNMGKCM@EndCharMetrics@ 1005522c     afmparse.obj
 0002:0000323c       ??_C@_0O@JABMALCH@EndComposites@ 1005523c     afmparse.obj
 0002:0000324c       ??_C@_0N@FNMEONKF@EndDirection@ 1005524c     afmparse.obj
 0002:0000325c       ??_C@_0P@FGFFCKLI@EndFontMetrics@ 1005525c     afmparse.obj
 0002:0000326c       ??_C@_0M@HKHGIIOM@EndKernData@ 1005526c     afmparse.obj
 0002:00003278       ??_C@_0N@IJIACAAI@EndKernPairs@ 10055278     afmparse.obj
 0002:00003288       ??_C@_0N@FEBBJBLC@EndTrackKern@ 10055288     afmparse.obj
 0002:00003298       ??_C@_07BNJNBMEL@EscChar@  10055298     afmparse.obj
 0002:000032a0       ??_C@_0L@KKMPOENF@FamilyName@ 100552a0     afmparse.obj
 0002:000032ac       ??_C@_08EBMMLPNI@FontBBox@ 100552ac     afmparse.obj
 0002:000032b8       ??_C@_08MKFDOKHL@FontName@ 100552b8     afmparse.obj
 0002:000032c4       ??_C@_08FPDCFGEH@FullName@ 100552c4     afmparse.obj
 0002:000032d0       ??_C@_0L@PAHDJIHN@IsBaseFont@ 100552d0     afmparse.obj
 0002:000032dc       ??_C@_09OIFAOJEJ@IsCIDFont@ 100552dc     afmparse.obj
 0002:000032e8       ??_C@_0N@LNIFJEBO@IsFixedPitch@ 100552e8     afmparse.obj
 0002:000032f8       ??_C@_08CHFNODLO@IsFixedV@ 100552f8     afmparse.obj
 0002:00003304       ??_C@_0M@ILCDBHGP@ItalicAngle@ 10055304     afmparse.obj
 0002:00003310       ??_C@_02MGMKBJJI@KP@       10055310     afmparse.obj
 0002:00003314       ??_C@_03MGLCBEGC@KPH@      10055314     afmparse.obj
 0002:00003318       ??_C@_03IMHAAGDD@KPX@      10055318     afmparse.obj
 0002:0000331c       ??_C@_03JFGLDHHC@KPY@      1005531c     afmparse.obj
 0002:00003320       ??_C@_01OCOKONAJ@L@        10055320     afmparse.obj
 0002:00003324       ??_C@_0O@NDBFHPJC@MappingScheme@ 10055324     afmparse.obj
 0002:00003334       ??_C@_0M@PGHPLBFB@MetricsSets@ 10055334     afmparse.obj
 0002:00003340       ??_C@_01NANMIPIL@N@        10055340     afmparse.obj
 0002:00003344       ??_C@_06JHGCIHDH@Notice@   10055344     afmparse.obj
 0002:0000334c       ??_C@_03LMDOAABO@PCC@      1005534c     afmparse.obj
 0002:00003350       ??_C@_09JMBADFPL@StartAxis@ 10055350     afmparse.obj
 0002:0000335c       ??_C@_0BB@JDMDJAID@StartCharMetrics@ 1005535c     afmparse.obj
 0002:00003370       ??_C@_0BA@DGMAPPPC@StartComposites@ 10055370     afmparse.obj
 0002:00003380       ??_C@_0P@DNGHFPAA@StartDirection@ 10055380     afmparse.obj
 0002:00003390       ??_C@_0BB@KAEKNABH@StartFontMetrics@ 10055390     afmparse.obj
 0002:000033a4       ??_C@_0O@GJEKPIHD@StartKernData@ 100553a4     afmparse.obj
 0002:000033b4       ??_C@_0P@OJCDJCKN@StartKernPairs@ 100553b4     afmparse.obj
 0002:000033c4       ??_C@_0BA@HHMIMKDE@StartKernPairs0@ 100553c4     afmparse.obj
 0002:000033d4       ??_C@_0BA@GONDPLHF@StartKernPairs1@ 100553d4     afmparse.obj
 0002:000033e4       ??_C@_0P@DELCCDBH@StartTrackKern@ 100553e4     afmparse.obj
 0002:000033f4       ??_C@_05PHECBFLF@StdHW@    100553f4     afmparse.obj
 0002:000033fc       ??_C@_05OBPKJLMP@StdVW@    100553fc     afmparse.obj
 0002:00003404       ??_C@_09DJCDMHFC@TrackKern@ 10055404     afmparse.obj
 0002:00003410       ??_C@_0BC@CCIMILPE@UnderlinePosition@ 10055410     afmparse.obj
 0002:00003424       ??_C@_0BD@KBICJDLM@UnderlineThickness@ 10055424     afmparse.obj
 0002:00003438       ??_C@_02IEGOIODN@VV@       10055438     afmparse.obj
 0002:0000343c       ??_C@_07HFOFDFIM@VVector@  1005543c     afmparse.obj
 0002:00003444       ??_C@_07NGFJPNPN@Version@  10055444     afmparse.obj
 0002:0000344c       ??_C@_01ELNMCGJD@W@        1005544c     afmparse.obj
 0002:00003450       ??_C@_02LGALCICL@W0@       10055450     afmparse.obj
 0002:00003454       ??_C@_03NOGICFDE@W0X@      10055454     afmparse.obj
 0002:00003458       ??_C@_03MHHDBEHF@W0Y@      10055458     afmparse.obj
 0002:0000345c       ??_C@_02KPBABJGK@W1@       1005545c     afmparse.obj
 0002:00003460       ??_C@_03NPKKEPAD@W1X@      10055460     afmparse.obj
 0002:00003464       ??_C@_03MGLBHOEC@W1Y@      10055464     afmparse.obj
 0002:00003468       ??_C@_02BLCPMJIE@WX@       10055468     afmparse.obj
 0002:0000346c       ??_C@_02CDEPIMF@WY@        1005546c     afmparse.obj
 0002:00003470       ??_C@_06ODJMJFLN@Weight@   10055470     afmparse.obj
 0002:00003478       ??_C@_0N@JPPBHHHF@WeightVector@ 10055478     afmparse.obj
 0002:00003488       ??_C@_07MIHJBPO@XHeight@   10055488     afmparse.obj
 0002:00003490       ??_C@_04LOAJBDKD@true@     10055490     afmparse.obj
 0002:00003498       _af_adlm_uniranges         10055498     afranges.obj
 0002:000034a8       _af_arab_uniranges         100554a8     afranges.obj
 0002:000034e0       _af_armn_uniranges         100554e0     afranges.obj
 0002:000034f8       _af_avst_uniranges         100554f8     afranges.obj
 0002:00003508       _af_bamu_uniranges         10055508     afranges.obj
 0002:00003518       _af_beng_uniranges         10055518     afranges.obj
 0002:00003528       _af_buhd_uniranges         10055528     afranges.obj
 0002:00003538       _af_cakm_uniranges         10055538     afranges.obj
 0002:00003548       _af_cans_uniranges         10055548     afranges.obj
 0002:00003560       _af_cari_uniranges         10055560     afranges.obj
 0002:00003570       _af_cher_uniranges         10055570     afranges.obj
 0002:00003588       _af_copt_uniranges         10055588     afranges.obj
 0002:00003598       _af_cprt_uniranges         10055598     afranges.obj
 0002:000035a8       _af_cyrl_uniranges         100555a8     afranges.obj
 0002:000035d8       _af_deva_uniranges         100555d8     afranges.obj
 0002:00003610       _af_dsrt_uniranges         10055610     afranges.obj
 0002:00003620       _af_ethi_uniranges         10055620     afranges.obj
 0002:00003648       _af_geor_uniranges         10055648     afranges.obj
 0002:00003660       _af_geok_uniranges         10055660     afranges.obj
 0002:00003678       _af_glag_uniranges         10055678     afranges.obj
 0002:00003690       _af_goth_uniranges         10055690     afranges.obj
 0002:000036a0       _af_grek_uniranges         100556a0     afranges.obj
 0002:000036b8       _af_gujr_uniranges         100556b8     afranges.obj
 0002:000036c8       _af_guru_uniranges         100556c8     afranges.obj
 0002:000036d8       _af_hebr_uniranges         100556d8     afranges.obj
 0002:000036f0       _af_kali_uniranges         100556f0     afranges.obj
 0002:00003700       _af_khmr_uniranges         10055700     afranges.obj
 0002:00003710       _af_khms_uniranges         10055710     afranges.obj
 0002:00003720       _af_knda_uniranges         10055720     afranges.obj
 0002:00003730       _af_lao_uniranges          10055730     afranges.obj
 0002:00003740       _af_latn_uniranges         10055740     afranges.obj
 0002:00003848       _af_latb_uniranges         10055848     afranges.obj
 0002:00003868       _af_latp_uniranges         10055868     afranges.obj
 0002:000038d8       _af_lisu_uniranges         100558d8     afranges.obj
 0002:000038e8       _af_mlym_uniranges         100558e8     afranges.obj
 0002:000038f8       _af_medf_uniranges         100558f8     afranges.obj
 0002:00003908       _af_mong_uniranges         10055908     afranges.obj
 0002:00003920       _af_mymr_uniranges         10055920     afranges.obj
 0002:00003940       _af_nkoo_uniranges         10055940     afranges.obj
 0002:00003950       _af_none_uniranges         10055950     afranges.obj
 0002:00003958       _af_olck_uniranges         10055958     afranges.obj
 0002:00003968       _af_orkh_uniranges         10055968     afranges.obj
 0002:00003978       _af_osge_uniranges         10055978     afranges.obj
 0002:00003988       _af_osma_uniranges         10055988     afranges.obj
 0002:00003998       _af_rohg_uniranges         10055998     afranges.obj
 0002:000039a8       _af_saur_uniranges         100559a8     afranges.obj
 0002:000039b8       _af_shaw_uniranges         100559b8     afranges.obj
 0002:000039c8       _af_sinh_uniranges         100559c8     afranges.obj
 0002:000039d8       _af_sund_uniranges         100559d8     afranges.obj
 0002:000039f0       _af_taml_uniranges         100559f0     afranges.obj
 0002:00003a00       _af_tavt_uniranges         10055a00     afranges.obj
 0002:00003a10       _af_telu_uniranges         10055a10     afranges.obj
 0002:00003a20       _af_tfng_uniranges         10055a20     afranges.obj
 0002:00003a30       _af_thai_uniranges         10055a30     afranges.obj
 0002:00003a40       _af_vaii_uniranges         10055a40     afranges.obj
 0002:00003a50       _af_limb_uniranges         10055a50     afranges.obj
 0002:00003a60       _af_orya_uniranges         10055a60     afranges.obj
 0002:00003a70       _af_sylo_uniranges         10055a70     afranges.obj
 0002:00003a80       _af_tibt_uniranges         10055a80     afranges.obj
 0002:00003a90       _af_hani_uniranges         10055a90     afranges.obj
 0002:00003ba0       _af_adlm_nonbase_uniranges 10055ba0     afranges.obj
 0002:00003bb0       _af_arab_nonbase_uniranges 10055bb0     afranges.obj
 0002:00003c50       _af_armn_nonbase_uniranges 10055c50     afranges.obj
 0002:00003c60       _af_avst_nonbase_uniranges 10055c60     afranges.obj
 0002:00003c70       _af_bamu_nonbase_uniranges 10055c70     afranges.obj
 0002:00003c80       _af_beng_nonbase_uniranges 10055c80     afranges.obj
 0002:00003cb8       _af_buhd_nonbase_uniranges 10055cb8     afranges.obj
 0002:00003cc8       _af_cakm_nonbase_uniranges 10055cc8     afranges.obj
 0002:00003ce8       _af_cans_nonbase_uniranges 10055ce8     afranges.obj
 0002:00003cf0       _af_cari_nonbase_uniranges 10055cf0     afranges.obj
 0002:00003cf8       _af_cher_nonbase_uniranges 10055cf8     afranges.obj
 0002:00003d00       _af_copt_nonbase_uniranges 10055d00     afranges.obj
 0002:00003d10       _af_cprt_nonbase_uniranges 10055d10     afranges.obj
 0002:00003d18       _af_cyrl_nonbase_uniranges 10055d18     afranges.obj
 0002:00003d40       _af_deva_nonbase_uniranges 10055d40     afranges.obj
 0002:00003d88       _af_dsrt_nonbase_uniranges 10055d88     afranges.obj
 0002:00003d90       _af_ethi_nonbase_uniranges 10055d90     afranges.obj
 0002:00003da0       _af_geor_nonbase_uniranges 10055da0     afranges.obj
 0002:00003da8       _af_geok_nonbase_uniranges 10055da8     afranges.obj
 0002:00003db0       _af_glag_nonbase_uniranges 10055db0     afranges.obj
 0002:00003dc0       _af_goth_nonbase_uniranges 10055dc0     afranges.obj
 0002:00003dc8       _af_grek_nonbase_uniranges 10055dc8     afranges.obj
 0002:00003e08       _af_gujr_nonbase_uniranges 10055e08     afranges.obj
 0002:00003e40       _af_guru_nonbase_uniranges 10055e40     afranges.obj
 0002:00003e70       _af_hebr_nonbase_uniranges 10055e70     afranges.obj
 0002:00003ea0       _af_kali_nonbase_uniranges 10055ea0     afranges.obj
 0002:00003eb0       _af_khmr_nonbase_uniranges 10055eb0     afranges.obj
 0002:00003ed8       _af_khms_nonbase_uniranges 10055ed8     afranges.obj
 0002:00003ee0       _af_knda_nonbase_uniranges 10055ee0     afranges.obj
 0002:00003f18       _af_lao_nonbase_uniranges  10055f18     afranges.obj
 0002:00003f38       _af_latn_nonbase_uniranges 10055f38     afranges.obj
 0002:00003fc0       _af_latb_nonbase_uniranges 10055fc0     afranges.obj
 0002:00003fc8       _af_latp_nonbase_uniranges 10055fc8     afranges.obj
 0002:00003fd0       _af_lisu_nonbase_uniranges 10055fd0     afranges.obj
 0002:00003fd8       _af_mlym_nonbase_uniranges 10055fd8     afranges.obj
 0002:00004000       _af_medf_nonbase_uniranges 10056000     afranges.obj
 0002:00004008       _af_mong_nonbase_uniranges 10056008     afranges.obj
 0002:00004020       _af_mymr_nonbase_uniranges 10056020     afranges.obj
 0002:00004088       _af_nkoo_nonbase_uniranges 10056088     afranges.obj
 0002:000040a0       _af_none_nonbase_uniranges 100560a0     afranges.obj
 0002:000040a8       _af_olck_nonbase_uniranges 100560a8     afranges.obj
 0002:000040b0       _af_orkh_nonbase_uniranges 100560b0     afranges.obj
 0002:000040b8       _af_osge_nonbase_uniranges 100560b8     afranges.obj
 0002:000040c0       _af_osma_nonbase_uniranges 100560c0     afranges.obj
 0002:000040c8       _af_rohg_nonbase_uniranges 100560c8     afranges.obj
 0002:000040d0       _af_saur_nonbase_uniranges 100560d0     afranges.obj
 0002:000040e8       _af_shaw_nonbase_uniranges 100560e8     afranges.obj
 0002:000040f0       _af_sinh_nonbase_uniranges 100560f0     afranges.obj
 0002:00004108       _af_sund_nonbase_uniranges 10056108     afranges.obj
 0002:00004120       _af_taml_nonbase_uniranges 10056120     afranges.obj
 0002:00004140       _af_tavt_nonbase_uniranges 10056140     afranges.obj
 0002:00004170       _af_telu_nonbase_uniranges 10056170     afranges.obj
 0002:000041a0       _af_tfng_nonbase_uniranges 100561a0     afranges.obj
 0002:000041a8       _af_thai_nonbase_uniranges 100561a8     afranges.obj
 0002:000041c8       _af_vaii_nonbase_uniranges 100561c8     afranges.obj
 0002:000041d0       _af_limb_nonbase_uniranges 100561d0     afranges.obj
 0002:000041f0       _af_orya_nonbase_uniranges 100561f0     afranges.obj
 0002:00004228       _af_sylo_nonbase_uniranges 10056228     afranges.obj
 0002:00004250       _af_tibt_nonbase_uniranges 10056250     afranges.obj
 0002:000042a0       _af_hani_nonbase_uniranges 100562a0     afranges.obj
 0002:000042b8       _cff_cmap_encoding_class_rec 100562b8     cffcmap.obj
 0002:000042e0       _cff_cmap_unicode_class_rec 100562e0     cffcmap.obj
 0002:00004308       _cff_driver_class          10056308     cffdrivr.obj
 0002:00004460       ??_C@_0L@POCJHJKN@glyph?9dict@ 10056460     cffdrivr.obj
 0002:0000446c       ??_C@_0BF@GDPJODJF@postscript?9font?9name@ 1005646c     cffdrivr.obj
 0002:00004484       ??_C@_08OHCKCLF@tt?9cmaps@ 10056484     cffdrivr.obj
 0002:00004490       ??_C@_0M@NJKHAGNP@font?9format@ 10056490     cffdrivr.obj
 0002:0000449c       ??_C@_03IFCOMOMB@CFF@      1005649c     cffdrivr.obj
 0002:000044a0       ??_C@_0O@DHADKGAK@multi?9masters@ 100564a0     cffdrivr.obj
 0002:000044b0       ??_C@_0BD@EFEGEJAN@metrics?9variations@ 100564b0     cffdrivr.obj
 0002:000044c4       ??_C@_0BA@EAOIOGJA@postscript?9info@ 100564c4     cffdrivr.obj
 0002:000044d4       ??_C@_03LMEEOLHO@CID@      100564d4     cffdrivr.obj
 0002:000044d8       ??_C@_08EOMLOCJG@cff?9load@ 100564d8     cffdrivr.obj
 0002:000044e4       ??_C@_03IINFADLN@cff@      100564e4     cffdrivr.obj
 0002:000044e8       ??_C@_04JAPIGAPK@sfnt@     100564e8     cffdrivr.obj
 0002:000044f0       ??_C@_0BB@JIMLNENF@postscript?9cmaps@ 100564f0     cffdrivr.obj
 0002:00004504       ??_C@_07IAJFBLNJ@?1FSType@ 10056504     cffdrivr.obj
 0002:0000450c       ??_C@_03BHEEIFFN@def@      1005650c     cffdrivr.obj
 0002:00004cf4       ??_C@_08MNGCAOLP@pshinter@ 10056cf4     cffobjs.obj
 0002:00004d00       ??_C@_05MNCLAAKB@psaux@    10056d00     cffobjs.obj
 0002:00004d08       ??_C@_07FFHPBFOK@Regular@  10056d08     cffobjs.obj
 0002:00004d10       ??_C@_04DIPHHIHJ@Bold@     10056d10     cffobjs.obj
 0002:00004d18       ??_C@_05BPGNDIAE@Black@    10056d18     cffobjs.obj
 0002:00005d54       ??_C@_0M@CKCGNNAK@CIDFontName@ 10057d54     cidload.obj
 0002:00005d60       ??_C@_0P@FDOGBFAP@CIDFontVersion@ 10057d60     cidload.obj
 0002:00005d70       ??_C@_0M@IBCFBNHK@CIDFontType@ 10057d70     cidload.obj
 0002:00005d7c       ??_C@_08EPBENDNC@Registry@ 10057d7c     cidload.obj
 0002:00005d88       ??_C@_08HMKBFHBJ@Ordering@ 10057d88     cidload.obj
 0002:00005d94       ??_C@_0L@EJNILPMC@Supplement@ 10057d94     cidload.obj
 0002:00005da0       ??_C@_07CNNFHHEA@UIDBase@  10057da0     cidload.obj
 0002:00005da8       ??_C@_04CGDDEPDG@XUID@     10057da8     cidload.obj
 0002:00005db0       ??_C@_0N@LBMCPKAC@CIDMapOffset@ 10057db0     cidload.obj
 0002:00005dc0       ??_C@_07NNGKIHHK@FDBytes@  10057dc0     cidload.obj
 0002:00005dc8       ??_C@_07BBMAIHOE@GDBytes@  10057dc8     cidload.obj
 0002:00005dd0       ??_C@_08LPCKMOBH@CIDCount@ 10057dd0     cidload.obj
 0002:00005ddc       ??_C@_07CPCPJPKL@version@  10057ddc     cidload.obj
 0002:00005de4       ??_C@_0N@OPLNPOL@isFixedPitch@ 10057de4     cidload.obj
 0002:00005df4       ??_C@_06FIINGLDE@FSType@   10057df4     cidload.obj
 0002:00005dfc       ??_C@_09PNDIDGHG@PaintType@ 10057dfc     cidload.obj
 0002:00005e08       ??_C@_08GBFACKAL@FontType@ 10057e08     cidload.obj
 0002:00005e14       ??_C@_0O@DKIHOHFK@SubrMapOffset@ 10057e14     cidload.obj
 0002:00005e24       ??_C@_07OJDBLIDF@SDBytes@  10057e24     cidload.obj
 0002:00005e2c       ??_C@_09NKAONILE@SubrCount@ 10057e2c     cidload.obj
 0002:00005e38       ??_C@_0BC@HBJENNOG@lenBuildCharArray@ 10057e38     cidload.obj
 0002:00005e4c       ??_C@_0BD@BGHMBBEO@ForceBoldThreshold@ 10057e4c     cidload.obj
 0002:00005e60       ??_C@_0M@GLGMDIGG@StrokeWidth@ 10057e60     cidload.obj
 0002:00005e6c       ??_C@_08OMJGNOHD@UniqueID@ 10057e6c     cidload.obj
 0002:00005e78       ??_C@_05CIIKKFON@lenIV@    10057e78     cidload.obj
 0002:00005e80       ??_C@_0O@PJDGHDCK@LanguageGroup@ 10057e80     cidload.obj
 0002:00005e90       ??_C@_08NLHBPEGP@password@ 10057e90     cidload.obj
 0002:00005e9c       ??_C@_09IPAGIEBG@BlueScale@ 10057e9c     cidload.obj
 0002:00005ea8       ??_C@_09GDCMDLCO@BlueShift@ 10057ea8     cidload.obj
 0002:00005eb4       ??_C@_08IPFLJFPM@BlueFuzz@ 10057eb4     cidload.obj
 0002:00005ec0       ??_C@_0L@DKDIMLOI@BlueValues@ 10057ec0     cidload.obj
 0002:00005ecc       ??_C@_0L@CCJAIIMC@OtherBlues@ 10057ecc     cidload.obj
 0002:00005ed8       ??_C@_0M@OIPOLIDA@FamilyBlues@ 10057ed8     cidload.obj
 0002:00005ee4       ??_C@_0BB@FMLCJJDP@FamilyOtherBlues@ 10057ee4     cidload.obj
 0002:00005ef8       ??_C@_0L@NKGPCONN@MinFeature@ 10057ef8     cidload.obj
 0002:00005f04       ??_C@_09NCKADFKP@StemSnapH@ 10057f04     cidload.obj
 0002:00005f10       ??_C@_09GOBAKHA@StemSnapV@ 10057f10     cidload.obj
 0002:00005f1c       ??_C@_09BDDIAPM@ForceBold@ 10057f1c     cidload.obj
 0002:00005f28       ??_C@_07PEKDNLEP@FDArray@  10057f28     cidload.obj
 0002:00005f30       ??_C@_0L@LNCCOCBB@FontMatrix@ 10057f30     cidload.obj
 0002:00005f3c       ??_C@_0BA@PKGIFANC@ExpansionFactor@ 10057f3c     cidload.obj
 0002:00005f4c       ??_C@_0BC@JBBEDJNJ@?$CFADOBeginFontDict@ 10057f4c     cidload.obj
 0002:00005f60       ??_C@_0CA@JGHPJJJF@?$CF?$CBPS?9Adobe?93?40?5Resource?9CIDFont@ 10057f60     cidparse.obj
 0002:00005f80       ??_C@_09BFOLOCGO@StartData@ 10057f80     cidparse.obj
 0002:00005f8c       ??_C@_06EMLBPOPP@?1sfnts@  10057f8c     cidparse.obj
 0002:00005f94       ??_C@_05NPBNGLLN@?$CIHex?$CJ@ 10057f94     cidparse.obj
 0002:00006000       _t1cid_driver_class        10058000     cidriver.obj
 0002:00006060       ??_C@_0L@DDPIBKML@CID?5Type?51@ 10058060     cidriver.obj
 0002:0000606c       ??_C@_05CNMLIGFM@t1cid@    1005806c     cidriver.obj
 0002:00006090       __xmm@80000001800000017fffffff7fffffff 10058090     ftbbox.obj
 0002:000060b8       _ft_bitmap_glyph_class     100580b8     ftglyph.obj
 0002:000060d8       _ft_outline_glyph_class    100580d8     ftglyph.obj
 0002:00006110       _ft_grays_raster           10058110     ftgrays.obj
 0002:00006158       ??_C@_0BE@LLDKDDBI@FREETYPE_PROPERTIES@ 10058158     ftinit.obj
 0002:0000616c       ??_C@_06LFMFFOBP@ot?9svg@  1005816c     ftobjs.obj
 0002:00006174       ??_C@_06JCBOBHIA@Type?51@  10058174     ftobjs.obj
 0002:0000617c       ??_C@_03LBLPCGAC@cid@      1005817c     ftobjs.obj
 0002:00006180       ??_C@_05MJDCDNNA@type1@    10058180     ftobjs.obj
 0002:00006188       ??_C@_08OKLLNAKL@truetype@ 10058188     ftobjs.obj
 0002:00006194       ??_C@_07IAOBDJBM@kerning@  10058194     ftobjs.obj
 0002:0000619c       ??_C@_0L@MBBJBANC@sfnt?9table@ 1005819c     ftobjs.obj
 0002:000061a8       ??_C@_06GNKBHGHD@type42@   100581a8     ftobjs.obj
 0002:000061b0       ??_C@_0BA@DHLLBDBB@truetype?9engine@ 100581b0     ftobjs.obj
 0002:000061d4       ??_C@_0P@DGAAAJJA@hinting?9engine@ 100581d4     ftpsprop.obj
 0002:000061e4       ??_C@_05NBLLDENH@adobe@    100581e4     ftpsprop.obj
 0002:000061ec       ??_C@_0M@LGDPDIPE@random?9seed@ 100581ec     ftpsprop.obj
 0002:000061f8       _ft_standard_raster        100581f8     ftraster.obj
 0002:00006210       _ft_raster1_renderer_class 10058210     ftrend1.obj
 0002:0000624c       ??_C@_07EFFNHEPH@raster1@  1005824c     ftrend1.obj
 0002:000062a0       ??_C@_02PEOAMJM@?4_@       100582a0     ftrfork.obj
 0002:000062a4       ??_C@_05FLPKNBDI@?1rsrc@   100582a4     ftrfork.obj
 0002:000062ac       ??_C@_0BC@OBHLCHMP@?1?4?4namedfork?1rsrc@ 100582ac     ftrfork.obj
 0002:000062c0       ??_C@_0O@FDMCFKOC@resource?4frk?1@ 100582c0     ftrfork.obj
 0002:000062d0       ??_C@_0L@FGJFJHGF@?4resource?1@ 100582d0     ftrfork.obj
 0002:000062dc       ??_C@_01FGNFDNOH@?$CF@     100582dc     ftrfork.obj
 0002:000062e0       ??_C@_0O@KCDCBAF@?4AppleDouble?1@ 100582e0     ftrfork.obj
 0002:000062f0       _ft_smooth_renderer_class  100582f0     ftsmooth.obj
 0002:0000632c       ??_C@_06INICNAFJ@smooth@   1005832c     ftsmooth.obj
 0002:00006334       ??_C@_02JDPG@rb@           10058334     ftsystem.obj
 0002:00006390       _cff_builder_funcs         10058390     psauxmod.obj
 0002:000063b0       _ps_builder_funcs          100583b0     psauxmod.obj
 0002:000063b8       _afm_parser_funcs          100583b8     psauxmod.obj
 0002:000063c4       _t1_cmap_classes           100583c4     psauxmod.obj
 0002:000063d4       _cff_decoder_funcs         100583d4     psauxmod.obj
 0002:000063e0       _psaux_module_class        100583e0     psauxmod.obj
 0002:00006404       _ps_table_funcs            10058404     psauxmod.obj
 0002:00006414       _ps_parser_funcs           10058414     psauxmod.obj
 0002:00006448       _t1_builder_funcs          10058448     psauxmod.obj
 0002:00006468       _t1_decoder_funcs          10058468     psauxmod.obj
 0002:00006528       _pshinter_module_class     10058528     pshmod.obj
 0002:00006588       _psnames_module_class      10058588     psmodule.obj
 0002:000065b0       _ft_standard_glyph_names   100585b0     psmodule.obj
 0002:00007420       _ft_mac_names              10059420     psmodule.obj
 0002:00007628       _ft_sid_names              10059628     psmodule.obj
 0002:00007938       _t1_standard_encoding      10059938     psmodule.obj
 0002:00007b38       _t1_expert_encoding        10059b38     psmodule.obj
 0002:00007d38       _ft_adobe_glyph_list       10059d38     psmodule.obj
 0002:000158d0       ??_C@_07POODEHEH@psnames@  100678d0     psmodule.obj
 0002:000158d8       _sfnt_module_class         100678d8     sfdriver.obj
 0002:00015aac       _t1_cmap_standard_class_rec 10067aac     t1cmap.obj
 0002:00015ad4       _t1_cmap_expert_class_rec  10067ad4     t1cmap.obj
 0002:00015afc       _t1_cmap_custom_class_rec  10067afc     t1cmap.obj
 0002:00015b24       _t1_cmap_unicode_class_rec 10067b24     t1cmap.obj
 0002:00015c60       _t1_driver_class           10067c60     t1driver.obj
 0002:0001635c       ??_C@_03DOACNACD@NDV@      1006835c     t1load.obj
 0002:00016360       ??_C@_03MMGIAIPO@CDV@      10068360     t1load.obj
 0002:00016364       ??_C@_0N@PGGOPDKP@DesignVector@ 10068364     t1load.obj
 0002:00016374       ??_C@_08EJAHIGCJ@Encoding@ 10068374     t1load.obj
 0002:00016380       ??_C@_05DHFNOCDJ@Subrs@    10068380     t1load.obj
 0002:00016388       ??_C@_0M@EKIFGBLL@CharStrings@ 10068388     t1load.obj
 0002:00016394       ??_C@_07CFINJGKH@Private@  10068394     t1load.obj
 0002:0001639c       ??_C@_0P@KEOGGALI@BuildCharArray@ 1006839c     t1load.obj
 0002:000163ac       ??_C@_05IBAMDCFI@Width@    100683ac     t1load.obj
 0002:000163b4       ??_C@_0M@EDHPABCB@OpticalSize@ 100683b4     t1load.obj
 0002:000163c0       ??_C@_07JBKHDJHE@?4notdef@ 100683c0     t1load.obj
 0002:000163c8       ??_C@_0BB@MLEHKAJM@StandardEncoding@ 100683c8     t1load.obj
 0002:000163dc       ??_C@_0P@LHOFAKJ@ExpertEncoding@ 100683dc     t1load.obj
 0002:000163ec       ??_C@_0BC@OHHLKLPP@ISOLatin1Encoding@ 100683ec     t1load.obj
 0002:00016400       ??_C@_03BHPKJDPK@dup@      10068400     t1load.obj
 0002:00016404       ??_C@_03KMONJGDG@put@      10068404     t1load.obj
 0002:00016408       ??_C@_05OJJBIBFE@eexec@    10068408     t1load.obj
 0002:00016410       ??_C@_09BJJLCLMA@closefile@ 10068410     t1load.obj
 0002:0001641c       ??_C@_0O@CJLBGMNG@FontDirectory@ 1006841c     t1load.obj
 0002:0001642c       ??_C@_0P@EMKCEFJO@?$CF?$CBPS?9AdobeFont@ 1006842c     t1parse.obj
 0002:0001643c       ??_C@_0L@LLIKMEDC@?$CF?$CBFontType@ 1006843c     t1parse.obj
 0002:00016448       _tt_cmap0_class_rec        10068448     ttcmap.obj
 0002:0001647c       _tt_cmap2_class_rec        1006847c     ttcmap.obj
 0002:000164b0       _tt_cmap4_class_rec        100684b0     ttcmap.obj
 0002:000164e4       _tt_cmap6_class_rec        100684e4     ttcmap.obj
 0002:00016518       _tt_cmap8_class_rec        10068518     ttcmap.obj
 0002:0001654c       _tt_cmap10_class_rec       1006854c     ttcmap.obj
 0002:00016580       _tt_cmap12_class_rec       10068580     ttcmap.obj
 0002:000165b4       _tt_cmap13_class_rec       100685b4     ttcmap.obj
 0002:000165e8       _tt_cmap14_class_rec       100685e8     ttcmap.obj
 0002:0001661c       _tt_cmap_unicode_class_rec 1006861c     ttcmap.obj
 0002:00016678       _tt_driver_class           10068678     ttdriver.obj
 0002:00016770       ??_C@_08KJILHNAM@TrueType@ 10068770     ttdriver.obj
 0002:0001677c       ??_C@_07CDLHCBDE@tt?9glyf@ 1006877c     ttdriver.obj
 0002:00016784       ??_C@_0BE@OJJAFABD@interpreter?9version@ 10068784     ttdriver.obj
 0002:00016800       ??_C@_05BCGFHEPH@Slant@    10068800     ttgxvar.obj
 0002:00016808       _tt_default_graphics_state 10068808     ttinterp.obj
 0002:00017190       __pRawDllMain              10069190     MSVCRT:dll_dllmain.obj
 0002:00017190       __pDefaultRawDllMain       10069190     MSVCRT:dll_dllmain.obj
 0002:00017208       __load_config_used         10069208     MSVCRT:loadcfg.obj
 0002:000172c0       ___safe_se_handler_table   100692c0     <linker-defined>
 0002:0001754c       ___rtc_iaa                 1006954c     MSVCRT:initsect.obj
 0002:00017550       ___rtc_izz                 10069550     MSVCRT:initsect.obj
 0002:00017554       ___rtc_taa                 10069554     MSVCRT:initsect.obj
 0002:00017558       ___rtc_tzz                 10069558     MSVCRT:initsect.obj
 0002:00018ad8       __IMPORT_DESCRIPTOR_KERNEL32 1006aad8     kernel32:KERNEL32.dll
 0002:00018aec       __IMPORT_DESCRIPTOR_VCRUNTIME140 1006aaec     vcruntime:VCRUNTIME140.dll
 0002:00018b00       __IMPORT_DESCRIPTOR_api-ms-win-crt-convert-l1-1-0 1006ab00     ucrt:api-ms-win-crt-convert-l1-1-0.dll
 0002:00018b14       __IMPORT_DESCRIPTOR_api-ms-win-crt-string-l1-1-0 1006ab14     ucrt:api-ms-win-crt-string-l1-1-0.dll
 0002:00018b28       __IMPORT_DESCRIPTOR_api-ms-win-crt-utility-l1-1-0 1006ab28     ucrt:api-ms-win-crt-utility-l1-1-0.dll
 0002:00018b3c       __IMPORT_DESCRIPTOR_api-ms-win-crt-environment-l1-1-0 1006ab3c     ucrt:api-ms-win-crt-environment-l1-1-0.dll
 0002:00018b50       __IMPORT_DESCRIPTOR_api-ms-win-crt-stdio-l1-1-0 1006ab50     ucrt:api-ms-win-crt-stdio-l1-1-0.dll
 0002:00018b64       __IMPORT_DESCRIPTOR_api-ms-win-crt-heap-l1-1-0 1006ab64     ucrt:api-ms-win-crt-heap-l1-1-0.dll
 0002:00018b78       __IMPORT_DESCRIPTOR_api-ms-win-crt-runtime-l1-1-0 1006ab78     ucrt:api-ms-win-crt-runtime-l1-1-0.dll
 0002:00018b8c       __NULL_IMPORT_DESCRIPTOR   1006ab8c     kernel32:KERNEL32.dll
 0003:00000000       ___security_cookie_complement 1006c000     MSVCRT:gs_cookie.obj
 0003:00000004       ___security_cookie         1006c004     MSVCRT:gs_cookie.obj
 0003:00000010       ___scrt_native_dllmain_reason 1006c010     MSVCRT:utility.obj
 0003:00000020       ___isa_enabled             1006c020     MSVCRT:cpu_disp.obj
 0003:00000024       ___scrt_ucrt_dll_is_in_use 1006c024     MSVCRT:ucrt_stubs.obj
 0003:00000348       ?__type_info_root_node@@3U__type_info_node@@A 1006c348     MSVCRT:tncleanup.obj
 0003:00000350       ?_OptionsStorage@?1??__local_stdio_printf_options@@9@4_KA 1006c350     MSVCRT:default_local_stdio_options.obj
 0003:00000358       ?_OptionsStorage@?1??__local_stdio_scanf_options@@9@4_KA 1006c358     MSVCRT:default_local_stdio_options.obj
 0003:00000360       ___scrt_current_native_startup_state 1006c360     MSVCRT:utility.obj
 0003:00000364       ___scrt_native_startup_lock 1006c364     MSVCRT:utility.obj
 0003:00000384       ___scrt_debugger_hook_flag 1006c384     MSVCRT:utility_desktop.obj
 0003:00000388       ___isa_available           1006c388     MSVCRT:cpu_disp.obj
 0003:0000038c       ___favor                   1006c38c     MSVCRT:cpu_disp.obj
 0003:00000390       ___dyn_tls_init_callback   1006c390     <common>

 entry point at        0001:000506fa

 Static symbols

 0000:fff90000       .debug$S                   10000000     freetype.exp
 0000:fff90000       .debug$S                   10000000     vcruntime:VCRUNTIME140.dll
 0000:fff90000       .debug$S                   10000000     vcruntime:VCRUNTIME140.dll
 0000:fff90000       .debug$S                   10000000     vcruntime:VCRUNTIME140.dll
 0000:fff90000       .debug$S                   10000000     vcruntime:VCRUNTIME140.dll
 0000:fff90000       .debug$S                   10000000     vcruntime:VCRUNTIME140.dll
 0000:fff90000       .debug$S                   10000000     vcruntime:VCRUNTIME140.dll
 0000:fff90000       .debug$S                   10000000     vcruntime:VCRUNTIME140.dll
 0000:fff90000       .debug$S                   10000000     vcruntime:VCRUNTIME140.dll
 0000:fff90000       .debug$S                   10000000     vcruntime:VCRUNTIME140.dll
 0000:fff90000       .debug$S                   10000000     vcruntime:VCRUNTIME140.dll
 0000:fff90000       .debug$S                   10000000     vcruntime:VCRUNTIME140.dll
 0000:fff90000       .debug$S                   10000000     vcruntime:VCRUNTIME140.dll
 0000:fff90000       .debug$S                   10000000     ucrt:api-ms-win-crt-convert-l1-1-0.dll
 0000:fff90000       .debug$S                   10000000     ucrt:api-ms-win-crt-environment-l1-1-0.dll
 0000:fff90000       .debug$S                   10000000     ucrt:api-ms-win-crt-heap-l1-1-0.dll
 0000:fff90000       .debug$S                   10000000     ucrt:api-ms-win-crt-heap-l1-1-0.dll
 0000:fff90000       .debug$S                   10000000     ucrt:api-ms-win-crt-heap-l1-1-0.dll
 0000:fff90000       .debug$S                   10000000     ucrt:api-ms-win-crt-runtime-l1-1-0.dll
 0000:fff90000       .debug$S                   10000000     ucrt:api-ms-win-crt-runtime-l1-1-0.dll
 0000:fff90000       .debug$S                   10000000     ucrt:api-ms-win-crt-runtime-l1-1-0.dll
 0000:fff90000       .debug$S                   10000000     ucrt:api-ms-win-crt-runtime-l1-1-0.dll
 0000:fff90000       .debug$S                   10000000     ucrt:api-ms-win-crt-runtime-l1-1-0.dll
 0000:fff90000       .debug$S                   10000000     ucrt:api-ms-win-crt-runtime-l1-1-0.dll
 0000:fff90000       .debug$S                   10000000     ucrt:api-ms-win-crt-runtime-l1-1-0.dll
 0000:fff90000       .debug$S                   10000000     ucrt:api-ms-win-crt-runtime-l1-1-0.dll
 0000:fff90000       .debug$S                   10000000     ucrt:api-ms-win-crt-runtime-l1-1-0.dll
 0000:fff90000       .debug$S                   10000000     ucrt:api-ms-win-crt-runtime-l1-1-0.dll
 0000:fff90000       .debug$S                   10000000     ucrt:api-ms-win-crt-runtime-l1-1-0.dll
 0000:fff90000       .debug$S                   10000000     ucrt:api-ms-win-crt-runtime-l1-1-0.dll
 0000:fff90000       .debug$S                   10000000     ucrt:api-ms-win-crt-stdio-l1-1-0.dll
 0000:fff90000       .debug$S                   10000000     ucrt:api-ms-win-crt-stdio-l1-1-0.dll
 0000:fff90000       .debug$S                   10000000     ucrt:api-ms-win-crt-stdio-l1-1-0.dll
 0000:fff90000       .debug$S                   10000000     ucrt:api-ms-win-crt-stdio-l1-1-0.dll
 0000:fff90000       .debug$S                   10000000     ucrt:api-ms-win-crt-stdio-l1-1-0.dll
 0000:fff90000       .debug$S                   10000000     ucrt:api-ms-win-crt-string-l1-1-0.dll
 0000:fff90000       .debug$S                   10000000     ucrt:api-ms-win-crt-string-l1-1-0.dll
 0000:fff90000       .debug$S                   10000000     ucrt:api-ms-win-crt-utility-l1-1-0.dll
 0000:fff90000       .debug$S                   10000000     kernel32:KERNEL32.dll
 0000:fff90000       .debug$S                   10000000     kernel32:KERNEL32.dll
 0000:fff90000       .debug$S                   10000000     kernel32:KERNEL32.dll
 0000:fff90000       .debug$S                   10000000     kernel32:KERNEL32.dll
 0000:fff90000       .debug$S                   10000000     kernel32:KERNEL32.dll
 0000:fff90000       .debug$S                   10000000     kernel32:KERNEL32.dll
 0000:fff90000       .debug$S                   10000000     kernel32:KERNEL32.dll
 0000:fff90000       .debug$S                   10000000     kernel32:KERNEL32.dll
 0000:fff90000       .debug$S                   10000000     kernel32:KERNEL32.dll
 0000:fff90000       .debug$S                   10000000     kernel32:KERNEL32.dll
 0000:fff90000       .debug$S                   10000000     kernel32:KERNEL32.dll
 0000:fff90000       .debug$S                   10000000     kernel32:KERNEL32.dll
 0000:fff90000       .debug$S                   10000000     kernel32:KERNEL32.dll
 0000:fff90000       .debug$S                   10000000     kernel32:KERNEL32.dll
 0001:000003d0       _af_indic_get_standard_widths 100013d0 f   afindic.obj
 0001:00000400       _af_cjk_compute_stem_width 10001400 f   afcjk.obj
 0001:000005f0       _af_cjk_hint_edges         100015f0 f   afcjk.obj
 0001:00000a40       _af_cjk_hints_compute_blue_edges 10001a40 f   afcjk.obj
 0001:00000c10       _af_cjk_hints_compute_edges 10001c10 f   afcjk.obj
 0001:00001020       _af_cjk_hints_detect_features 10002020 f   afcjk.obj
 0001:000010b0       _af_cjk_hints_link_segments 100020b0 f   afcjk.obj
 0001:00001440       _af_cjk_metrics_init_blues 10002440 f   afcjk.obj
 0001:00001a90       _af_cjk_metrics_scale_dim  10002a90 f   afcjk.obj
 0001:00001c50       _af_hint_normal_stem       10002c50 f   afcjk.obj
 0001:00001df0       _af_dummy_hints_init       10002df0 f   afdummy.obj
 0001:00001e30       _af_dummy_hints_apply      10002e30 f   afdummy.obj
 0001:00001e60       _af_face_globals_compute_style_coverage 10002e60 f   afglobal.obj
 0001:00003430       _af_iup_interp             10004430 f   afhints.obj
 0001:00003880       _af_indic_metrics_init     10004880 f   afindic.obj
 0001:000038e0       _af_indic_metrics_scale    100048e0 f   afindic.obj
 0001:000038f0       _af_indic_hints_init       100048f0 f   afindic.obj
 0001:00003900       _af_indic_hints_apply      10004900 f   afindic.obj
 0001:00003ac0       _af_latin_hints_init       10004ac0 f   aflatin.obj
 0001:00003b70       _af_latin_hints_apply      10004b70 f   aflatin.obj
 0001:00003ca0       _af_latin_compute_stem_width 10004ca0 f   aflatin.obj
 0001:00003f70       _af_latin_hint_edges       10004f70 f   aflatin.obj
 0001:000046c0       _af_latin_hints_compute_blue_edges 100056c0 f   aflatin.obj
 0001:00005850       _af_latin_metrics_init_blues 10006850 f   aflatin.obj
 0001:00006640       _af_latin_metrics_scale_dim 10007640 f   aflatin.obj
 0001:00007560       _af_property_set           10008560 f   afmodule.obj
 0001:00007920       _af_property_get           10008920 f   afmodule.obj
 0001:00007b70       _af_get_interface          10008b70 f   afmodule.obj
 0001:00007b80       _af_autofitter_init        10008b80 f   afmodule.obj
 0001:00007be0       _af_autofitter_done        10008be0 f   afmodule.obj
 0001:00007be0       _parse_font_name           10008be0 f   cidload.obj
 0001:00007be0       _gray_raster_reset         10008be0 f   ftgrays.obj
 0001:00007be0       _Horizontal_Sweep_Init     10008be0 f   ftraster.obj
 0001:00007be0       _Horizontal_Sweep_Step     10008be0 f   ftraster.obj
 0001:00007be0       _ft_black_reset            10008be0 f   ftraster.obj
 0001:00007bf0       _af_autofitter_load_glyph  10008bf0 f   afmodule.obj
 0001:00007c90       _afm_compare_kern_pairs    10008c90 f   afmparse.obj
 0001:00007c90       _compare_kern_pairs        10008c90 f   t1afm.obj
 0001:00007cc0       _afm_parse_kern_pairs      10008cc0 f   afmparse.obj
 0001:00007ea4       $LN98                      10008ea4     afmparse.obj
 0001:00007eb4       $LN97                      10008eb4     afmparse.obj
 0001:00007ef0       _afm_parse_track_kern      10008ef0 f   afmparse.obj
 0001:000080ac       $LN116                     100090ac     afmparse.obj
 0001:000080bc       $LN115                     100090bc     afmparse.obj
 0001:0000858c       $LN401                     1000958c     afmparse.obj
 0001:000085b0       $LN400                     100095b0     afmparse.obj
 0001:000085e4       $LN403                     100095e4     afmparse.obj
 0001:000085f8       $LN402                     100095f8     afmparse.obj
 0001:0000875c       $LN27                      1000975c     afmparse.obj
 0001:00008780       _afm_stream_read_one       10009780 f   afmparse.obj
 0001:00008800       _afm_stream_read_string    10009800 f   afmparse.obj
 0001:00008860       _afm_stream_skip_spaces    10009860 f   afmparse.obj
 0001:000088d0       _afm_tokenize              100098d0 f   afmparse.obj
 0001:00008a60       _gray_raster_set_mode      10009a60 f   ftgrays.obj
 0001:00008a60       _ft_black_set_mode         10009a60 f   ftraster.obj
 0001:00008a60       _tt_cmap14_char_index      10009a60 f   ttcmap.obj
 0001:00008ab0       _cff_cmap_encoding_init    10009ab0 f   cffcmap.obj
 0001:00008ad0       _cff_cmap_encoding_done    10009ad0 f   cffcmap.obj
 0001:00008ae0       _cff_cmap_encoding_char_index 10009ae0 f   cffcmap.obj
 0001:00008b00       _cff_cmap_encoding_char_next 10009b00 f   cffcmap.obj
 0001:00008b50       _cff_cmap_unicode_init     10009b50 f   cffcmap.obj
 0001:00008ba0       _cff_cmap_unicode_done     10009ba0 f   cffcmap.obj
 0001:00008ba0       _t1_cmap_unicode_done      10009ba0 f   t1cmap.obj
 0001:00008ba0       _tt_cmap_unicode_done      10009ba0 f   ttcmap.obj
 0001:00008bd0       _cff_cmap_unicode_char_index 10009bd0 f   cffcmap.obj
 0001:00008bf0       _cff_cmap_unicode_char_next 10009bf0 f   cffcmap.obj
 0001:00008c10       _cff_sid_to_glyph_name     10009c10 f   cffcmap.obj
 0001:00008e30       _cff_get_kerning           10009e30 f   cffdrivr.obj
 0001:00008e30       _tt_get_kerning            10009e30 f   ttdriver.obj
 0001:00008e70       _cff_glyph_load            10009e70 f   cffdrivr.obj
 0001:00008ec0       _cff_get_advances          10009ec0 f   cffdrivr.obj
 0001:00009060       _cff_get_glyph_name        1000a060 f   cffdrivr.obj
 0001:000090f0       _cff_get_name_index        1000a0f0 f   cffdrivr.obj
 0001:000091e0       _cff_ps_has_glyph_names    1000a1e0 f   cffdrivr.obj
 0001:00009200       _cff_ps_get_font_info      1000a200 f   cffdrivr.obj
 0001:000092e0       _cff_ps_get_font_extra     1000a2e0 f   cffdrivr.obj
 0001:000093d0       _cff_get_ps_name           1000a3d0 f   cffdrivr.obj
 0001:00009430       _cff_get_cmap_info         1000a430 f   cffdrivr.obj
 0001:00009490       _cff_get_ros               1000a490 f   cffdrivr.obj
 0001:00009520       _cff_get_is_cid            1000a520 f   cffdrivr.obj
 0001:00009560       _cff_get_cid_from_glyph_index 1000a560 f   cffdrivr.obj
 0001:000095a0       _cff_set_mm_blend          1000a5a0 f   cffdrivr.obj
 0001:000095c0       _cff_get_mm_blend          1000a5c0 f   cffdrivr.obj
 0001:000095e0       _cff_set_mm_weightvector   1000a5e0 f   cffdrivr.obj
 0001:00009600       _cff_get_mm_weightvector   1000a600 f   cffdrivr.obj
 0001:00009620       _cff_get_mm_var            1000a620 f   cffdrivr.obj
 0001:00009640       _cff_set_var_design        1000a640 f   cffdrivr.obj
 0001:00009660       _cff_get_var_design        1000a660 f   cffdrivr.obj
 0001:00009680       _cff_set_instance          1000a680 f   cffdrivr.obj
 0001:000096a0       _cff_hadvance_adjust       1000a6a0 f   cffdrivr.obj
 0001:000096c0       _cff_metrics_adjust        1000a6c0 f   cffdrivr.obj
 0001:000096e0       _cff_get_interface         1000a6e0 f   cffdrivr.obj
 0001:0000a770       _cff_charset_compute_cids  1000b770 f   cffload.obj
 0001:0000a820       _cff_charset_load          1000b820 f   cffload.obj
 0001:0000ab20       _cff_encoding_load         1000bb20 f   cffload.obj
 0001:0000bad0       _cff_index_done            1000cad0 f   cffload.obj
 0001:0000bbe0       _cff_index_get_pointers    1000cbe0 f   cffload.obj
 0001:0000be00       _cff_index_init            1000ce00 f   cffload.obj
 0001:0000bf80       _cff_index_load_offsets    1000cf80 f   cffload.obj
 0001:0000c110       _cff_index_read_offset     1000d110 f   cffload.obj
 0001:0000c330       _cff_subfont_done          1000d330 f   cffload.obj
 0001:0000c400       _cff_subfont_load          1000d400 f   cffload.obj
 0001:0000c8e0       _cff_vstore_done           1000d8e0 f   cffload.obj
 0001:0000c980       _cff_vstore_load           1000d980 f   cffload.obj
 0001:0000d850       _cff_make_private_dict     1000e850 f   cffobjs.obj
 0001:0000e060       _remove_style              1000f060 f   cffobjs.obj
 0001:0000e0e0       _cff_parse_font_matrix     1000f0e0 f   cffparse.obj
 0001:0000e360       _cff_parse_font_bbox       1000f360 f   cffparse.obj
 0001:0000e4f0       _cff_parse_private_dict    1000f4f0 f   cffparse.obj
 0001:0000e590       _cff_parse_multiple_master 1000f590 f   cffparse.obj
 0001:0000e640       _cff_parse_cid_ros         1000f640 f   cffparse.obj
 0001:0000e770       _cff_parse_vsindex         1000f770 f   cffparse.obj
 0001:0000e7c0       _cff_parse_blend           1000f7c0 f   cffparse.obj
 0001:0000e860       _cff_parse_maxstack        1000f860 f   cffparse.obj
 0001:0000e8e0       _cff_parse_integer         1000f8e0 f   cffparse.obj
 0001:0000e9e0       _cff_parse_real            1000f9e0 f   cffparse.obj
 0001:0000f160       $LN115                     10010160     cffparse.obj
 0001:0000f180       _do_fixed                  10010180 f   cffparse.obj
 0001:0000f210       _cid_load_glyph            10010210 f   cidgload.obj
 0001:0000fae0       _cid_parse_font_matrix     10010ae0 f   cidload.obj
 0001:0000fc40       _parse_fd_array            10010c40 f   cidload.obj
 0001:0000fd10       _parse_expansion_factor    10010d10 f   cidload.obj
 0001:0000fff0       _cid_hex_to_binary         10010ff0 f   cidload.obj
 0001:00010180       _cid_parse_dict            10011180 f   cidload.obj
 0001:00010394       $LN88                      10011394     cidload.obj
 0001:000103b0       _cid_read_subrs            100113b0 f   cidload.obj
 0001:00011090       _cid_get_postscript_name   10012090 f   cidriver.obj
 0001:000110b0       _cid_ps_get_font_info      100120b0 f   cidriver.obj
 0001:000110d0       _cid_ps_get_font_extra     100120d0 f   cidriver.obj
 0001:000110f0       _cid_get_ros               100120f0 f   cidriver.obj
 0001:00011130       _cid_get_is_cid            10012130 f   cidriver.obj
 0001:00011140       _cid_get_cid_from_glyph_index 10012140 f   cidriver.obj
 0001:00011160       _cid_get_interface         10012160 f   cidriver.obj
 0001:00011320       __ft_face_scale_advances   10012320 f   ftadvanc.obj
 0001:00011380       _BBox_Move_To              10012380 f   ftbbox.obj
 0001:000113c0       _BBox_Line_To              100123c0 f   ftbbox.obj
 0001:000113e0       _BBox_Conic_To             100123e0 f   ftbbox.obj
 0001:000114a0       _BBox_Cubic_To             100124a0 f   ftbbox.obj
 0001:00011530       _BBox_Cubic_Check          10012530 f   ftbbox.obj
 0001:000117b0       _cubic_peak                100127b0 f   ftbbox.obj
 0001:00012338       $LN115                     10013338     ftbitmap.obj
 0001:000127d0       $LN81                      100137d0     ftbitmap.obj
 0001:00012890       _ft_bitmap_assure_buffer   10013890 f   ftbitmap.obj
 0001:00012ac0       $LN47                      10013ac0     ftbitmap.obj
 0001:00013a50       _FT_GlyphLoader_Adjust_Points 10014a50 f   ftgloadr.obj
 0001:00013e80       _ft_bitmap_glyph_copy      10014e80 f   ftglyph.obj
 0001:00013eb0       _ft_bitmap_glyph_done      10014eb0 f   ftglyph.obj
 0001:00013ed0       _ft_bitmap_glyph_bbox      10014ed0 f   ftglyph.obj
 0001:00013f10       _ft_outline_glyph_init     10014f10 f   ftglyph.obj
 0001:00013f60       _ft_outline_glyph_done     10014f60 f   ftglyph.obj
 0001:00013f80       _ft_outline_glyph_copy     10014f80 f   ftglyph.obj
 0001:00013fc0       _ft_outline_glyph_transform 10014fc0 f   ftglyph.obj
 0001:00014000       _ft_outline_glyph_bbox     10015000 f   ftglyph.obj
 0001:00014010       _ft_outline_glyph_prepare  10015010 f   ftglyph.obj
 0001:00014040       _ft_bitmap_glyph_init      10015040 f   ftglyph.obj
 0001:00014690       _ft_new_glyph              10015690 f   ftglyph.obj
 0001:000146e0       _gray_move_to              100156e0 f   ftgrays.obj
 0001:00014720       _gray_line_to              10015720 f   ftgrays.obj
 0001:00014740       _gray_conic_to             10015740 f   ftgrays.obj
 0001:00014760       _gray_cubic_to             10015760 f   ftgrays.obj
 0001:00014780       _gray_raster_render        10015780 f   ftgrays.obj
 0001:00014910       _gray_raster_new           10015910 f   ftgrays.obj
 0001:00014910       _ft_black_new              10015910 f   ftraster.obj
 0001:00014950       _gray_raster_done          10015950 f   ftgrays.obj
 0001:00014950       _ft_black_done             10015950 f   ftraster.obj
 0001:00014960       _gray_convert_glyph        10015960 f   ftgrays.obj
 0001:00014ba0       _gray_convert_glyph_inner  10015ba0 f   ftgrays.obj
 0001:00014bf0       _gray_render_conic         10015bf0 f   ftgrays.obj
 0001:00014f60       _gray_render_cubic         10015f60 f   ftgrays.obj
 0001:000151b0       _gray_render_line          100161b0 f   ftgrays.obj
 0001:000155c0       _gray_set_cell             100165c0 f   ftgrays.obj
 0001:00015640       _gray_sweep                10016640 f   ftgrays.obj
 0001:000157d8       $LN64                      100167d8     ftgrays.obj
 0001:000157f8       $LN65                      100167f8     ftgrays.obj
 0001:00015820       _gray_sweep_direct         10016820 f   ftgrays.obj
 0001:00015af0       _hash_bucket               10016af0 f   fthash.obj
 0001:00015b50       _hash_insert               10016b50 f   fthash.obj
 0001:00015c70       _hash_num_compare          10016c70 f   fthash.obj
 0001:00015c80       _hash_num_lookup           10016c80 f   fthash.obj
 0001:000168c0       _ft_face_get_mvar_service  100178c0 f   ftmm.obj
 0001:00018fc4       $LN39                      10019fc4     ftobjs.obj
 0001:00019810       _IsMacResource             1001a810 f   ftobjs.obj
 0001:00019a90       _Mac_Read_POST_Resource    1001aa90 f   ftobjs.obj
 0001:00019da0       _destroy_charmaps          1001ada0 f   ftobjs.obj
 0001:00019e10       _destroy_face              1001ae10 f   ftobjs.obj
 0001:00019f40       _destroy_size              1001af40 f   ftobjs.obj
 0001:00019f90       _find_unicode_charmap      1001af90 f   ftobjs.obj
 0001:0001a010       _find_variant_selector_charmap 1001b010 f   ftobjs.obj
 0001:0001a0a0       _ft_cmap_done_internal     1001b0a0 f   ftobjs.obj
 0001:0001a120       _ft_glyphslot_done         1001b120 f   ftobjs.obj
 0001:0001a5d0       _ft_open_face_internal     1001b5d0 f   ftobjs.obj
 0001:0001ae30       _ft_recompute_scaled_metrics 1001be30 f   ftobjs.obj
 0001:0001b070       _load_face_in_embedded_rfork 1001c070 f   ftobjs.obj
 0001:0001b250       _memory_stream_close       1001c250 f   ftobjs.obj
 0001:0001b280       _open_face                 1001c280 f   ftobjs.obj
 0001:0001cd90       _ft_black_render           1001dd90 f   ftraster.obj
 0001:0001cf30       _Bezier_Up                 1001df30 f   ftraster.obj
 0001:0001d0b0       _Conic_To                  1001e0b0 f   ftraster.obj
 0001:0001d2c0       _Convert_Glyph             1001e2c0 f   ftraster.obj
 0001:0001d520       _Cubic_To                  1001e520 f   ftraster.obj
 0001:0001d710       _Decompose_Curve           1001e710 f   ftraster.obj
 0001:0001da90       _Draw_Sweep                1001ea90 f   ftraster.obj
 0001:0001e0e0       _End_Profile               1001f0e0 f   ftraster.obj
 0001:0001e170       _Horizontal_Sweep_Drop     1001f170 f   ftraster.obj
 0001:0001e2e0       $LN34                      1001f2e0     ftraster.obj
 0001:0001e300       _Horizontal_Sweep_Span     1001f300 f   ftraster.obj
 0001:0001e3a0       _Line_To                   1001f3a0 f   ftraster.obj
 0001:0001e520       _Line_Up                   1001f520 f   ftraster.obj
 0001:0001e6e0       _New_Profile               1001f6e0 f   ftraster.obj
 0001:0001e7a0       _Render_Glyph              1001f7a0 f   ftraster.obj
 0001:0001e8d0       _Render_Single_Pass        1001f8d0 f   ftraster.obj
 0001:0001e9b0       _Split_Conic               1001f9b0 f   ftraster.obj
 0001:0001ea00       _Split_Cubic               1001fa00 f   ftraster.obj
 0001:0001ea90       _Vertical_Sweep_Drop       1001fa90 f   ftraster.obj
 0001:0001ec00       $LN34                      1001fc00     ftraster.obj
 0001:0001ec20       _Vertical_Sweep_Init       1001fc20 f   ftraster.obj
 0001:0001ec40       _Vertical_Sweep_Span       1001fc40 f   ftraster.obj
 0001:0001ed10       _Vertical_Sweep_Step       1001fd10 f   ftraster.obj
 0001:0001ed20       _ft_raster1_init           1001fd20 f   ftrend1.obj
 0001:0001ed40       _ft_raster1_set_mode       1001fd40 f   ftrend1.obj
 0001:0001ed40       _ft_smooth_set_mode        1001fd40 f   ftsmooth.obj
 0001:0001ed60       _ft_raster1_transform      1001fd60 f   ftrend1.obj
 0001:0001ed60       _ft_smooth_transform       1001fd60 f   ftsmooth.obj
 0001:0001edb0       _ft_raster1_get_cbox       1001fdb0 f   ftrend1.obj
 0001:0001edb0       _ft_smooth_get_cbox        1001fdb0 f   ftsmooth.obj
 0001:0001ede0       _ft_raster1_render         1001fde0 f   ftrend1.obj
 0001:0001efb0       _raccess_guess_darwin_hfsplus 1001ffb0 f   ftrfork.obj
 0001:0001f030       _raccess_guess_vfat        10020030 f   ftrfork.obj
 0001:0001f070       _raccess_guess_linux_cap   10020070 f   ftrfork.obj
 0001:0001f0b0       _raccess_guess_linux_double 100200b0 f   ftrfork.obj
 0001:0001f110       _raccess_guess_linux_netatalk 10020110 f   ftrfork.obj
 0001:0001f170       _raccess_guess_apple_double 10020170 f   ftrfork.obj
 0001:0001f1a0       _raccess_guess_apple_single 100201a0 f   ftrfork.obj
 0001:0001f1d0       _raccess_guess_darwin_ufs_export 100201d0 f   ftrfork.obj
 0001:0001f230       _raccess_guess_darwin_newvfs 10020230 f   ftrfork.obj
 0001:0001f880       _ft_raccess_sort_ref_by_id 10020880 f   ftrfork.obj
 0001:0001f8a0       _raccess_guess_apple_generic 100208a0 f   ftrfork.obj
 0001:0001f9b0       _raccess_guess_linux_double_from_file_name 100209b0 f   ftrfork.obj
 0001:0001fa30       _raccess_make_file_name    10020a30 f   ftrfork.obj
 0001:0001fb20       _ft_smooth_init            10020b20 f   ftsmooth.obj
 0001:0001fb70       _ft_smooth_render          10020b70 f   ftsmooth.obj
 0001:00020110       _ft_smooth_lcd_spans       10021110 f   ftsmooth.obj
 0001:00020170       _ft_smooth_overlap_spans   10021170 f   ftsmooth.obj
 0001:000209e4       $LN50                      100219e4     ftstream.obj
 0001:00020a0c       $LN49                      10021a0c     ftstream.obj
 0001:000225f0       _ft_cubic_is_small_enough  100235f0 f   ftstroke.obj
 0001:000227d0       _ft_stroke_border_arcto    100237d0 f   ftstroke.obj
 0001:00022a30       _ft_stroke_border_close    10023a30 f   ftstroke.obj
 0001:00022b00       _ft_stroke_border_cubicto  10023b00 f   ftstroke.obj
 0001:00022b70       _ft_stroke_border_get_counts 10023b70 f   ftstroke.obj
 0001:00022c00       _ft_stroke_border_grow     10023c00 f   ftstroke.obj
 0001:00022c80       _ft_stroke_border_lineto   10023c80 f   ftstroke.obj
 0001:00022d20       _ft_stroker_cap            10023d20 f   ftstroke.obj
 0001:00022e40       _ft_stroker_outside        10023e40 f   ftstroke.obj
 0001:00023140       _ft_stroker_process_corner 10024140 f   ftstroke.obj
 0001:000232a0       _ft_stroker_subpath_start  100242a0 f   ftstroke.obj
 0001:000235c0       _ft_alloc                  100245c0 f   ftsystem.obj
 0001:000235d0       _ft_ansi_stream_close      100245d0 f   ftsystem.obj
 0001:00023600       _ft_ansi_stream_io         10024600 f   ftsystem.obj
 0001:00023650       _ft_free                   10024650 f   ftsystem.obj
 0001:00023660       _ft_realloc                10024660 f   ftsystem.obj
 0001:00023a90       _ft_trig_downscale         10024a90 f   fttrigon.obj
 0001:00023ad0       _ft_trig_prenorm           10024ad0 f   fttrigon.obj
 0001:00023b20       _ft_trig_pseudo_polarize   10024b20 f   fttrigon.obj
 0001:00023bf0       _ft_trig_pseudo_rotate     10024bf0 f   fttrigon.obj
 0001:000244a0       _cf2_arrstack_setNumElements 100254a0 f   psarrst.obj
 0001:00025160       _cf2_computeDarkening      10026160 f   psfont.obj
 0001:00025380       _cf2_font_setup            10026380 f   psfont.obj
 0001:000257a0       _cf2_builder_cubeTo        100267a0 f   psft.obj
 0001:00025820       _cf2_builder_lineTo        10026820 f   psft.obj
 0001:00025870       _cf2_builder_moveTo        10026870 f   psft.obj
 0001:00025c60       _cf2_free_instance         10026c60 f   psft.obj
 0001:000267d0       _psh_glyph_init            100277d0 f   pshalgo.obj
 0001:00026c40       _psh_glyph_interpolate_normal_points 10027c40 f   pshalgo.obj
 0001:00026ed0       _psh_glyph_interpolate_other_points 10027ed0 f   pshalgo.obj
 0001:00027130       _psh_glyph_load_points     10028130 f   pshalgo.obj
 0001:000271b0       _psh_hint_align            100281b0 f   pshalgo.obj
 0001:00027570       _psh_hint_table_activate_mask 10028570 f   pshalgo.obj
 0001:00027640       _psh_hint_table_align_hints 10028640 f   pshalgo.obj
 0001:00027a40       _psh_hint_table_done       10028a40 f   pshalgo.obj
 0001:00027ab0       _psh_hint_table_find_strong_points 10028ab0 f   pshalgo.obj
 0001:00027c80       _psh_hint_table_init       10028c80 f   pshalgo.obj
 0001:00027ec0       _psh_hint_table_record     10028ec0 f   pshalgo.obj
 0001:00027f40       _psh_blues_scale_zones     10028f40 f   pshglob.obj
 0001:00028200       _psh_blues_set_zones       10029200 f   pshglob.obj
 0001:00028380       _psh_blues_set_zones_0     10029380 f   pshglob.obj
 0001:00028590       _psh_globals_destroy       10029590 f   pshglob.obj
 0001:00028600       _psh_globals_new           10029600 f   pshglob.obj
 0001:00028870       _psh_globals_scale_widths  10029870 f   pshglob.obj
 0001:00028bb0       _cf2_glyphpath_computeIntersection 10029bb0 f   pshints.obj
 0001:00028e60       _cf2_glyphpath_computeOffset 10029e60 f   pshints.obj
 0001:00029370       _cf2_glyphpath_hintPoint   1002a370 f   pshints.obj
 0001:00029a70       _cf2_glyphpath_pushMove    1002aa70 f   pshints.obj
 0001:00029b20       _cf2_glyphpath_pushPrevElem 1002ab20 f   pshints.obj
 0001:00029d70       _cf2_hint_init             1002ad70 f   pshints.obj
 0001:00029f00       _cf2_hintmap_adjustHints   1002af00 f   pshints.obj
 0001:0002a530       _cf2_hintmap_insertHint    1002b530 f   pshints.obj
 0001:0002a740       _cf2_hintmap_map           1002b740 f   pshints.obj
 0001:0002a870       _ps_hinter_done            1002b870 f   pshmod.obj
 0001:0002a8a0       _ps_hinter_init            1002b8a0 f   pshmod.obj
 0001:0002a8e0       _pshinter_get_globals_funcs 1002b8e0 f   pshmod.obj
 0001:0002a8f0       _pshinter_get_t1_funcs     1002b8f0 f   pshmod.obj
 0001:0002a900       _pshinter_get_t2_funcs     1002b900 f   pshmod.obj
 0001:0002a910       _ps_dimension_add_counter  1002b910 f   pshrec.obj
 0001:0002ab50       _ps_dimension_add_t1stem   1002bb50 f   pshrec.obj
 0001:0002acd0       _ps_dimension_set_mask_bits 1002bcd0 f   pshrec.obj
 0001:0002ae00       _ps_hints_close            1002be00 f   pshrec.obj
 0001:0002af00       _ps_hints_stem             1002bf00 f   pshrec.obj
 0001:0002b100       _ps_hints_t1reset          1002c100 f   pshrec.obj
 0001:0002b180       _ps_hints_t1stem3          1002c180 f   pshrec.obj
 0001:0002b260       _ps_hints_t2counter        1002c260 f   pshrec.obj
 0001:0002b2c0       _ps_hints_t2mask           1002c2c0 f   pshrec.obj
 0001:0002b320       _ps_mask_ensure            1002c320 f   pshrec.obj
 0001:0002b380       _ps_mask_table_alloc       1002c380 f   pshrec.obj
 0001:0002b420       _ps_mask_table_done        1002c420 f   pshrec.obj
 0001:0002b490       _ps_mask_table_merge_all   1002c490 f   pshrec.obj
 0001:0002b670       _t1_hints_open             1002c670 f   pshrec.obj
 0001:0002b6b0       _t1_hints_stem             1002c6b0 f   pshrec.obj
 0001:0002b740       _t2_hints_open             1002c740 f   pshrec.obj
 0001:0002b780       _t2_hints_stems            1002c780 f   pshrec.obj
 0001:0002b8c0       _cf2_doFlex                1002c8c0 f   psintrp.obj
 0001:0002ba80       _cf2_doStems               1002ca80 f   psintrp.obj
 0001:0002bc20       _cf2_hintmask_read         1002cc20 f   psintrp.obj
 0001:0002e0bc       $LN803                     1002f0bc     psintrp.obj
 0001:0002e13c       $LN805                     1002f13c     psintrp.obj
 0001:0002e154       $LN804                     1002f154     psintrp.obj
 0001:0002e174       $LN806                     1002f174     psintrp.obj
 0001:0002e1fc       $LN808                     1002f1fc     psintrp.obj
 0001:0002e23c       $LN807                     1002f23c     psintrp.obj
 0001:0002e260       _ps_unicode_value          1002f260 f   psmodule.obj
 0001:0002e400       _ps_unicodes_init          1002f400 f   psmodule.obj
 0001:0002e740       _ps_unicodes_char_index    1002f740 f   psmodule.obj
 0001:0002e7b0       _ps_unicodes_char_next     1002f7b0 f   psmodule.obj
 0001:0002e870       _ps_get_macintosh_name     1002f870 f   psmodule.obj
 0001:0002e890       _ps_get_standard_strings   1002f890 f   psmodule.obj
 0001:0002e8b0       _psnames_get_service       1002f8b0 f   psmodule.obj
 0001:0002e8c0       _compare_uni_maps          1002f8c0 f   psmodule.obj
 0001:0002f5e4       $LN121                     100305e4     psobjs.obj
 0001:0002ff10       _ps_table_realloc          10030f10 f   psobjs.obj
 0001:0002ffd0       _ps_tofixedarray           10030fd0 f   psobjs.obj
 0001:00030110       _skip_comment              10031110 f   psobjs.obj
 0001:00030140       _skip_literal_string       10031140 f   psobjs.obj
 0001:000301c4       $LN34                      100311c4     psobjs.obj
 0001:000301cc       $LN33                      100311cc     psobjs.obj
 0001:00030220       _skip_procedure            10031220 f   psobjs.obj
 0001:000302d4       $LN36                      100312d4     psobjs.obj
 0001:000302ec       $LN35                      100312ec     psobjs.obj
 0001:00030350       _skip_spaces               10031350 f   psobjs.obj
 0001:000303b0       _skip_string               100313b0 f   psobjs.obj
 0001:00030df0       _get_sfnt_table            10031df0 f   sfdriver.obj
 0001:00030e6c       $LN19                      10031e6c     sfdriver.obj
 0001:00030e90       _sfnt_table_info           10031e90 f   sfdriver.obj
 0001:00030f00       _sfnt_get_glyph_name       10031f00 f   sfdriver.obj
 0001:00030f40       _sfnt_get_name_index       10031f40 f   sfdriver.obj
 0001:00030fc0       _sfnt_get_name_id          10031fc0 f   sfdriver.obj
 0001:000310a0       _sfnt_get_ps_name          100320a0 f   sfdriver.obj
 0001:00031180       _sfnt_get_interface        10032180 f   sfdriver.obj
 0001:00031190       _fixed2float               10032190 f   sfdriver.obj
 0001:00031300       _get_apple_string          10032300 f   sfdriver.obj
 0001:000313f0       _get_win_string            100323f0 f   sfdriver.obj
 0001:00031500       _murmur_hash_3_128         10032500 f   sfdriver.obj
 0001:000317b0       $LN35                      100327b0     sfdriver.obj
 0001:000317f0       _sfnt_get_var_ps_name      100327f0 f   sfdriver.obj
 0001:00031ce0       _sfnt_is_alphanumeric      10032ce0 f   sfdriver.obj
 0001:00031d10       _sfnt_is_postscript        10032d10 f   sfdriver.obj
 0001:00033200       $LN51                      10034200     sfobjs.obj
 0001:00033210       _tt_name_ascii_from_other  10034210 f   sfobjs.obj
 0001:00033280       _tt_name_ascii_from_utf16  10034280 f   sfobjs.obj
 0001:000336a0       _T1_Read_PFM               100346a0 f   t1afm.obj
 0001:000338d0       _t1_get_index              100348d0 f   t1afm.obj
 0001:00033950       _t1_cmap_std_done          10034950 f   t1cmap.obj
 0001:00033980       _t1_cmap_std_char_index    10034980 f   t1cmap.obj
 0001:00033a10       _t1_cmap_std_char_next     10034a10 f   t1cmap.obj
 0001:00033ad0       _t1_cmap_standard_init     10034ad0 f   t1cmap.obj
 0001:00033b00       _t1_cmap_expert_init       10034b00 f   t1cmap.obj
 0001:00033b30       _t1_cmap_custom_init       10034b30 f   t1cmap.obj
 0001:00033b60       _t1_cmap_custom_done       10034b60 f   t1cmap.obj
 0001:00033b80       _t1_cmap_custom_char_index 10034b80 f   t1cmap.obj
 0001:00033bb0       _t1_cmap_custom_char_next  10034bb0 f   t1cmap.obj
 0001:00033c10       _t1_cmap_unicode_init      10034c10 f   t1cmap.obj
 0001:00033c50       _t1_cmap_unicode_char_index 10034c50 f   t1cmap.obj
 0001:00033c70       _t1_cmap_unicode_char_next 10034c70 f   t1cmap.obj
 0001:00033c90       _psaux_get_glyph_name      10034c90 f   t1cmap.obj
 0001:00034104       $LN148                     10035104     t1decode.obj
 0001:00034120       $LN147                     10035120     t1decode.obj
 0001:00034220       $LN150                     10035220     t1decode.obj
 0001:00034238       $LN149                     10035238     t1decode.obj
 0001:000342e0       _t1_get_glyph_name         100352e0 f   t1driver.obj
 0001:00034310       _t1_get_name_index         10035310 f   t1driver.obj
 0001:00034380       _t1_get_ps_name            10035380 f   t1driver.obj
 0001:00034390       _t1_ps_get_font_info       10035390 f   t1driver.obj
 0001:000343b0       _t1_ps_get_font_extra      100353b0 f   t1driver.obj
 0001:000343d0       _t1_ps_has_glyph_names     100353d0 f   t1driver.obj
 0001:000343e0       _t1_ps_get_font_private    100353e0 f   t1driver.obj
 0001:00034400       _t1_ps_get_font_value      10035400 f   t1driver.obj
 0001:00034e7c       $LN133                     10035e7c     t1driver.obj
 0001:00034f34       $LN134                     10035f34     t1driver.obj
 0001:00034f44       $LN135                     10035f44     t1driver.obj
 0001:00034f60       _Get_Interface             10035f60 f   t1driver.obj
 0001:00034f70       _Get_Kerning               10035f70 f   t1driver.obj
 0001:00035820       _T1_Parse_Glyph            10036820 f   t1gload.obj
 0001:00035880       _T1_Parse_Glyph_And_Get_Char_String 10036880 f   t1gload.obj
 0001:00035a90       _parse_blend_axis_types    10036a90 f   t1load.obj
 0001:00035c00       _parse_blend_design_positions 10036c00 f   t1load.obj
 0001:00035e50       _parse_blend_design_map    10036e50 f   t1load.obj
 0001:00036030       _parse_weight_vector       10037030 f   t1load.obj
 0001:00036190       _parse_buildchar           10037190 f   t1load.obj
 0001:000361b0       _parse_private             100371b0 f   t1load.obj
 0001:000361c0       _t1_parse_font_matrix      100371c0 f   t1load.obj
 0001:000362f0       _parse_encoding            100372f0 f   t1load.obj
 0001:00036720       _parse_subrs               10037720 f   t1load.obj
 0001:00036a60       _parse_charstrings         10037a60 f   t1load.obj
 0001:00038060       _mm_axis_unmap             10039060 f   t1load.obj
 0001:000380e0       _mm_weights_unmap          100390e0 f   t1load.obj
 0001:000381b0       _parse_dict                100391b0 f   t1load.obj
 0001:000385e0       _read_binary_data          100395e0 f   t1load.obj
 0001:00038660       _t1_allocate_blend         10039660 f   t1load.obj
 0001:000387e0       _t1_load_keyword           100397e0 f   t1load.obj
 0001:000388f8       $LN38                      100398f8     t1load.obj
 0001:00038920       _t1_set_mm_blend           10039920 f   t1load.obj
 0001:00038fec       $LN76                      10039fec     t1objs.obj
 0001:000397a0       _check_type1_format        1003a7a0 f   t1parse.obj
 0001:00039870       _read_pfb_tag              1003a870 f   t1parse.obj
 0001:000398e0       _tt_cmap_init              1003a8e0 f   ttcmap.obj
 0001:000398f0       _tt_cmap0_validate         1003a8f0 f   ttcmap.obj
 0001:00039970       _tt_cmap0_char_index       1003a970 f   ttcmap.obj
 0001:00039990       _tt_cmap0_char_next        1003a990 f   ttcmap.obj
 0001:000399d0       _tt_cmap0_get_info         1003a9d0 f   ttcmap.obj
 0001:00039a00       _tt_cmap2_validate         1003aa00 f   ttcmap.obj
 0001:00039bc0       _tt_cmap2_char_index       1003abc0 f   ttcmap.obj
 0001:00039c50       _tt_cmap2_char_next        1003ac50 f   ttcmap.obj
 0001:00039e10       _tt_cmap2_get_info         1003ae10 f   ttcmap.obj
 0001:00039e40       _tt_cmap4_init             1003ae40 f   ttcmap.obj
 0001:00039e80       _tt_cmap4_validate         1003ae80 f   ttcmap.obj
 0001:0003a260       _tt_cmap4_char_index       1003b260 f   ttcmap.obj
 0001:0003a2a0       _tt_cmap4_char_next        1003b2a0 f   ttcmap.obj
 0001:0003a300       _tt_cmap4_get_info         1003b300 f   ttcmap.obj
 0001:0003a330       _tt_cmap6_validate         1003b330 f   ttcmap.obj
 0001:0003a3c0       _tt_cmap6_char_index       1003b3c0 f   ttcmap.obj
 0001:0003a410       _tt_cmap6_char_next        1003b410 f   ttcmap.obj
 0001:0003a4b0       _tt_cmap6_get_info         1003b4b0 f   ttcmap.obj
 0001:0003a4e0       _tt_cmap8_validate         1003b4e0 f   ttcmap.obj
 0001:0003a760       _tt_cmap8_char_index       1003b760 f   ttcmap.obj
 0001:0003a840       _tt_cmap8_char_next        1003b840 f   ttcmap.obj
 0001:0003a980       _tt_cmap8_get_info         1003b980 f   ttcmap.obj
 0001:0003a9c0       _tt_cmap10_validate        1003b9c0 f   ttcmap.obj
 0001:0003aa80       _tt_cmap10_char_index      1003ba80 f   ttcmap.obj
 0001:0003ab00       _tt_cmap10_char_next       1003bb00 f   ttcmap.obj
 0001:0003aba0       _tt_cmap10_get_info        1003bba0 f   ttcmap.obj
 0001:0003abe0       _tt_cmap12_init            1003bbe0 f   ttcmap.obj
 0001:0003abe0       _tt_cmap13_init            1003bbe0 f   ttcmap.obj
 0001:0003ac20       _tt_cmap12_validate        1003bc20 f   ttcmap.obj
 0001:0003ad90       _tt_cmap12_char_index      1003bd90 f   ttcmap.obj
 0001:0003adb0       _tt_cmap12_char_next       1003bdb0 f   ttcmap.obj
 0001:0003ae00       _tt_cmap12_get_info        1003be00 f   ttcmap.obj
 0001:0003ae40       _tt_cmap13_validate        1003be40 f   ttcmap.obj
 0001:0003afb0       _tt_cmap13_char_index      1003bfb0 f   ttcmap.obj
 0001:0003afd0       _tt_cmap13_char_next       1003bfd0 f   ttcmap.obj
 0001:0003b020       _tt_cmap13_get_info        1003c020 f   ttcmap.obj
 0001:0003b060       _tt_cmap14_done            1003c060 f   ttcmap.obj
 0001:0003b090       _tt_cmap14_init            1003c090 f   ttcmap.obj
 0001:0003b0d0       _tt_cmap14_validate        1003c0d0 f   ttcmap.obj
 0001:0003b3d0       _tt_cmap14_char_next       1003c3d0 f   ttcmap.obj
 0001:0003b3e0       _tt_cmap14_get_info        1003c3e0 f   ttcmap.obj
 0001:0003b400       _tt_cmap14_char_var_index  1003c400 f   ttcmap.obj
 0001:0003b4b0       _tt_cmap14_char_var_isdefault 1003c4b0 f   ttcmap.obj
 0001:0003b560       _tt_cmap14_variants        1003c560 f   ttcmap.obj
 0001:0003b5f0       _tt_cmap14_char_variants   1003c5f0 f   ttcmap.obj
 0001:0003b720       _tt_cmap14_variant_chars   1003c720 f   ttcmap.obj
 0001:0003ba20       _tt_cmap_unicode_init      1003ca20 f   ttcmap.obj
 0001:0003ba50       _tt_cmap_unicode_char_index 1003ca50 f   ttcmap.obj
 0001:0003ba70       _tt_cmap_unicode_char_next 1003ca70 f   ttcmap.obj
 0001:0003ba90       _tt_cmap12_char_map_binary 1003ca90 f   ttcmap.obj
 0001:0003bc20       _tt_cmap12_next            1003cc20 f   ttcmap.obj
 0001:0003bd30       _tt_cmap13_char_map_binary 1003cd30 f   ttcmap.obj
 0001:0003bec0       _tt_cmap13_next            1003cec0 f   ttcmap.obj
 0001:0003bf80       _tt_cmap14_char_map_def_binary 1003cf80 f   ttcmap.obj
 0001:0003c000       _tt_cmap14_char_map_nondef_binary 1003d000 f   ttcmap.obj
 0001:0003c090       _tt_cmap14_def_char_count  1003d090 f   ttcmap.obj
 0001:0003c0e0       _tt_cmap14_ensure          1003d0e0 f   ttcmap.obj
 0001:0003c130       _tt_cmap14_find_variant    1003d130 f   ttcmap.obj
 0001:0003c1b0       _tt_cmap14_get_def_chars   1003d1b0 f   ttcmap.obj
 0001:0003c280       _tt_cmap14_get_nondef_chars 1003d280 f   ttcmap.obj
 0001:0003c330       _tt_cmap2_get_subheader    1003d330 f   ttcmap.obj
 0001:0003c390       _tt_cmap4_char_map_binary  1003d390 f   ttcmap.obj
 0001:0003c8e0       _tt_cmap4_char_map_linear  1003d8e0 f   ttcmap.obj
 0001:0003cb10       _tt_cmap4_next             1003db10 f   ttcmap.obj
 0001:0003cc10       _tt_cmap4_set_range        1003dc10 f   ttcmap.obj
 0001:0003cfb0       _tt_get_glyph_name         1003dfb0 f   ttcmap.obj
 0001:0003cfe0       _get_child_table_pointer   1003dfe0 f   ttcolr.obj
 0001:0003d030       _read_color_line           1003e030 f   ttcolr.obj
 0001:0003d070       _read_paint                1003e070 f   ttcolr.obj
 0001:0003ec80       _tt_property_set           1003fc80 f   ttdriver.obj
 0001:0003ed00       _tt_property_get           1003fd00 f   ttdriver.obj
 0001:0003ed50       _tt_get_advances           1003fd50 f   ttdriver.obj
 0001:0003ee30       _tt_size_select            1003fe30 f   ttdriver.obj
 0001:0003ee80       _tt_size_request           1003fe80 f   ttdriver.obj
 0001:0003ef80       _tt_glyph_load             1003ff80 f   ttdriver.obj
 0001:0003f030       _tt_get_interface          10040030 f   ttdriver.obj
 0001:0003f090       _TT_Access_Glyph_Frame     10040090 f   ttgload.obj
 0001:0003f0e0       _TT_Forget_Glyph_Frame     100400e0 f   ttgload.obj
 0001:0003f1d0       _TT_Hint_Glyph             100401d0 f   ttgload.obj
 0001:0003f4c0       _TT_Load_Composite_Glyph   100404c0 f   ttgload.obj
 0001:0003fd18       $LN67                      10040d18     ttgload.obj
 0001:0003fd30       _TT_Load_Glyph_Header      10040d30 f   ttgload.obj
 0001:0003fdc0       _TT_Load_Simple_Glyph      10040dc0 f   ttgload.obj
 0001:00040220       _TT_Process_Composite_Component 10041220 f   ttgload.obj
 0001:00040420       _TT_Process_Composite_Glyph 10041420 f   ttgload.obj
 0001:00040640       _TT_Process_Simple_Glyph   10041640 f   ttgload.obj
 0001:00040b40       _compute_glyph_metrics     10041b40 f   ttgload.obj
 0001:00040d80       _load_truetype_glyph       10041d80 f   ttgload.obj
 0001:00041c10       _tt_get_metrics_incremental 10042c10 f   ttgload.obj
 0001:00041cc0       _tt_loader_done            10042cc0 f   ttgload.obj
 0001:00041ce0       _tt_loader_init            10042ce0 f   ttgload.obj
 0001:00042010       _tt_loader_set_pp          10043010 f   ttgload.obj
 0001:000420b0       _tt_prepare_zone           100430b0 f   ttgload.obj
 0001:000435d0       _ft_var_apply_tuple        100445d0 f   ttgxvar.obj
 0001:000436a0       _ft_var_done_item_variation_store 100446a0 f   ttgxvar.obj
 0001:00043760       _ft_var_get_item_delta     10044760 f   ttgxvar.obj
 0001:000438c0       _ft_var_get_value_pointer  100448c0 f   ttgxvar.obj
 0001:00043c2c       $LN74                      10044c2c     ttgxvar.obj
 0001:00043c50       _ft_var_load_avar          10044c50 f   ttgxvar.obj
 0001:00043e10       _ft_var_load_delta_set_index_mapping 10044e10 f   ttgxvar.obj
 0001:00043fd0       _ft_var_load_gvar          10044fd0 f   ttgxvar.obj
 0001:000442f0       _ft_var_load_hvvar         100452f0 f   ttgxvar.obj
 0001:00044480       _ft_var_load_item_variation_store 10045480 f   ttgxvar.obj
 0001:00044980       _ft_var_load_mvar          10045980 f   ttgxvar.obj
 0001:00044bd0       _ft_var_readpackeddeltas   10045bd0 f   ttgxvar.obj
 0001:00044d20       _ft_var_readpackedpoints   10045d20 f   ttgxvar.obj
 0001:00044e90       _ft_var_to_design          10045e90 f   ttgxvar.obj
 0001:00045030       _ft_var_to_normalized      10046030 f   ttgxvar.obj
 0001:000452c0       _tt_cvt_ready_iterator     100462c0 f   ttgxvar.obj
 0001:000452e0       _tt_delta_interpolate      100462e0 f   ttgxvar.obj
 0001:00045c50       _tt_hvadvance_adjust       10046c50 f   ttgxvar.obj
 0001:00045d30       _tt_interpolate_deltas     10046d30 f   ttgxvar.obj
 0001:00045e70       _tt_set_mm_blend           10046e70 f   ttgxvar.obj
 0001:00046170       _tt_size_reset_iterator    10047170 f   ttgxvar.obj
 0001:000461b0       _Compute_Funcs             100471b0 f   ttinterp.obj
 0001:00046300       _Compute_Point_Displacement 10047300 f   ttinterp.obj
 0001:000463e0       _Current_Ppem              100473e0 f   ttinterp.obj
 0001:000463f0       _Current_Ppem_Stretched    100473f0 f   ttinterp.obj
 0001:00046440       _Current_Ratio             10047440 f   ttinterp.obj
 0001:000464c0       _Direct_Move               100474c0 f   ttinterp.obj
 0001:00046580       _Direct_Move_Orig          10047580 f   ttinterp.obj
 0001:000465f0       _Direct_Move_Orig_X        100475f0 f   ttinterp.obj
 0001:00046610       _Direct_Move_Orig_Y        10047610 f   ttinterp.obj
 0001:00046630       _Direct_Move_X             10047630 f   ttinterp.obj
 0001:00046680       _Direct_Move_Y             10047680 f   ttinterp.obj
 0001:000466e0       _Dual_Project              100476e0 f   ttinterp.obj
 0001:00046710       _Ins_Goto_CodeRange        10047710 f   ttinterp.obj
 0001:00046780       _Ins_IP                    10047780 f   ttinterp.obj
 0001:00046ac0       _Ins_ISECT                 10047ac0 f   ttinterp.obj
 0001:00046d10       _Ins_IUP                   10047d10 f   ttinterp.obj
 0001:00046f00       _Ins_MDRP                  10047f00 f   ttinterp.obj
 0001:00047180       _Ins_MIRP                  10048180 f   ttinterp.obj
 0001:000473a0       _Ins_SHPIX                 100483a0 f   ttinterp.obj
 0001:00047560       _Ins_SxVTL                 10048560 f   ttinterp.obj
 0001:000475f0       _Ins_UNKNOWN               100485f0 f   ttinterp.obj
 0001:00047690       _Modify_CVT_Check          10048690 f   ttinterp.obj
 0001:00047740       _Move_CVT                  10048740 f   ttinterp.obj
 0001:00047770       _Move_CVT_Stretched        10048770 f   ttinterp.obj
 0001:000477b0       _Normalize                 100487b0 f   ttinterp.obj
 0001:00047810       _Project                   10048810 f   ttinterp.obj
 0001:00047840       _Project_x                 10048840 f   ttinterp.obj
 0001:00047850       _Project_y                 10048850 f   ttinterp.obj
 0001:00047860       _Read_CVT                  10048860 f   ttinterp.obj
 0001:00047880       _Read_CVT_Stretched        10048880 f   ttinterp.obj
 0001:000478e0       _Round_Down_To_Grid        100488e0 f   ttinterp.obj
 0001:00047920       _Round_None                10048920 f   ttinterp.obj
 0001:00047950       _Round_Super               10048950 f   ttinterp.obj
 0001:000479b0       _Round_Super_45            100489b0 f   ttinterp.obj
 0001:00047a20       _Round_To_Double_Grid      10048a20 f   ttinterp.obj
 0001:00047a60       _Round_To_Grid             10048a60 f   ttinterp.obj
 0001:00047aa0       _Round_To_Half_Grid        10048aa0 f   ttinterp.obj
 0001:00047ae0       _Round_Up_To_Grid          10048ae0 f   ttinterp.obj
 0001:00047b20       _SetSuperRound             10048b20 f   ttinterp.obj
 0001:00047bec       $LN18                      10048bec     ttinterp.obj
 0001:00047bfc       $LN17                      10048bfc     ttinterp.obj
 0001:00047cc0       $LN20                      10048cc0     ttinterp.obj
 0001:00047cd4       $LN19                      10048cd4     ttinterp.obj
 0001:00047d10       _SkipCode                  10048d10 f   ttinterp.obj
 0001:00047e80       _TT_DotFix14               10048e80 f   ttinterp.obj
 0001:00048250       _TT_MulFix14               10049250 f   ttinterp.obj
 0001:0004ae60       $LN1110                    1004be60     ttinterp.obj
 0001:0004ae80       $LN1111                    1004be80     ttinterp.obj
 0001:0004b2c0       _Write_CVT                 1004c2c0 f   ttinterp.obj
 0001:0004b2f0       _Write_CVT_Stretched       1004c2f0 f   ttinterp.obj
 0001:0004b330       __iup_worker_interpolate   1004c330 f   ttinterp.obj
 0001:0004b930       _check_table_dir           1004c930 f   ttload.obj
 0001:0004c8c0       _tt_check_trickyness_sfnt_ids 1004d8c0 f   ttobjs.obj
 0001:0004cf70       _tt_size_done_bytecode     1004df70 f   ttobjs.obj
 0001:0004d0a0       _tt_size_init_bytecode     1004e0a0 f   ttobjs.obj
 0001:0004db90       _compare_ppem              1004eb90 f   ttpload.obj
 0001:0004e240       _load_format_20            1004f240 f   ttpost.obj
 0001:0004e4d0       _load_post_names           1004f4d0 f   ttpost.obj
 0001:0004eec0       _tt_face_load_sbix_image   1004fec0 f   ttsbit.obj
 0001:0004f380       _tt_sbit_decoder_load_bit_aligned 10050380 f   ttsbit.obj
 0001:0004f600       _tt_sbit_decoder_load_bitmap 10050600 f   ttsbit.obj
 0001:0004f848       $LN45                      10050848     ttsbit.obj
 0001:0004f854       $LN44                      10050854     ttsbit.obj
 0001:0004f868       $LN47                      10050868     ttsbit.obj
 0001:0004f884       $LN46                      10050884     ttsbit.obj
 0001:0004f898       $LN49                      10050898     ttsbit.obj
 0001:0004f8b0       $LN48                      100508b0     ttsbit.obj
 0001:0004f8d0       _tt_sbit_decoder_load_byte_aligned 100508d0 f   ttsbit.obj
 0001:0004fa80       _tt_sbit_decoder_load_compound 10050a80 f   ttsbit.obj
 0001:0004fbb0       _tt_sbit_decoder_load_image 10050bb0 f   ttsbit.obj
 0001:0004ff30       $LN72                      10050f30     ttsbit.obj
 0001:0004ff48       $LN71                      10050f48     ttsbit.obj
 0001:0004ff60       _tt_sbit_decoder_load_metrics 10050f60 f   ttsbit.obj
 0001:00050010       $$000000                   10051010     MSVCRT:chkstk.obj
 0001:00050040       $$000000                   10051040     MSVCRT:llmul.obj
 0001:00050080       $$000000                   10051080     MSVCRT:ulldiv.obj
 0001:000500f0       $$000000                   100510f0     MSVCRT:lldiv.obj
 0001:000501a0       $$000000                   100511a0     MSVCRT:llshl.obj
 0001:000503ba       ?dllmain_crt_dispatch@@YGHQAUHINSTANCE__@@KQAX@Z 100513ba f   MSVCRT:dll_dllmain.obj
 0001:0005040d       ?dllmain_crt_process_attach@@YAHQAUHINSTANCE__@@QAX@Z 1005140d f   MSVCRT:dll_dllmain.obj
 0001:00050514       ?dllmain_crt_process_detach@@YAH_N@Z 10051514 f   MSVCRT:dll_dllmain.obj
 0001:000505c4       ?dllmain_dispatch@@YAHQAUHINSTANCE__@@KQAX@Z 100515c4 f   MSVCRT:dll_dllmain.obj
 0001:000506cf       ?dllmain_raw@@YGHQAUHINSTANCE__@@KQAX@Z 100516cf f   MSVCRT:dll_dllmain.obj
 0001:0005071d       ___get_entropy             1005171d f   MSVCRT:gs_support.obj
 0001:00050818       ?find_pe_section@@YAPAU_IMAGE_SECTION_HEADER@@QAEI@Z 10051818 f   MSVCRT:utility.obj
 0001:00050c70       $$000000                   10051c70     MSVCRT:sehprolg4.obj
 0002:00002f9c       _af_service_properties     10054f9c     afmodule.obj
 0002:00002fa4       _af_services               10054fa4     afmodule.obj
 0002:00003040       _afm_key_table             10055040     afmparse.obj
 0002:00004368       _cff_service_glyph_dict    10056368     cffdrivr.obj
 0002:00004370       _cff_service_ps_info       10056370     cffdrivr.obj
 0002:00004384       _cff_service_ps_name       10056384     cffdrivr.obj
 0002:00004388       _cff_service_get_cmap_info 10056388     cffdrivr.obj
 0002:0000438c       _cff_service_cid_info      1005638c     cffdrivr.obj
 0002:00004398       _cff_service_properties    10056398     cffdrivr.obj
 0002:000043a0       _cff_service_multi_masters 100563a0     cffdrivr.obj
 0002:000043d0       _cff_service_metrics_variations 100563d0     cffdrivr.obj
 0002:000043f0       _cff_service_cff_load      100563f0     cffdrivr.obj
 0002:00004408       _cff_services              10056408     cffdrivr.obj
 0002:00004510       _cff_isoadobe_charset      10056510     cffload.obj
 0002:000046e0       _cff_expert_charset        100566e0     cffload.obj
 0002:00004830       _cff_expertsubset_charset  10056830     cffload.obj
 0002:000048e0       _cff_standard_encoding     100568e0     cffload.obj
 0002:00004ae0       _cff_expert_encoding       10056ae0     cffload.obj
 0002:00004ce0       ?cff_header_fields@?1??cff_font_load@@9@9 10056ce0     cffload.obj
 0002:00004d20       _power_tens                10056d20     cffparse.obj
 0002:00004d48       _power_ten_limits          10056d48     cffparse.obj
 0002:00004d70       _cff_field_handlers        10056d70     cffparse.obj
 0002:000055e0       _cid_field_records         100575e0     cidload.obj
 0002:00005fa0       _cid_service_ps_name       10057fa0     cidriver.obj
 0002:00005fa4       _cid_service_ps_info       10057fa4     cidriver.obj
 0002:00005fb8       _cid_service_cid_info      10057fb8     cidriver.obj
 0002:00005fc4       _cid_service_properties    10057fc4     cidriver.obj
 0002:00005fcc       _cid_services              10057fcc     cidriver.obj
 0002:00006074       _bbox_interface            10058074     ftbbox.obj
 0002:000060a0       _null_bitmap               100580a0     ftbitmap.obj
 0002:000060f8       _func_interface            100580f8     ftgrays.obj
 0002:00006128       _ft_default_modules        10058128     ftinit.obj
 0002:000061c0       _null_outline              100581c0     ftoutln.obj
 0002:00006258       _ft_raccess_guess_table    10058258     ftrfork.obj
 0002:00006338       _ft_trig_arctan_table      10058338     fttrigon.obj
 0002:00006478       _psaux_interface           10058478     psauxmod.obj
 0002:000064a8       _ft_char_table             100584a8     psconv.obj
 0002:0000654c       _pshinter_interface        1005854c     pshmod.obj
 0002:00006558       ?readFromStack@?DP@??cf2_interpT2CharString@@9@9 10058558     psintrp.obj
 0002:00006564       ?readFromStack@?EB@??cf2_interpT2CharString@@9@9 10058564     psintrp.obj
 0002:00006570       ?readFromStack@?ED@??cf2_interpT2CharString@@9@9 10058570     psintrp.obj
 0002:0000657c       ?readFromStack@?EF@??cf2_interpT2CharString@@9@9 1005857c     psintrp.obj
 0002:000157f8       _ft_extra_glyph_unicodes   100677f8     psmodule.obj
 0002:00015820       _ft_extra_glyph_names      10067820     psmodule.obj
 0002:00015878       _ft_extra_glyph_name_offsets 10067878     psmodule.obj
 0002:000158a0       _pscmaps_interface         100678a0     psmodule.obj
 0002:000158c0       _pscmaps_services          100678c0     psmodule.obj
 0002:000158fc       _sfnt_service_sfnt_table   100678fc     sfdriver.obj
 0002:00015908       _sfnt_service_glyph_dict   10067908     sfdriver.obj
 0002:00015910       _sfnt_ps_map               10067910     sfdriver.obj
 0002:00015920       _hexdigits                 10067920     sfdriver.obj
 0002:00015930       _sfnt_service_ps_name      10067930     sfdriver.obj
 0002:00015934       _tt_service_get_cmap_info  10067934     sfdriver.obj
 0002:00015938       _sfnt_services             10067938     sfdriver.obj
 0002:00015960       _sfnt_interface            10067960     sfdriver.obj
 0002:00015a18       ?tt_encodings@?1??sfnt_find_encoding@@9@9 10067a18     sfobjs.obj
 0002:00015a9c       ?ttc_header_fields@?1??sfnt_open_font@@9@9 10067a9c     sfobjs.obj
 0002:00015b50       _t1_args_count             10067b50     t1decode.obj
 0002:00015bc0       _t1_service_glyph_dict     10067bc0     t1driver.obj
 0002:00015bc8       _t1_service_ps_name        10067bc8     t1driver.obj
 0002:00015bcc       _t1_service_multi_masters  10067bcc     t1driver.obj
 0002:00015bfc       _t1_service_ps_info        10067bfc     t1driver.obj
 0002:00015c10       _t1_service_kerning        10067c10     t1driver.obj
 0002:00015c14       _t1_service_properties     10067c14     t1driver.obj
 0002:00015c20       _t1_services               10067c20     t1driver.obj
 0002:00015cc0       _t1_keywords               10067cc0     t1load.obj
 0002:00016650       _tt_cmap_classes           10068650     ttcmap.obj
 0002:000166d8       _tt_service_properties     100686d8     ttdriver.obj
 0002:000166e0       _tt_service_gx_multi_masters 100686e0     ttdriver.obj
 0002:00016710       _tt_service_metrics_variations 10068710     ttdriver.obj
 0002:00016730       _tt_service_truetype_engine 10068730     ttdriver.obj
 0002:00016734       _tt_service_truetype_glyf  10068734     ttdriver.obj
 0002:00016738       _tt_services               10068738     ttdriver.obj
 0002:00016798       ?gvar_fields@?1??ft_var_load_gvar@@9@9 10068798     ttgxvar.obj
 0002:000167bc       ?fvar_fields@?1??TT_Get_MM_Var@@9@9 100687bc     ttgxvar.obj
 0002:000167e0       ?fvaraxis_fields@?1??TT_Get_MM_Var@@9@9 100687e0     ttgxvar.obj
 0002:00016850       _Pop_Push_Count            10068850     ttinterp.obj
 0002:00016950       _opcode_length             10068950     ttinterp.obj
 0002:00016a50       ?table_dir_entry_fields@?1??check_table_dir@@9@9 10068a50     ttload.obj
 0002:00016a68       ?offset_table_fields@?1??tt_face_load_font_dir@@9@9 10068a68     ttload.obj
 0002:00016a80       ?header_fields@?1??tt_face_load_generic_header@@9@9 10068a80     ttload.obj
 0002:00016ad4       ?maxp_fields@?1??tt_face_load_maxp@@9@9 10068ad4     ttload.obj
 0002:00016ae4       ?maxp_fields_extra@?1??tt_face_load_maxp@@9@9 10068ae4     ttload.obj
 0002:00016b20       ?name_table_fields@?1??tt_face_load_name@@9@9 10068b20     ttload.obj
 0002:00016b34       ?name_record_fields@?1??tt_face_load_name@@9@9 10068b34     ttload.obj
 0002:00016b50       ?langTag_record_fields@?1??tt_face_load_name@@9@9 10068b50     ttload.obj
 0002:00016b5c       ?os2_fields_extra2@?1??tt_face_load_os2@@9@9 10068b5c     ttload.obj
 0002:00016b78       ?os2_fields@?1??tt_face_load_os2@@9@9 10068b78     ttload.obj
 0002:00016c28       ?os2_fields_extra1@?1??tt_face_load_os2@@9@9 10068c28     ttload.obj
 0002:00016c38       ?os2_fields_extra5@?1??tt_face_load_os2@@9@9 10068c38     ttload.obj
 0002:00016c48       ?post_fields@?1??tt_face_load_post@@9@9 10068c48     ttload.obj
 0002:00016c78       ?pclt_fields@?1??tt_face_load_pclt@@9@9 10068c78     ttload.obj
 0002:00016cc0       ?metrics_header_fields@?1??tt_face_load_hhea@@9@9 10068cc0     ttmtx.obj
 0002:00016d10       ?trick_names@?1??tt_check_trickyness_family@@9@9 10068d10     ttobjs.obj
 0002:00016ea0       ?sfnt_id@?1??tt_check_trickyness_sfnt_ids@@9@9 10068ea0     ttobjs.obj
 0002:00017188       _GS_ExceptionPointers      10069188     MSVCRT:gs_report.obj
 0002:00017560       __sehtable$?dllmain_crt_process_attach@@YAHQAUHINSTANCE__@@QAX@Z 10069560     MSVCRT:dll_dllmain.obj
 0002:00017580       __sehtable$?dllmain_crt_process_detach@@YAH_N@Z 10069580     MSVCRT:dll_dllmain.obj
 0002:000175a8       __sehtable$?dllmain_dispatch@@YAHQAUHINSTANCE__@@KQAX@Z 100695a8     MSVCRT:dll_dllmain.obj
 0002:000175c8       __sehtable$___scrt_is_nonwritable_in_current_image 100695c8     MSVCRT:utility.obj
 0002:000175f0       .edata                     100695f0     freetype.exp
 0002:00017618       rgpv                       10069618     freetype.exp
 0002:000178f0       rgszName                   100698f0     freetype.exp
 0002:00017bc8       rgwOrd                     10069bc8     freetype.exp
 0002:00017d34       szName                     10069d34     freetype.exp
 0002:00017d41       $N00001                    10069d41     freetype.exp
 0002:00017d52       $N00002                    10069d52     freetype.exp
 0002:00017d69       $N00003                    10069d69     freetype.exp
 0002:00017d77       $N00004                    10069d77     freetype.exp
 0002:00017d85       $N00005                    10069d85     freetype.exp
 0002:00017d8e       $N00006                    10069d8e     freetype.exp
 0002:00017d9d       $N00007                    10069d9d     freetype.exp
 0002:00017dae       $N00008                    10069dae     freetype.exp
 0002:00017dbe       $N00009                    10069dbe     freetype.exp
 0002:00017dd0       $N00010                    10069dd0     freetype.exp
 0002:00017ddf       $N00011                    10069ddf     freetype.exp
 0002:00017dee       $N00012                    10069dee     freetype.exp
 0002:00017e01       $N00013                    10069e01     freetype.exp
 0002:00017e10       $N00014                    10069e10     freetype.exp
 0002:00017e1e       $N00015                    10069e1e     freetype.exp
 0002:00017e29       $N00016                    10069e29     freetype.exp
 0002:00017e30       $N00017                    10069e30     freetype.exp
 0002:00017e3a       $N00018                    10069e3a     freetype.exp
 0002:00017e47       $N00019                    10069e47     freetype.exp
 0002:00017e58       $N00020                    10069e58     freetype.exp
 0002:00017e66       $N00021                    10069e66     freetype.exp
 0002:00017e76       $N00022                    10069e76     freetype.exp
 0002:00017e85       $N00023                    10069e85     freetype.exp
 0002:00017e92       $N00024                    10069e92     freetype.exp
 0002:00017eaf       $N00025                    10069eaf     freetype.exp
 0002:00017ecb       $N00026                    10069ecb     freetype.exp
 0002:00017eeb       $N00027                    10069eeb     freetype.exp
 0002:00017f05       $N00028                    10069f05     freetype.exp
 0002:00017f21       $N00029                    10069f21     freetype.exp
 0002:00017f3b       $N00030                    10069f3b     freetype.exp
 0002:00017f4e       $N00031                    10069f4e     freetype.exp
 0002:00017f6b       $N00032                    10069f6b     freetype.exp
 0002:00017f77       $N00033                    10069f77     freetype.exp
 0002:00017f86       $N00034                    10069f86     freetype.exp
 0002:00017f96       $N00035                    10069f96     freetype.exp
 0002:00017fb2       $N00036                    10069fb2     freetype.exp
 0002:00017fd5       $N00037                    10069fd5     freetype.exp
 0002:00017ffd       $N00038                    10069ffd     freetype.exp
 0002:00018010       $N00039                    1006a010     freetype.exp
 0002:00018028       $N00040                    1006a028     freetype.exp
 0002:0001803a       $N00041                    1006a03a     freetype.exp
 0002:0001804f       $N00042                    1006a04f     freetype.exp
 0002:0001806a       $N00043                    1006a06a     freetype.exp
 0002:00018083       $N00044                    1006a083     freetype.exp
 0002:0001809c       $N00045                    1006a09c     freetype.exp
 0002:000180b3       $N00046                    1006a0b3     freetype.exp
 0002:000180c7       $N00047                    1006a0c7     freetype.exp
 0002:000180d9       $N00048                    1006a0d9     freetype.exp
 0002:000180ec       $N00049                    1006a0ec     freetype.exp
 0002:000180f8       $N00050                    1006a0f8     freetype.exp
 0002:00018105       $N00051                    1006a105     freetype.exp
 0002:00018117       $N00052                    1006a117     freetype.exp
 0002:00018126       $N00053                    1006a126     freetype.exp
 0002:00018142       $N00054                    1006a142     freetype.exp
 0002:00018150       $N00055                    1006a150     freetype.exp
 0002:00018167       $N00056                    1006a167     freetype.exp
 0002:00018175       $N00057                    1006a175     freetype.exp
 0002:00018189       $N00058                    1006a189     freetype.exp
 0002:0001819b       $N00059                    1006a19b     freetype.exp
 0002:000181ac       $N00060                    1006a1ac     freetype.exp
 0002:000181c0       $N00061                    1006a1c0     freetype.exp
 0002:000181d7       $N00062                    1006a1d7     freetype.exp
 0002:000181ec       $N00063                    1006a1ec     freetype.exp
 0002:000181f9       $N00064                    1006a1f9     freetype.exp
 0002:0001820d       $N00065                    1006a20d     freetype.exp
 0002:00018224       $N00066                    1006a224     freetype.exp
 0002:00018234       $N00067                    1006a234     freetype.exp
 0002:00018248       $N00068                    1006a248     freetype.exp
 0002:00018259       $N00069                    1006a259     freetype.exp
 0002:00018270       $N00070                    1006a270     freetype.exp
 0002:00018282       $N00071                    1006a282     freetype.exp
 0002:00018297       $N00072                    1006a297     freetype.exp
 0002:000182ac       $N00073                    1006a2ac     freetype.exp
 0002:000182bd       $N00074                    1006a2bd     freetype.exp
 0002:000182d9       $N00075                    1006a2d9     freetype.exp
 0002:000182ef       $N00076                    1006a2ef     freetype.exp
 0002:0001830c       $N00077                    1006a30c     freetype.exp
 0002:0001832a       $N00078                    1006a32a     freetype.exp
 0002:00018341       $N00079                    1006a341     freetype.exp
 0002:00018357       $N00080                    1006a357     freetype.exp
 0002:0001836c       $N00081                    1006a36c     freetype.exp
 0002:00018384       $N00082                    1006a384     freetype.exp
 0002:00018392       $N00083                    1006a392     freetype.exp
 0002:000183a4       $N00084                    1006a3a4     freetype.exp
 0002:000183b4       $N00085                    1006a3b4     freetype.exp
 0002:000183ca       $N00086                    1006a3ca     freetype.exp
 0002:000183dd       $N00087                    1006a3dd     freetype.exp
 0002:000183f0       $N00088                    1006a3f0     freetype.exp
 0002:00018406       $N00089                    1006a406     freetype.exp
 0002:00018417       $N00090                    1006a417     freetype.exp
 0002:0001842f       $N00091                    1006a42f     freetype.exp
 0002:0001844e       $N00092                    1006a44e     freetype.exp
 0002:00018468       $N00093                    1006a468     freetype.exp
 0002:0001847b       $N00094                    1006a47b     freetype.exp
 0002:00018487       $N00095                    1006a487     freetype.exp
 0002:00018498       $N00096                    1006a498     freetype.exp
 0002:000184a5       $N00097                    1006a4a5     freetype.exp
 0002:000184b4       $N00098                    1006a4b4     freetype.exp
 0002:000184c4       $N00099                    1006a4c4     freetype.exp
 0002:000184d3       $N00100                    1006a4d3     freetype.exp
 0002:000184de       $N00101                    1006a4de     freetype.exp
 0002:000184eb       $N00102                    1006a4eb     freetype.exp
 0002:000184f9       $N00103                    1006a4f9     freetype.exp
 0002:0001850c       $N00104                    1006a50c     freetype.exp
 0002:0001851d       $N00105                    1006a51d     freetype.exp
 0002:00018530       $N00106                    1006a530     freetype.exp
 0002:0001853a       $N00107                    1006a53a     freetype.exp
 0002:00018544       $N00108                    1006a544     freetype.exp
 0002:00018550       $N00109                    1006a550     freetype.exp
 0002:0001855d       $N00110                    1006a55d     freetype.exp
 0002:0001856c       $N00111                    1006a56c     freetype.exp
 0002:0001857f       $N00112                    1006a57f     freetype.exp
 0002:0001858b       $N00113                    1006a58b     freetype.exp
 0002:00018598       $N00114                    1006a598     freetype.exp
 0002:000185a9       $N00115                    1006a5a9     freetype.exp
 0002:000185b9       $N00116                    1006a5b9     freetype.exp
 0002:000185ce       $N00117                    1006a5ce     freetype.exp
 0002:000185de       $N00118                    1006a5de     freetype.exp
 0002:000185f2       $N00119                    1006a5f2     freetype.exp
 0002:00018608       $N00120                    1006a608     freetype.exp
 0002:00018623       $N00121                    1006a623     freetype.exp
 0002:0001863f       $N00122                    1006a63f     freetype.exp
 0002:00018653       $N00123                    1006a653     freetype.exp
 0002:00018669       $N00124                    1006a669     freetype.exp
 0002:0001867d       $N00125                    1006a67d     freetype.exp
 0002:00018698       $N00126                    1006a698     freetype.exp
 0002:000186a7       $N00127                    1006a6a7     freetype.exp
 0002:000186b9       $N00128                    1006a6b9     freetype.exp
 0002:000186cc       $N00129                    1006a6cc     freetype.exp
 0002:000186e1       $N00130                    1006a6e1     freetype.exp
 0002:000186f6       $N00131                    1006a6f6     freetype.exp
 0002:00018706       $N00132                    1006a706     freetype.exp
 0002:00018716       $N00133                    1006a716     freetype.exp
 0002:00018728       $N00134                    1006a728     freetype.exp
 0002:0001873d       $N00135                    1006a73d     freetype.exp
 0002:0001874e       $N00136                    1006a74e     freetype.exp
 0002:0001875e       $N00137                    1006a75e     freetype.exp
 0002:0001876e       $N00138                    1006a76e     freetype.exp
 0002:0001877a       $N00139                    1006a77a     freetype.exp
 0002:0001878c       $N00140                    1006a78c     freetype.exp
 0002:0001879b       $N00141                    1006a79b     freetype.exp
 0002:000187ac       $N00142                    1006a7ac     freetype.exp
 0002:000187bb       $N00143                    1006a7bb     freetype.exp
 0002:000187cd       $N00144                    1006a7cd     freetype.exp
 0002:000187e8       $N00145                    1006a7e8     freetype.exp
 0002:00018802       $N00146                    1006a802     freetype.exp
 0002:00018815       $N00147                    1006a815     freetype.exp
 0002:00018831       $N00148                    1006a831     freetype.exp
 0002:0001884e       $N00149                    1006a84e     freetype.exp
 0002:00018865       $N00150                    1006a865     freetype.exp
 0002:0001887b       $N00151                    1006a87b     freetype.exp
 0002:0001888e       $N00152                    1006a88e     freetype.exp
 0002:0001889e       $N00153                    1006a89e     freetype.exp
 0002:000188af       $N00154                    1006a8af     freetype.exp
 0002:000188cc       $N00155                    1006a8cc     freetype.exp
 0002:000188ea       $N00156                    1006a8ea     freetype.exp
 0002:000188fd       $N00157                    1006a8fd     freetype.exp
 0002:00018904       $N00158                    1006a904     freetype.exp
 0002:0001891c       $N00159                    1006a91c     freetype.exp
 0002:0001892f       $N00160                    1006a92f     freetype.exp
 0002:00018942       $N00161                    1006a942     freetype.exp
 0002:00018952       $N00162                    1006a952     freetype.exp
 0002:00018968       $N00163                    1006a968     freetype.exp
 0002:0001897a       $N00164                    1006a97a     freetype.exp
 0002:00018992       $N00165                    1006a992     freetype.exp
 0002:000189ad       $N00166                    1006a9ad     freetype.exp
 0002:000189c2       $N00167                    1006a9c2     freetype.exp
 0002:000189d4       $N00168                    1006a9d4     freetype.exp
 0002:000189e3       $N00169                    1006a9e3     freetype.exp
 0002:000189fb       $N00170                    1006a9fb     freetype.exp
 0002:00018a0d       $N00171                    1006aa0d     freetype.exp
 0002:00018a1c       $N00172                    1006aa1c     freetype.exp
 0002:00018a23       $N00173                    1006aa23     freetype.exp
 0002:00018a3e       $N00174                    1006aa3e     freetype.exp
 0002:00018a51       $N00175                    1006aa51     freetype.exp
 0002:00018a66       $N00176                    1006aa66     freetype.exp
 0002:00018a77       $N00177                    1006aa77     freetype.exp
 0002:00018a8a       $N00178                    1006aa8a     freetype.exp
 0002:00018a9b       $N00179                    1006aa9b     freetype.exp
 0002:00018aaf       $N00180                    1006aaaf     freetype.exp
 0002:00018abe       $N00181                    1006aabe     freetype.exp
 0002:00018acd       $N00182                    1006aacd     freetype.exp
 0002:00018d94       .idata$6                   1006ad94     kernel32:KERNEL32.dll
 0002:00018e2e       .idata$6                   1006ae2e     vcruntime:VCRUNTIME140.dll
 0002:00018f5c       .idata$6                   1006af5c     ucrt:api-ms-win-crt-convert-l1-1-0.dll
 0002:00018f7e       .idata$6                   1006af7e     ucrt:api-ms-win-crt-string-l1-1-0.dll
 0002:00018fa0       .idata$6                   1006afa0     ucrt:api-ms-win-crt-utility-l1-1-0.dll
 0002:00018fc2       .idata$6                   1006afc2     ucrt:api-ms-win-crt-environment-l1-1-0.dll
 0002:00018fe8       .idata$6                   1006afe8     ucrt:api-ms-win-crt-stdio-l1-1-0.dll
 0002:00019008       .idata$6                   1006b008     ucrt:api-ms-win-crt-heap-l1-1-0.dll
 0002:00019028       .idata$6                   1006b028     ucrt:api-ms-win-crt-runtime-l1-1-0.dll
 0003:00000028       _GS_ExceptionRecord        1006c028     MSVCRT:gs_report.obj
 0003:00000078       _GS_ContextRecord          1006c078     MSVCRT:gs_report.obj
 0003:00000344       ?__proc_attached@@3HA      1006c344     MSVCRT:dll_dllmain.obj
 0003:00000368       ?is_initialized_as_dll@@3_NA 1006c368     MSVCRT:utility.obj
 0003:00000369       ?module_local_atexit_table_initialized@@3_NA 1006c369     MSVCRT:utility.obj
 0003:0000036c       ?module_local_atexit_table@@3U_onexit_table_t@@A 1006c36c     MSVCRT:utility.obj
 0003:00000378       ?module_local_at_quick_exit_table@@3U_onexit_table_t@@A 1006c378     MSVCRT:utility.obj
 0004:00000060       $R000000                   1006d060     freetype.dll.res
